:020000040800F2
:1000000000000110B9BB030851D8020811D1000843
:10001000BDBC0308BDBC0308BDBC03080000000054
:1000200000000000000000000000000099DE02084F
:1000300095DE02080000000091DE020805E50008D8
:10004000BDBC0308BDBC0308BDBC0308BDBC0308A0
:10005000BDBC0308BDBC0308399B0008659C0008B3
:10006000299C0008ED9B0008B19B0008B9B6000868
:10007000A9B6000899B6000889B6000879B6000844
:1000800065B6000851B60008BDBC0308BDBC030836
:10009000BDBC0308BDBC0308BDBC0308759B0008BC
:1000A00099D5000809D60008BDBC030819D6000878
:1000B000F9D50008E9D50008D9D50008E1BE000847
:1000C000E9BE0008D5BE0008DDBE0008BDBC0308BF
:1000D000BDBC03087D910008E19000084590000830
:1000E000FD9A0008BDBC0308A9E90208BDBC0308CD
:1000F000A9D50008BDBC0308B9D500083DB6000865
:10010000BDBC0308BDBC0308C9D50008BDBC0308BD
:100110002DE60008BDBC030889BF01086DBF0108BA
:1001200029B6000815B6000801B60008EDB50008AC
:10013000D9B50008BDBC0308BDBC0308BDBC03089D
:10014000BDBC0308BDBC0308BDBC030855D80208EC
:10015000C5B50008B1B500089DB5000891E50008D7
:10016000C9BE0008D1BE0008BDBC0308BDBC030861
:10017000BDBC0308BDBC0308BDBC0308BDBC03086F
:08018000BDBC0308BDBC03086F
:1001880002020300C41E0020C01E00200000000060
:100198000000000016000800C81E0020D01E002025
:1001A80000000000FC0500080300010054240020A2
:1001B8005C24002000000000000000001D00010079
:1001C8006C240020FC240020000000000406000825
:1001D800270004008C2400200025002000000000D7
:1001E800060600080101040044250020203D0020E7
:1001F800000000000000000008020900F63B002093
:10020800243D0020000000002982000806020C009E
:100218006C3C0020303D002000000000758E000876
:1002280007020200A03C00203C3D00200000000026
:100238000A060008FF010100B43C0020403D0020F0
:10024800000000000C06000802000C00783C0020AA
:10025800443D00200000000000000000F7010600F7
:10026800F03B0020503D0020000000000E06000872
:100278000A020A00C8250020583D0020000000009E
:1002880014060008031233002F450020FC44002008
:10029800000000002006000825005A0048440020FD
:1002A800A24400200000000000000000F6110C002D
:1002B8003C440020304400200000000054060008A0
:1002C8000120080068450020B44500200000000017
:1002D800600600080902010078470020D047002086
:1002E800000000006806000812100C00EC46002010
:1002F800D4470020000000006A0600080C00240013
:10030800FC460020E0470020000000003DB6010840
:1003180000020500C4460020044800200000000038
:10032800000000001A000800B04F0020C84F00204D
:1003380000000000760600082A0060003050002007
:10034800D04F002000000000BD54020815007000C6
:100358003C490020905000200000000000000000F0
:10036800F9010400285D0020385D0020000000002D
:100378001182000818102C00F85C00203C5D002059
:10038800000000006D670308FB010100B45C002059
:10039800685D002000000000DDBF0008FC010900C6
:1003A800805B00206C5D002000000000A9BF0008F1
:1003B8000A101200545B0020785D00200000000045
:1003C8007E06000806001600245800208C5D0020D8
:1003D80000000000F953020829005000A86000201E
:1003E800FC60002000000000000000001400020073
:1003F800A46000204C610020000000009006000866
:1004080013000400986000205061002000000000E4
:100418009406000810000300946000205461002036
:10042800000000009806000828000C0088600020E2
:1004380058610020000000009C06000823001000FE
:10044800786000206461002000000000E17102086B
:100458001900050070600020746100200000000091
:10046800A8060008F81101006C6000207C610020DB
:1004780000000000AE0600080001040068600020CB
:100488008061002000000000B00600082F00110065
:10049800546000208461002000000000B4060008B9
:1004A8001F000E00DC620020FC620020000000003B
:1004B800C606000805020100C46200200C63002083
:1004C80000000000D4060008030106005662002060
:1004D8001063002000000000D60600081E0004007B
:1004E8009C6500208467002000000000DC060008EE
:1004F80022000C000865002088670020000000002A
:10050800E006000826000E00A4670020946700207B
:10051800000000008DFD0208340010008C6E0020E1
:100528005C6F002000000000B55302080D00440075
:10053800486E00206C6F0020000000009DEB010851
:10054800FD0124002C680020B06F0020000000008E
:10055800A1810008FE01080018680020D46F00205F
:100568000000000019C000080500060020710020E6
:100578006471002000000000EC0600080E20EA006C
:10058800047000206C71002000000000E55402088F
:1005980002010300F16F00205872002000000000E3
:1005A8006DB501080B201000B8740020F07400200D
:1005B80000000000F20600082C001000447700201C
:1005C8003477002000000000E96403082B002400B1
:1005D800787700205477002000000000B9640308F1
:1005E8000400800028A500205CA600200000000070
:0405F80000000000FF
:1005FC00C409000019012828000020030000013C58
:10060C00000055000100000000004A01B400D601B2
:10061C0000000000000000000000000000000000CE
:10062C0000000000000000000000000000000000BE
:10063C0000000000000000000000000000000000AE
:10064C00000000000000010000000000000000009D
:10065C0000000000E8036400040A00011000000020
:10066C00000100054634425900007E05EA05B40538
:10067C00320000300100005A0000000090012C01F3
:10068C00C800640003000000080000000001050021
:10069C000000000100000000000000000000280124
:1006AC0000000400900100000000000000000000A9
:1006BC00000000000000000000000000000000002E
:1006CC000100000000050000000004010100000012
:1006DC0000000100C800141E010064002C01280059
:1006EC002000020001002B21231E640102000000E7
:0606FC0001000A012900C3
:100702005001000007000000020000000000803FCE
:100712000000803F0000803F000000000000000059
:100722000102030406070809010100006814040815
:10073200A43F040800000000000000007814040830
:100742008014040800000000012000008414040842
:100752008C140408000000000140000090140408FA
:100762001829040800000000012000009C1404085D
:10077200A81404080000000004000000AC140408DF
:10078200B81404080000000004000000BC140408AF
:100792005C38040800000000010000000201FF00B4
:1007A2000000803F0000803F60EA03080508040063
:1007B20000000000600B0408FC0A04084CEA03086D
:1007C200000000008CEA030805080A00000000008F
:1007D200600B0408FC0A0408800B040800000000F7
:1007E200F1AB0208A9AB0208F9AA02080000000056
:1007F20065A802084DAA0208CDAA0208B5A90208F6
:10080200000000000000000059A8020851D60208AA
:100812004DD6020849D602083DD6020839D602084A
:1008220045D6020841D6020861D6020855D602080A
:10083200E5D60208F9D60208D1D60208BDD60208CA
:10084200A9D602080000803FFFFFFFFF0101000060
:1008520000010101617702080000000000000000B1
:100862000100000000600240106002400000000031
:10087200000B00000000200000000000000000004B
:10088200006002402860024000000000060C0000E8
:100892000000200000000000000000000060024094
:1008A2004060024000000000100D00000000200027
:1008B200000000000000000000600240586002409A
:1008C20000000000160E00000000200000000000E2
:1008D2000000000000600240706002400000000062
:1008E200200F0000000020000000000000000000B7
:1008F20000600240886002400000000026100000F4
:100902000000200000000000000000000060024023
:10091200A060024000000000301100000000200032
:10092200000000000000000000600240B8600240C9
:1009320000000000362F0000000020000000000030
:100942000000000000640240106402400000000049
:10095200003800000000400000000000000000001D
:1009620000640240286402400000000006390000D2
:10097200000040000000000000000000006402408F
:100982004064024000000000103A000000004000F5
:1009920000000000000000000064024058640240B1
:1009A20000000000163B00000000400000000000B4
:1009B2000000000000640240706402400000000079
:1009C200203C000000004000000000000000000089
:1009D20000640240886402400000000026440000D7
:1009E200000040000000000000000000006402401F
:1009F200A0640240000000003045000000004000FA
:100A0200000000000000000000640240B8640240E0
:100A12000000000036460000000040000000000018
:100A2200000000000100000009024300020100C0B2
:100A32003209040000010202010005240010010530
:100A42002401000104240202052406000107058294
:100A5200030800FF09040100020A00000007050163
:100A6200024000000705810240000000FF00000074
:100A7200303030302D30312D30315430303A30304A
:100A82003A3030000403090412010002020200405D
:100A9200830440570002010203010000B9AD0208BD
:100AA200D9AC0208813E0308A9A8020885AC020855
:100AB200B9A80208D5A8020899A8020889A80208BC
:100AC200000000000000000000FFFF000000000026
:100AD200AA5503009FAA5505010000AA5507010067
:100AE2000001AA550B010000AA55090200000000EE
:100AF20001000000C0120000D02F04080000000016
:100B0200000000007DB50108A0860100040000007D
:100B120000000000000000000000000000000000D3
:100B2200000000000000000000000000FC4004087B
:100B3200202F0408000000003D4A01087D0000004B
:100B4200060000000000000000000000000000009D
:100B52000000000000000000000000000000000093
:100B6200AC4204080000000000000000419E03089F
:100B7200E803000003000000000000000000000085
:100B82000000000000000000000000000000000063
:100B920000000000B4420408000000000000000051
:100BA200890802081027000003000000000000006E
:100BB2000000000000000000000000000000000033
:100BC20000000000000000009C4604080000000035
:100BD2006D790208C5280108204E000005000000BA
:100BE2000000000000000000000000000000000003
:100BF2000000000000000000000000004431040872
:100C02000000000000000000FD980308102700000B
:100C120001000000000000000000000000000000D1
:100C220000000000000000000000000000000000C2
:100C3200C0420408000000000000000075BF000868
:100C4200E8030000050000000000000000000000B2
:100C52000000000000000000000000000000000092
:100C620000000000CC420408000000000000000068
:100C72005DB80108204E00000300000000000000E3
:100C82000000000000000000000000000000000062
:100C92000000000000000000DC4204080000000028
:100CA2000000000065B60108204E000003000000AD
:100CB2000000000000000000000000000000000032
:100CC200000000000000000000000000EC420408E8
:100CD2000000000000000000CD470108400D0300A5
:100CE20003000000000000000000000000000000FF
:100CF20000000000000000000000000000000000F2
:100D0200843004080000000000000000C103020853
:100D12001027000001000000000000000000000099
:100D220000000000000000000000000000000000C1
:100D3200000000003C2F040800000000000000003A
:100D4200D53D02081027000003000000000000004B
:100D52000000000000000000000000000000000091
:100D62000000000000000000FC4204080000000037
:100D720000000000F5AF0308A0860100010000009A
:100D82000000000000000000000000000000000061
:100D92000000000000000000000000002C2F0408EA
:100DA200000000000000000015AF030850C300005F
:100DB2000100000000000000000000000000000030
:100DC2000000000000000000000000000000000021
:100DD2000443040800000000000000007DAA03088C
:100DE200A8610000010000000000000000000000F7
:100DF20000000000000000000000000000000000F1
:100E02000000000010430408000000000000000081
:100E1200F1480208A0860100010000000000000065
:100E220000000000000000000000000000000000C0
:100E320000000000000000004C3104080000000027
:100E420000000000C9E60008A00F00000100000039
:100E52000000000000000000000000000000000090
:100E6200000000000000000000000000B031040893
:100E72000000000000000000F9EC0208102700004A
:100E8200010000000000000000000000000000005F
:100E92000000000000000000000000000000000050
:100EA200142F04080000000000000000B1590308DC
:100EB2001A410000010000000000000000000000D4
:100EC2000000000000000000000000000000000020
:100ED200000000001C4304080000000000000000A5
:100EE20079EB0108400D0300000000000000000043
:100EF20000000000000000000000000000000000F0
:100F0200000000000000000024430408000000006C
:100F12000000000035EB0108400D03000000000056
:100F220000000000000000000000000000000000BF
:100F32000000000000000000000000002C43040834
:100F4200000000000000000009EC0108A08601007A
:100F5200030000000000000000000000000000008C
:100F6200000000000000000000000000000000007F
:100F72000000803F01010100404504080E0000000E
:100F82004D2903080000000000000000F8090020BD
:100F920004450408000000000000000000000000FA
:100FA20000000000A43F0408000000000000000050
:100FB200840A002004000000904404080C00000091
:100FC20051310308980E002000000000B4430408C9
:100FD2000C000000213103088C0E002000000000EC
:100FE200244504080800000000000000800E0020D4
:100FF20004000000144504080C0000003930030806
:10100200740E002000000000A0430408030000004A
:101012007D5803085C0E0020000000001C450408F7
:10102200030000007D580308440E00200000000069
:10103200A4430408010000000000000000000000BA
:1010420000000000000000000D0000000000000091
:101052000000000000000000044504080000000039
:10106200000000000000000000000000A43F04088F
:101072000000000000000000840A002004000000BC
:101082003444040803000000052F03082C0E00203E
:1010920008000000144504080C0000003930030861
:1010A200740E002000000000A043040803000000AA
:1010B2007D5803085C0E0020000000001C45040857
:1010C200030000007D580308440E002000000000C9
:1010D200A44304080100000000000000000000001A
:1010E20000000000000000000D00000000000000F1
:1010F20000000000000000002C4504080000000071
:10110200000000000000000000000000A43F0408EE
:101112000000000000000000840A0020040000001B
:101122003C440408030000007D580308A40E00207C
:1011320000000000A44304080100000000000000B9
:101142000000000000000000000000000D00000090
:1011520000000000000000000000000020700020DD
:10116200702D72002D202D2D202D2D2D2D202D2D79
:101172002D2D000000000000000000000000000013
:10118200000000002D202D2D202D2D2D2D202D2D68
:101192002D00000000000000000000000000000020
:1011A20000000000EA6F002088130C170100000005
:1011B200EC6F002088130C1700000000784304082D
:1011C200000000000000000000000000000000001D
:1011D200884304080800000000000000B00A002054
:1011E200040000009443040808000000000000000E
:1011F200A40A002000000000A0430408040000002C
:101202001D3003080000000000000000A443040891
:1012120001000000000000000000000000000000CB
:10122200000000000D0000000000000000000000AF
:1012320000000000E86F002088130C170100000076
:10124200E66F002088130C1700000000E443040836
:101252000E000000A52903080000000000000000A5
:10126200BC0A00205271002001000000200B04087B
:10127200E56F0020010000002C0B0408C062002072
:1012820002000000340B0408EEA50020000000005C
:1012920000000000ECA5002000000000000000009B
:1012A200EAA500200000000000000000E8A50020E0
:1012B2000000000000000000E6A500200000000081
:1012C20000000000E4A50020000000000000000073
:1012D200F40300200000000000000000E46F002082
:1012E20002000000400B0408EC4304080000000068
:1012F2000000000000000000000000008843040815
:101302000800000000000000400B00200400000064
:10131200944304080800000000000000340B002081
:1013220000000000A043040804000000852903080F
:101332000000000000000000A443040801000000B7
:10134200000000000000000000000000000000009B
:101352000D0000000000000000000000000000007E
:10136200FC43040800000000000000000000000030
:10137200000000000C4404080C000000C130030807
:101382007C0B002004000000184404080C0000003C
:10139200C9290308700B002004000000244404083B
:1013A2000C00000081300308640B002000000000E4
:1013B2003044040803000000252F03084C0B0020D2
:1013C200080000003C440408030000007D580308A4
:1013D200A40E002000000000A44304080100000045
:1013E20000000000000000000000000000000000FB
:1013F2000D000000000000000000000000000000DE
:101402004444040800000000000000000000000046
:10141200000000004C44040804000000813103086D
:101422000000000000000000A443040801000000C6
:1014320000000000000000000000000000000000AA
:101442000D0000000000000000000000000000008D
:1014520098440408000000000000000000000000A2
:1014620000000000443204080C00000000000000EC
:10147200DC0B002004000000A8440408080000005F
:1014820000000000D00B002004000000B444040857
:101492000800000000000000C40B0020040000004F
:1014A200BC4404080800000000000000B80B002043
:1014B20004000000C444040808000000000000000A
:1014C200AC0B002004000000CC440408080000001B
:1014D20000000000A00B002004000000D444040817
:1014E2000800000000000000940B0020040000002F
:1014F200DC4404080800000000000000880B002003
:1015020004000000A44304080100000000000000E1
:101512000000000000000000000000000D000000BC
:10152200000000000000000000000000E444040885
:101532000E000000952903080000000000000000D2
:10154200E80B0020EC4404080E000000000000003C
:101552000000000000000000600C0020F4440408B9
:101562000E0000000000000000000000000000006B
:10157200000D002051710020040000004C0B0408F3
:10158200E06F0020E0150C1700000000E36F002060
:1015920008000000FC0A0408E26F002005000000B9
:1015A200600B0408FC4404080E0000000000000068
:1015B2000000000000000000500D002000000000AC
:1015C2000102030401020304060708099C4A0408F5
:1015D2000E000000000000000000000000000000FB
:1015E200241C0020FFFFFFFFFA00000001000000A2
:1015F2000100000044440408000000000000000054
:1016020000000000000000006A4504080400000019
:10161200972E03080000000000000000A443040805
:1016220001000000000000000000000000000000B7
:10163200000000000D00000000000000000000009B
:101642000000000012A600200100C40900000000F2
:1016520010A600200100C409000000000EA6002010
:101662000100C409000000000CA600200100C4090A
:101672000000000008A600200100C40900000000CC
:101682000AA600200100C4090000000006A60020EE
:101692000100C4090000000004A600200100C409E2
:1016A20000000000944504080E0000000000000045
:1016B2000000000000000000F40E002094620020F0
:1016C2009CFF2C0100000000760800200A000000A8
:1016D200800B0408DC6F0020E0150C1700000000EE
:1016E2007508002008000000FC0A040874080020A5
:1016F20005000000600B0408DE6F002002000000FD
:10170200980B0408267100200100FF7F01000000F1
:101712001E71002002000000A40B0408F86F0020D4
:1017220003000000B40B0408F76F00200300000060
:10173200B40B0408F67000200000F4010100000060
:10174200F47000200000F40101000000F27000209B
:101752000000F40101000000F07000200000F4011C
:1017620001000000EE70002000FF01000A7100205D
:10177200E803D0070A00000008710020006401009D
:101782000A00000009710020006401000A00000044
:1017920002710020006401000A00000007710020AD
:1017A200006401000A0000000671002000640100CC
:1017B2000A00000005710020006401000A00000018
:1017C2000171002000FF01000A00000000710020EA
:1017D20000FF01000A000000007000200000F40178
:1017E20001000000FE6F00200000F4010100000073
:1017F200FC6F00200000F40101000000FA6F0020DD
:101802000000F40101000000FD70002000C801008A
:10181200FC70002000C80100FB70002000C801001D
:10182200FA700020006401000A000000F970002034
:1018320000FF01000A0000001571002000C801002D
:101842001471002000C801001371002000C80100BB
:101852001271002000C801001171002000C80100AF
:101862001071002000C801000F71002000C80100A3
:101872000E71002000C801000D71002000C8010097
:101882009C45040800000000000000000000000069
:1018920000000000AC450408090000000000000040
:1018A200980F002004000000B4450408090000005D
:1018B200000000008C0F00200400000044490408CE
:1018C2000900000000000000800F0020040000005A
:1018D2007C3E04080900000000000000740F002094
:1018E20004000000BC4504080900000000000000DC
:1018F200680F002004000000C4450408090000002D
:10190200000000005C0F002004000000CC45040829
:101912000900000000000000500F00200400000039
:10192200D44504080900000000000000440F002014
:1019320004000000A44304080100000000000000AD
:101942000000000000000000000000000D00000088
:10195200000000000000000000000000AC46040887
:101962000000000000000000000000000000000075
:10197200A43F04080000000000000000640A0020E8
:1019820004000000783E04080C000000DD2E03086D
:10199200F80F002000000000904404080C00000032
:1019A200F9280308EC0F002000000000B4430408EB
:1019B2000C000000C5280308E00F00200000000012
:1019C200244504080800000000000000D40F002095
:1019D20004000000144504080C000000B1280308AC
:1019E200C80F002000000000B846040809000000EB
:1019F20000000000BC0F002004000000A043040807
:101A0200030000007D580308A40F0020000000001E
:101A1200A4430408010000000000000000000000D0
:101A220000000000000000000D00000000000000A7
:101A32000000000000000000C04604080000000092
:101A4200000000000000000000000000D046040872
:101A52000C00000000000000101000200000000038
:101A6200D84604080A000000000000003971002076
:101A720000000000E44604080A0000000000000024
:101A82004171002000000000EC4604080A0000003A
:101A9200000000004971002000000000F446040824
:101AA20008000000000000000410002000000000F8
:101AB200A443040801000000000000000000000030
:101AC20000000000000000000D0000000000000007
:101AD2000000000000000000FC46040800000000B6
:101AE2000000000000000000000000001047040891
:101AF2000C00000000000000281000200000000080
:101B02002047040804000000193203080000000006
:101B120000000000284704080C000000000000003C
:101B22001C100020000000003C47040804000000D4
:101B3200F93103080000000000000000A44304087B
:101B42000100000000000000000000000000000092
:101B5200000000000D000000000000000000000076
:101B620000000000444704080000000000000000DC
:101B720000000000000000005847040807000000B1
:101B82000000000064100020000000006447040808
:101B920008000000000000005810002000000000B3
:101BA2007047040808000000000000004C100020EC
:101BB200000000007C47040808000000000000004C
:101BC20040100020000000008847040808000000C0
:101BD200000000003410002000000000A4430408AC
:101BE20001000000000000000000000000000000F2
:101BF200000000000D0000000000000000000000D6
:101C020000000000944704080000000000000000EB
:101C12005F0A002000000000A04704080B0000003B
:101C220000000000CC10002000000000A8470408BB
:101C32000B00000000000000C010002000000000A7
:101C4200B44704080B00000000000000B41000209C
:101C520000000000C04704080B0000000000000064
:101C6200A810002000000000CC4704080B00000070
:101C7200000000009C10002000000000D84704086B
:101C82000B00000000000000901000200000000087
:101C9200E04704080B000000000000008410002050
:101CA20000000000EC4704080B00000000000000E8
:101CB2007810002000000000F84704080800000027
:101CC200000000006C10002000000000A443040883
:101CD2000100000000000000000000000000000001
:101CE200000000000D0000000000000000000000E5
:101CF200000000000448040800000000000000008A
:101D0200000000000000000018480408080000005D
:101D120000000000FC10002000000000244804081D
:101D22000800000000000000F01000200000000089
:101D3200304804080800000000000000E410002001
:101D4200000000003C4804080800000000000000F9
:101D5200D810002000000000A44304080100000085
:101D62000000000000000000000000000000000071
:101D72000D00000000000000000000000000000054
:101D82004448040800000000000000005C0A002033
:101D920000000000544804080B000000000000008E
:101DA2002C11002000000000604804080B00000015
:101DB2000000000020110020000000006C48040810
:101DC20007000000000000001811002000000000C1
:101DD20078480408070000000000000010110020ED
:101DE2000000000084480408070000000000000012
:101DF2000811002000000000A443040801000000B4
:101E020000000000000000000000000000000000D0
:101E12000D000000000000000000000000000000B3
:101E22009048040800000000000000005C0A002046
:101E3200000000009C4804080700000000000000A9
:101E42007811002000000000A448040807000000E8
:101E5200000000007011002000000000AC480408DF
:101E620007000000000000006811002000000000D0
:101E7200B4480408070000000000000060110020C0
:101E820000000000BC480408070000000000000039
:101E92005811002000000000C44804080700000098
:101EA200000000005011002000000000CC4804088F
:101EB20007000000000000004811002000000000A0
:101EC200D448040807000000000000004011002070
:101ED20000000000DC4804080700000000000000C9
:101EE2003811002000000000A44304080100000093
:101EF20000000000000000000000000000000000E0
:101F02000D000000000000000000000000000000C2
:101F1200E44804080E00000000000000852A0308BF
:101F22000000000080110020F66F00201700000062
:101F3200C40B0408F56F00200A320100F46F002080
:101F420001FA0100F06F002000C80100EE6F0020CE
:101F5200E803D007010000004634425900000000A7
:101F6200EC4804080E0000001128030800000000DD
:101F7200000000005C120020F44804080E0000007B
:101F8200452F0308BD2C0308B92C03083813002081
:101F9200FC4804080E0000009B2A03080000000011
:101FA20000000000D8130020044904080E000000BD
:101FB200292B0308F92A03080000000064140020FA
:101FC2000C4904080E000000A52B0308ED2B0308A2
:101FD2000000000004150020FE7000200103010033
:101FE200184904080E000000CD2A0308A92A030894
:101FF20000000000F4150020204904080E00000033
:10200200592B030839320308000000008016002013
:102012002C4904080E0000001D2C03088532030819
:102022000000000020170020F870002001030100CA
:102032003449040800000000000000000000000015
:1020420000000000404904080800000000000000F1
:102052004C18002000000000484904080700000056
:102062000000000044180020000000005849040845
:1020720007000000000000003C18002000000000E3
:102082006449040807000000000000003418002022
:1020920000000000704904080C000000000000006D
:1020A20028180020000000007C49040803000000FA
:1020B2007D5803081018002000000000A443040803
:1020C200010000000000000000000000000000000D
:1020D200000000000D0000000000000000000000F1
:1020E2000000000084490408000000000000000015
:1020F2000000000000000000944904080A000000EB
:1021020000000000C8140408000000009C490408F4
:102112000A0000000000000048140408000000004B
:10212200A44904080A000000000000001671002003
:1021320000000000AC4904080A0000000000000092
:102142005818002000000000A44304080100000009
:10215200000000000000000000000000000000007D
:102162000D00000000000000000000000000000060
:10217200B449040800000000000000000000000054
:1021820000000000C8490408030000007D5803084D
:102192007818002000000000D44904080300000061
:1021A2007D5803087808002000000000DC4904087C
:1021B200030000007D5803086018002000000000A2
:1021C200A443040801000000000000000000000019
:1021D20000000000000000000D00000000000000F0
:1021E2000000000000000000E449040800000000B4
:1021F200000000000000000000000000F049040898
:1022020007000000D1320308281900200000000056
:10221200FC400408030000007D5803081019002048
:1022220000000000FC490408030000007D58030878
:10223200F818002000000000044A0408030000000F
:102242007D580308E0180020000000000C4A040832
:1022520007000000B5320308D81800200000000073
:10226200AC440408030000007D580308C018002095
:1022720000000000184A0408030000007D5803080B
:10228200A818002000000000244A040803000000EF
:102292007D5803089018002000000000A4430408A1
:1022A200010000000000000000000000000000002B
:1022B200000000000D00000000000000000000000F
:1022C20000000000304A04080E0000004D2A0308F6
:1022D200152A03080000000030190020384A0408BB
:1022E2000E0000008D2C030800000000000000001A
:1022F200E4190020444A04080E0000000000000017
:102302000000000000000000701A0020544A040877
:102312000E000000652C0308ED32030800000000E7
:10232200E81A00205C4A04080000000000000000D7
:102332000000000000000000803E040803000000CE
:102342007D5803080C1C002000000000484A0408C5
:10235200030000007D580308F41B00200000000069
:10236200684A0408030000007D580308DC1B0020B3
:1023720000000000744A0408030000007D580308AE
:10238200C41B0020000000007C4A04080200000078
:102392007D5703080000000000000000844A040882
:1023A200020000007D570308010000000000000049
:1023B200904A0408020000007D5703080200000052
:1023C20000000000000000000D00000000000000FE
:1023D200000000000000000001000000685E0C0028
:1023E20043000000000000000000000000000000A8
:1023F20000000000000000000000000000000000DB
:102402004300000000000000000000000000000087
:1024120000000000000000000000000000000000BA
:102422004300000000000000000000000000000067
:10243200000000000000000000000000000000009A
:102442004300000000000000000000000000000047
:10245200000000000000000000000000000000007A
:102462004300000000000000000000000000000027
:10247200000000000000000000000000000000005A
:102482004300000000000000000000000000000007
:10249200000000000000000000000000000000003A
:1024A20043000000000000000000000000000000E7
:1024B200000000000000000000000000000000001A
:1024C20011BF030869BD030800000000054D0408A0
:1024D20065450408D63B0408D63B0408D63B0408ED
:1024E200D63B0408D63B0408D63B0408D63B040876
:1024F200D63B0408D63B0408FFFFFFFFFFFFFFFFA8
:10250200FFFFFFFFFFFF0000010041534349490065
:1025120000000000000000000000000000000000B9
:102522000000000000000000000041534349490040
:102532000000000000000000000000000000000099
:10254200000000000000000000000000501E0020FB
:102552000000000000000000000000000000000079
:102562000000000000000000000000000000000069
:102572000000000000000000000000000000000059
:102582000000000000000000000000000000000049
:102592000000000000000000000000000000000039
:1025A2000000000000000000000000000000000029
:0425B2000100000024
:1080000070B4EFF31186502383F31288436B1A6820
:10801000D20720D45D686DB9446A826A944217D051
:1080200081691144D9600ED9A21A5A608462002273
:1080300080F858201A6842F00102F1B21A6081F308
:10804000118870BC704701698A1A5A608562EEE730
:10805000012380F85830F3B283F3118870BC704765
:10806000436A8269D154436A0169426B01338B428E
:1080700028BF00234362002A2FD0EFF31182502340
:1080800083F31288436B1968C9072CD470B45E68F7
:108090006EB9456A816A8D4217D084690C44DC60F0
:1080A0000ED9691A59608562002180F85810196844
:1080B00041F00101D2B2196082F3118870BC70479F
:1080C0000469611A59608662EEE7012380F858302E
:1080D000D2B282F3118870BC7047426DD36843F00E
:1080E0008003D3607047D2B282F31188704700BF1B
:1080F000026B10B462B1836CC2684469D11A013B4F
:10810000615C5DF8044B08BF13468364C8B27047D6
:10811000016A4369C4685B5C0131A14228BF114612
:1081200001625DF8044BD8B2704700BF436B13B1D6
:1081300090F858007047836A406A181AB0FA80F0C5
:1081400040097047416A836A99420AD3CB1A416B4E
:10815000026961B14968501E0B4483420AD2C01AB9
:10816000704702691144CB1A416B0029F2D1501EAD
:10817000C01A704700207047036B43B1826C5B6884
:1081800093422FBF981AC0689B1AC0187047C269E3
:10819000036A9A422FBFD01AC0688018C01A70476D
:1081A0000A4B30B503F11C0493F900205D78072ACF
:1081B000C8BF143A811804330D7313F8025C855458
:1081C00013F8012C0A76A342EED130BDF0E3030888
:1081D00003682DE9F041DF691FB13B46BDE8F0417E
:1081E0001847002A164611DD04460D460E4400E0ED
:1081F00023689B68204698470028F9D0236815F823
:10820000011B1B6820469847AE42F1D1BDE8F081C2
:1082100010B4522153245122002304704170827003
:10822000C3705DF8044B704710B5084B03F10C01A7
:1082300093F900205C78845402449C78D470DC78F4
:10824000947104338B42F3D110BD00BF0CE40308DA
:10825000F0B5846814B12568A4886C8341F080016E
:10826000446840F2E93501E0002D58D02689013DEF
:1082700016F0020FADB2F7D089B2A18140F2E93118
:1082800001E0002960D02589013915F0010F89B27C
:10829000F7D0A189A1894FF0000C4FF47A714FF605
:1082A000FF764FF0FF0E634502D131E0B1421BD0A3
:1082B0002589013915F0020589B2F7D0A4F80CE040
:1082C0004FF47A7102E0B9B2B1420DD0258915F0B0
:1082D000010501F1FF37F6D0A589ADB20AB11570DD
:1082E00001320CF1010CDEE7244B9C4208D0A3F5CF
:1082F00078439C423CD003F580639C4208D1022520
:108300001F4B03EB05156B8901339BB26B816B89A6
:10831000836813B11A689B8813830120F0BD174945
:108320008C4208D0A1F578418C4223D001F58061C0
:108330008C42AFD10225124901EB05156989013143
:1083400089B269816989A5E70C4DAC4207D00D4916
:108350008C4211D001F580618C429BD10221084DE5
:1083600005EB01114D890135ADB24D81498991E788
:108370000125C5E70125DEE70121F0E700300140D6
:1083800084A700200038004030B4846814B123680A
:10839000A5885D83436840F2E93001E0002833D0CE
:1083A0001D89013815F0020F80B2F7D089B299818A
:1083B00040F2E93101E0002950D01889013910F06C
:1083C000010F89B2F7D0998940F2E93101E0002923
:1083D0002FD01889013910F0020F89B2F7D092B26C
:1083E0009A8140F2E93201E0002A4BD01989013A22
:1083F00011F0010F92B2F7D09B8914B12368A288C3
:108400001A83012030BC70472C498B4208D0A1F55B
:1084100078418B424CD001F580618B42D4D102204F
:10842000274901EB00104189013189B2418141891D
:10843000CAE7224A934208D0A2F57842934235D047
:1084400002F580629342D8D102211D4B03EB01114A
:108450004B8901339BB24B814B89CEE7174883424E
:1084600007D018498B4227D001F580618B42ABD1F0
:108470000221134800EB01114889013080B2488184
:108480004989A1E70D498B4207D00E4A934211D08A
:1084900002F580629342B0D10222094B03EB021233
:1084A000538901339BB253815389A6E70121CCE75D
:1084B0000120B5E70122F0E70121DAE700300140B1
:1084C00084A7002000380040002870B51EDB092872
:1084D000044620DD012303EB83035B00B0FBF3F2D2
:1084E000092AF8D87BB10E4EB4FBF3F00928CCBFB3
:1084F00057223022A6FB03E5024403FB1044EB089D
:1085000001F8012BF0D100230B7070BD2D230B70EF
:1085100040420131DBE7303001F8010BF3E700BFE7
:10852000CDCCCCCC884230B44FF001042ED301FB2B
:1085300004F4B0FBF4F58D42F9D284B1AAB901E09C
:10854000B0FBF4F5092DCCBF572230222A4404FB9E
:10855000150003F8012BB4FBF1F4002CF0D100223C
:108560001A7030BC7047B0FBF4F5092DCCBF372230
:1085700030222A4404FB150003F8012BB4FBF1F46C
:10858000002CF0D100221A7030BC70470546002A3A
:10859000EBD1D7E703685A1C02601970704700BF1F
:1085A0002DE9F047089C2578002B804689460CBFB2
:1085B0004FF0200A4FF0300A661C35B3002A29DD3F
:1085C000334601E0024698B113F8011B501E002902
:1085D000F8D1971E60B13D46013D51464046C8471F
:1085E0006B1C002BF8DC257827EAE770013055B1C9
:1085F000041B29464046C847301916F8015B002D78
:10860000F7D1BDE8F087BDE8F087002A04DC2846F2
:10861000BDE8F0870020EBE7571EDCE7836842687F
:10862000D0ED037A00EB83010133934281ED040A1C
:10863000836004BF0023836000EB830393ED047A1F
:10864000036870EE277A9A42C0ED037A77EEC77A14
:10865000C0ED037A0CDA013307EE103AF8EEC76A80
:10866000B7EE007A87EEA60A036030EE070A70477D
:1086700007EE102AB8EEC77A87EE870A704700BF68
:1086800090ED057A90ED004AD0ED066AD0ED014AF2
:10869000D0ED047A90ED035AD0ED025AA4EE007AA0
:1086A000B0EE406AB0EE470AB0EE667AA6EE247AE3
:1086B00067EEC07AA0EE457AE6EE257A80ED057A7F
:1086C000C0ED067A704700BFD0ED057A90ED013A13
:1086D000D0ED003AD0ED064A90ED024A90ED077ACF
:1086E00090ED035A90ED086AD0ED045AC0ED067A79
:1086F000F0EE406A27EE830AC0ED056AA3EEA60AF3
:1087000080ED087AA4EE240AA5EE470AA5EEC60A73
:1087100080ED070A704700BFD0ED007A90ED017A36
:1087200030EE670AE7EE007AB0EE670AC0ED007A35
:10873000704700BF704700BF0A44914214D030B464
:108740000139551E41F2210211F8014F082380EA38
:10875000042004044CBF82EA40004000013B80B288
:10876000F7D18D42F0D130BC704700BF2DE9F04FFA
:10877000DFF8F8C1DFF8F8E1BCF80A70DEF8006055
:10878000BCF80C30BCF808A03C028BB0361B4FF094
:108790000004CDE90034009CBCF806304FEA1765B0
:1087A0004FF0000767EB0507B946B046A4FB066724
:1087B0000024CDE90634009C002304FB0977002443
:1087C000CDE90034AAFB0823CDE90223039AF30D77
:1087D00000930AFB09230393009B43EA472300937A
:1087E000029B4FEAD31AFB150193039B4AEA436AA3
:1087F000DDE9002344464D46CDE90845069C12F5C7
:10880000FA62A4FB086743F1000304FB0977CDE992
:108810000623BCF80440039BBCF802204FEAE31B8C
:10882000230C059323040493340A44EA07643D129D
:10883000DDE904674FEAC23816EB0A0647EB0B077F
:1088400018EB0408DDE906344FEA524949EB050903
:10885000B3F5FA6F74F10004B246BB463CDADDE9C9
:108860000067BC00B20044EA9673B41847EB0305F6
:1088700022463C462B4602FB04F406FB0344A2FBC3
:1088800006232344940844EA83749D105B104FEA46
:108890003202B8EB040869EB0509BAEB020A6BEB8C
:1088A000030BDDE90623304C4FF0FF35A242AB410C
:1088B0002CDBDDE90856A5FB052305FB06F403EBDD
:1088C0004403D40F44EA4304DD17DDE90623121BF9
:1088D00063EB0503CDE90623DEF80440A4FB08237F
:1088E00004FB0933540D44EAC3245D15B4EB0A0AB2
:1088F00065EB0B0B4FEADA3343EA4B4300B10360FD
:1089000009B1069B0B600BB0BDE8F08F40F6AC528E
:10891000B4184FF0000347EB03052246A2FB0223E5
:1089200004FB05F403EB4403941843EB0305A4187C
:108930005D414FEA850CA6004CEA947CB41A6CEBBE
:108940000305DF00D6006D104FEA340447EA527782
:10895000921B63EB0703B8EB040869EB05091AEBFC
:10896000020A4BEB030BA4E724FAFFFF2857002071
:10897000B41E00204FF480538382704750F8043CAB
:10898000012280F84520103803B11847704700BF16
:10899000BFF34F8F0549064BCA6802F4E0621343E8
:1089A000CB60BFF34F8F00BFFDE700BF00ED00E0DD
:1089B0000400FA05F8B5057B466903681F2D29D91F
:1089C000A5F120045F682021A1400F422A4613D060
:1089D0001022A240D960DA605A68E240D10703D57C
:1089E000012202FA04F4DC6004463046FFF708FB7B
:1089F000227B23681F2A20D9A2F1200008215A686F
:108A00008140114200D0D9600422596882400A4254
:108A100021D1F8BD20211C68A9400C422A460CD067
:108A20001022AA4099609A601A68EA40D207DBD502
:108A3000012202FA05F59D60D6E7082118689140E9
:108A4000014200D099600421186801FA02F2024242
:108A500003D09A60F8BDDA60F8BDF8BD70B4037B4E
:108A600004681F2B08D9203B2021626801FA03F318
:108A70001A421CD170BC70472021226801FA03F30E
:108A80001A42F7D042691449582000FB021251687B
:108A90005689CD680868296821F00101296082891A
:108AA00092B222EA06028281A36070BC70474269DA
:108AB0000949582000FB021251685689CD680868A0
:108AC000296821F001012960828992B222EA060216
:108AD0008281E36070BC70474C58002030B4094B71
:108AE0001C786CB1084A002502EBC4041168938815
:108AF0004D628889083203439BB2A2428B81F5D133
:108B000030BC70470C5B0020105B0020F0B5C40047
:108B100022189200AE498B585B689D8AADB2EEB2C6
:108B2000F7070A445CD4B70732D5BFF35F8F167ED0
:108B3000F6B2012E00F0C780A64D1A8BBFF35F8FEF
:108B4000221801EB8202167E022E00F0D580221838
:108B500001EB8202167E032E00F088809A8895F938
:108B6000086092B242F480629A80221801EB82027D
:108B7000127E013296425BD1AA7A00266E72002ADA
:108B800040F09580204401EB800000234375F0BD48
:108B900077074ED416F0400600F0C9808D4D1E8A2E
:108BA00095F908E0176AF6B207F80E605FFA8EFED4
:108BB0000EF1010C4FFA8CFC177E85F808C00CF101
:108BC00003029742664600F01C81221801EB8202E4
:108BD000127E9445C9D10EF1020676B22E72C4E718
:108BE0001E887C4D26F400663604360C1E801E88D6
:108BF000B6B246F480661E80967E00272F72002E45
:108C000048D06E7A002E42D0221801EB8202012653
:108C1000127E6E72022A00F0B980221801EB8202E5
:108C2000927D42F001021A82204401EB8000037E13
:108C3000F0BD684D967E0127AF72002E73D06E7A1C
:108C4000002E7BD1221801EB8202527E002A00F016
:108C5000A3801A882E7A92B2013642F4007276B25C
:108C60001A802E721A88D205FCD47EE7927E002AE2
:108C70003FF474AF6A7A002A3FF470AF9A8895F98E
:108C8000086022F480621204120C9A806DE7D27D93
:108C9000FF2AB9D0221801EB8202967D06F0FE066B
:108CA0001E82D37DFF2BBFD0FF232B72BCE79A8897
:108CB00022F4407212042044120C01EB80009A80CE
:108CC00000234375F0BD927E424D002A3FF435AF3C
:108CD0006A7A002A3FF431AF1A8822F480621204C3
:108CE000120C1A80BFF35F8F1A8B1A88AE7292B281
:108CF00042F400721A8031E7927E002A3FF427AFD7
:108D00006A7A002A3FF423AF1A8895F9086022F4A2
:108D100080621204120C1A809A8822F48062120473
:108D2000120C9A8021E76A7A002A8BD091E715F01D
:108D3000800F284D3AD195F9086016E7167ED2F8D3
:108D400020E01F88022E95F9086045D927F4806736
:108D50003F043F0C1F801F8AFFB20EF806701F8869
:108D6000D2F820E0BFB247F400771F80F2B21F8A2A
:108D7000561C76B2FFB20EF806709F88961CBAB2E7
:108D800076B242F480622E729A806BE71A8892B2B1
:108D900042F400621A8040E71A8895F9086092B29E
:108DA00042F4807201271A806F725BE795F90870B0
:108DB000B7F1FF3F2CD0D669F65D1E8292F818E01D
:108DC00001377AB2964516462A727FF4CEAEA3E7F3
:108DD000003C0020B41E0020BFB247F400771F8083
:108DE0001F8AFFB20EF80670F6B21F8AD2F820E092
:108DF000721C52B20336FFB276B20EF802702E72B7
:108E000030E79A8822F480621204120C9A80DCE621
:108E1000D77D1F822E72957E1DB9127E002A7FF4A7
:108E200003AF9A8822F480621204120C9A80FBE647
:108E300070B5044682B00830656A06236A463B2155
:108E4000A847A8B19DF804009DF800609DF80110A6
:108E50009DF802509DF803209DF8053041EA062157
:108E600043EA002342EA0522E18222836383012050
:108E700002B070BD00234360036083602A23437007
:108E80002B2303710123C37183727047F8B5046803
:108E9000C4F30D0405460E4604B32F682BF098FC6E
:108EA000092840F08880454C236923F440732361EE
:108EB000236943F400732361236943F001032361B1
:108EC0003E602BF085FC2369092823F00103236110
:108ED00071D12B6804332B600020F8BD384B394A20
:108EE00093422BD902F58042934226D902F5804263
:108EF00093422AD902F58042934228D902F5803262
:108F0000934226D902F50032934224D902F5003269
:108F1000934222D902F50032934220D902F5003261
:108F200093421ED902F5802293421CD9B3F1016FFE
:108F30001BD3052004F094FDFBE708242BF048FC2C
:108F4000092814D04FF0FF30F8BD1024F6E718249C
:108F5000F4E72024F2E72824F0E73024EEE7382471
:108F6000ECE74024EAE74824E8E75824E6E7134F13
:108F70003B6923F440733B613B6943F400733B61FD
:108F80003B6923F0F8033B613B6943F002031C4358
:108F90003C613B6943F480333B612BF019FC3B6936
:108FA00023F002033B613B69092823F0F8033B618E
:108FB0003FF473AFC6E76FF00100F8BD003C02401C
:108FC00000400008FF3F0008F8B504460D468E1823
:108FD0000027B54201D12069F8BDE368591CE16062
:108FE000234415F8012B1A720429F2D1206918B90B
:108FF000A1682046FFF74AFF2061E760E9E700BF6C
:1090000070B582B004466946143028F045FCB0B112
:109010009DF805009DF801609DF802109DF8035031
:109020009DF804209DF8063041EA062143EA00231A
:1090300042EA0522A187E287A4F84030012002B06D
:1090400070BD00BF38B5254B9C68236B73B1636D51
:10905000626BCAB1998A1A88C90592B201D5D20742
:1090600000D438BD4FF6F7721A8038BD636D998908
:109070001A88890692B2EBD59206E9D5E26ACAB19E
:10908000988880B29047E2E799891A880D0692B2D3
:10909000E0D51006DED5A26A616A8A4219D0A169BC
:1090A0002569885C98800132B2FBF5F105FB11223D
:1090B000A262CFE79B88E2696169DBB28B54E26907
:1090C000E068636D0132B2FBF0F100FB1122E26156
:1090D000BEE7DA6822F08002DA60BBE7D83B002006
:1090E00038B5254B5C68236B73B1636D626BCAB195
:1090F000998A1A88C90592B201D5D20700D438BD21
:109100004FF6F7721A8038BD636D99891A888906FF
:1091100092B2EBD59206E9D5E26ACAB1988880B2DC
:109120009047E2E799891A880D0692B2E0D51006B9
:10913000DED5A26A616A8A4219D0A1692569885C74
:1091400098800132B2FBF5F105FB1122A262CFE754
:109150009B88E2696169DBB28B54E269E068636D08
:109160000132B2FBF0F100FB1122E261BEE7DA68E6
:1091700022F08002DA60BBE7D83B002038B5254BEF
:109180001C68236B73B1636D626BCAB1998A1A88CC
:10919000C90592B201D5D20700D438BD4FF6F77297
:1091A0001A8038BD636D99891A88890692B2EBD509
:1091B0009206E9D5E26ACAB1988880B29047E2E7A0
:1091C00099891A880D0692B2E0D51006DED5A26AFA
:1091D000616A8A4219D0A1692569885C9880013248
:1091E000B2FBF5F105FB1122A262CFE79B88E26991
:1091F0006169DBB28B54E269E068636D0132B2FBF6
:10920000F0F100FB1122E261BEE7DA6822F0800291
:10921000DA60BBE7D83B002003685B6A03B11847FC
:10922000704700BF03681B6A03B11847704700BF4F
:1092300003682DE9F041DF691FB13B46BDE8F0410D
:109240001847002A164611DD04460D460E4400E07C
:1092500023689B68204698470028F9D0236815F8B2
:10926000011B1B6820469847AE42F1D1BDE8F08152
:1092700003689B69184700BF03685B69184700BF14
:1092800003681B69184700BF0368DB68184700BF05
:1092900003689B68184700BF03685B68184700BFF6
:1092A00003681B68184700BF014B1868F8E700BF48
:1092B00004A7002038B50C46097849B105460134A9
:1092C0002B6828461B68984714F8011B0029F7D122
:1092D00038BD00BF064B53F820302BB11A689B886D
:1092E00051690B4201D1138370475383704700BF0C
:1092F00020B2002003682DE9F04F03F13F4404F54C
:109300007E04604EA40A0125345D04F01F06640942
:10931000032C05FA06F500F0AF80042C00F0A780BE
:10932000022C54D08588B5FA85F0C0F11F0080B2B8
:10933000C40803EB840400F00700266A80000F27AE
:10934000874026EA07062662276A01F0030602FA2A
:1093500000F0721E3843012AC1F3810CC1F30018DA
:109360002062C1F3411137D90024224601274FF072
:10937000030E03E0102A04F1020426D007FA02F0DB
:10938000A84302F10102F5D1D3F800C00EFA04F0AF
:10939000C04300EA0C0CC3F800C0D3F8008006FA02
:1093A00004FC4CEA080CC3F800C0D3F80CC000EA77
:1093B0000C00D860D3F80CC001FA04F040EA0C00AD
:1093C000102AD86004F10204D8D1BDE8F08F2E4CE9
:1093D000666C35436564A5E7002002464FF0010E38
:1093E0004FF0030904E00132102A00F102003CD0E2
:1093F0000EFA02F737EA0504F5D1D3F800A009FA0E
:1094000000F4E4430AEA040AC3F800A0D3F800B069
:1094100006FA00FA4AEA0B0AC3F800A0D3F808A03B
:1094200004EA0A0AC3F808A0D3F808B00CFA00FA54
:109430004AEA0B0AC3F808A0D3F804A02AEA0707EF
:109440005F60D3F804A008FA02F747EA0A075F60F2
:10945000DF683C40DC60DF6801FA00F401323C4325
:10946000102ADC6000F10200C2D1BDE8F08F064C8A
:10947000266B3543256355E7034C266C354325643D
:1094800050E700BFE813040800380240026802F108
:109490003F4303F57E032DE9F04F9B0A544DEB5CEF
:1094A00003F01F055B090124032B04FA05F400F007
:1094B0009980042B00F09180022B3ED001F003062E
:1094C000731E012BC1F3810CC1F300188588C1F311
:1094D000411137D90024234601274FF0030E03E042
:1094E000102B04F1020426D007FA03F0A84303F17D
:1094F0000103F5D1D2F800C00EFA04F0C04300EA2F
:109500000C0CC2F800C0D2F8008006FA04FC4CEA49
:10951000080CC2F800C0D2F80CC000EA0C00D06001
:10952000D2F80CC001FA04F040EA0C00102BD06015
:1095300004F10204D8D1BDE8F08F2E4B5D6C2C43B2
:109540005C64BBE7002003464FF0010E4FF00309B7
:1095500004E00133102B00F102003CD00EFA03F7B7
:1095600037EA0504F5D1D2F800A009FA00F4E44383
:109570000AEA040AC2F800A0D2F800B006FA00FA1B
:109580004AEA0B0AC2F800A0D2F808A004EA0A0AC4
:10959000C2F808A0D2F808B00CFA00FA4AEA0B0A9E
:1095A000C2F808A0D2F804A02AEA07075760D2F848
:1095B00004A008FA03F747EA0A075760D7683C4057
:1095C000D460D76801FA00F401333C43102BD46017
:1095D00000F10200C2D1BDE8F08F064B1D6B2C4399
:1095E0001C636BE7034B1D6C2C431C6466E700BFD8
:1095F000E81304080038024010B50409013C042CAB
:1096000017D80D4B33F8142000F00F0042FA00F386
:1096100013F001030DD0012303FA00F001381040CC
:1096200032F0B6FA054A064B125D104403EBC00057
:1096300010BD002010BD00BFF8130408F01304088B
:109640009CAF00202DE9F04F4A484B494B4B4C4C06
:109650004FF0010A4FF002094FF004084FF0080CD8
:109660004FF0100E20274026802530F8022B12F0F4
:10967000010F03D01960A3F804A0083312F0020F01
:1096800003D01960A3F80490083312F0040F03D03C
:109690001960A3F80480083312F0080F03D0196092
:1096A000A3F804C0083312F0100F03D01960A3F818
:1096B00004E0083312F0200F02D019609F800833B5
:1096C00012F0400F02D019609E80083312F0800F14
:1096D00002D019609D80083312F4807F05D04FF4CA
:1096E000807B1960A3F804B0083312F4007F05D022
:1096F0004FF4007B1960A3F804B0083312F4806FB4
:1097000005D04FF4806B1960A3F804B0083312F44D
:10971000006F05D04FF4006B1960A3F804B0083354
:1097200012F4805F05D04FF4805B1960A3F804B099
:10973000083312F4005F05D04FF4005B1960A3F802
:1097400004B0083312F4804F05D04FF4804B1960F9
:10975000A3F804B00833D20B04D04FF400421960D0
:109760009A80083301F58061A1427FF47EAFBDE8A5
:10977000F08F00BFF8130408000002409CAF0020E7
:109780000014024000286AD003682DE9F04F03F16D
:109790003F4404F57E045F4EA40A0125345D04F0C5
:1097A0001F066409032C05FA06F559D0042C00F0B5
:1097B000AC80022C59D08588B5FA85F0C0F11F0025
:1097C00080B2C40803EB840400F00700266A80001E
:1097D0000F27874026EA07062662276A01F003065C
:1097E0008240701E3A430128C1F3810CC1F3001876
:1097F0002262C1F341113DD90024224601274FF0D6
:10980000030E03E0102A04F1020426D007FA02F046
:10981000A84302F10102F5D1D3F800C00EFA04F01A
:10982000C04300EA0C0CC3F800C0D3F8008006FA6D
:1098300004FC4CEA080CC3F800C0D3F80CC000EAE2
:109840000C00D860D3F80CC001FA04F040EA0C0018
:10985000102AD86004F10204D8D1BDE8F08F704717
:109860002D4C266C35432564A5E72B4C666C35439F
:109870006564A0E7002002464FF0010E4FF0030997
:1098800004E00132102A00F102003CD00EFA02F787
:1098900037EA0504F5D1D3F800A009FA00F4E4434F
:1098A0000AEA040AC3F800A0D3F800B006FA00FAE6
:1098B0004AEA0B0AC3F800A0D3F808A004EA0A0A8F
:1098C000C3F808A0D3F808B00CFA00FA4AEA0B0A69
:1098D000C3F808A0D3F804A02AEA07075F60D3F80A
:1098E00004A008FA02F747EA0A075F60DF683C4015
:1098F000DC60DF6801FA00F401323C43102ADC60CE
:1099000000F10200C2D1BDE8F08F034C266B354355
:10991000256350E7E813040800380240002855D0BA
:10992000026802F13F4303F57E032DE9F04F9B0AE5
:10993000544DEB5C03F01F055B090124032B04FA73
:1099400005F444D0042B00F09780022B44D001F0A2
:109950000306731E012BC1F3810CC1F30018858827
:10996000C1F341113DD90024234601274FF0030ED6
:1099700003E0102B04F1020426D007FA03F0A843F9
:1099800003F10103F5D1D2F800C00EFA04F0C04390
:1099900000EA0C0CC2F800C0D2F8008006FA04FC01
:1099A0004CEA080CC2F800C0D2F80CC000EA0C0067
:1099B000D060D2F80CC001FA04F040EA0C00102B81
:1099C000D06004F10204D8D1BDE8F08F70472E4B6F
:1099D0001D6C2C431C64BAE72B4B5D6C2C435C6400
:1099E000B5E7002003464FF0010E4FF0030904E0F5
:1099F0000133102B00F102003CD00EFA03F737EAD6
:109A00000504F5D1D2F800A009FA00F4E4430AEA0B
:109A1000040AC2F800A0D2F800B006FA00FA4AEA36
:109A20000B0AC2F800A0D2F808A004EA0A0AC2F899
:109A300008A0D2F808B00CFA00FA4AEA0B0AC2F8F9
:109A400008A0D2F804A02AEA07075760D2F804A0B9
:109A500008FA03F747EA0A075760D7683C40D46022
:109A6000D76801FA00F401333C43102BD46000F1B5
:109A70000200C2D1BDE8F08F034B1D6B2C431C6369
:109A800065E700BFE81304080038024010B103681E
:109A900082885A83704700BF10B1036882881A8396
:109AA000704700BF18B10368828809B95A837047AC
:109AB0001A83704710B40A4B0A4A1C78012383406A
:109AC000234052F8200029B9B3FA83F149095DF81F
:109AD000044BE7E7191C18BF01215DF8044BE1E7CF
:109AE0001CB2002020B2002030B1036882881B69BC
:109AF0001A4214BF01200020704700BF2DE9F04139
:109B00000B4E346873691C400FD0DFF828800127A2
:109B1000B4FA84F3C3F11F0307FA03F558F82300DE
:109B200003689847AC437561F2D1BDE8F08100BF8E
:109B3000003C0140BC6700202DE9F0410B4E346829
:109B400073691C400FD0DFF828800127B4FA84F332
:109B5000C3F11F0307FA03F558F823000368984779
:109B6000AC437561F2D1BDE8F08100BF003C01401B
:109B7000BC6700202DE9F0410B4E346873691C402E
:109B80000FD0DFF828800127B4FA84F3C3F11F0354
:109B900007FA03F558F8230003689847AC4375614A
:109BA000F2D1BDE8F08100BF003C0140BC6700205D
:109BB0002DE9F0410B4E346873691C400FD0DFF87B
:109BC00028800127B4FA84F3C3F11F0307FA03F5D1
:109BD00058F8230003689847AC437561F2D1BDE89B
:109BE000F08100BF003C0140BC6700202DE9F0413E
:109BF0000B4E346873691C400FD0DFF828800127B2
:109C0000B4FA84F3C3F11F0307FA03F558F82300ED
:109C100003689847AC437561F2D1BDE8F08100BF9D
:109C2000003C0140BC6700202DE9F0410B4E346838
:109C300073691C400FD0DFF828800127B4FA84F341
:109C4000C3F11F0307FA03F558F823000368984788
:109C5000AC437561F2D1BDE8F08100BF003C01402A
:109C6000BC6700202DE9F0410B4E346873691C403D
:109C70000FD0DFF828800127B4FA84F3C3F11F0363
:109C800007FA03F558F8230003689847AC43756159
:109C9000F2D1BDE8F08100BF003C0140BC6700206C
:109CA000084A094808B5536C43F4804353640021C3
:109CB000402234F0E9FA054B4FF0FF321A60C3F846
:109CC000032008BD00380240BC670020FC6700206C
:109CD0002DE9F041044618460D461646984631F0E7
:109CE000ADFA2768E6722844A07229467D6943468A
:109CF00032462046AC46BDE8F0416047036810B5E7
:109D000004461B689847236820469B689847A37BB6
:109D10000133A37310BD08B5FFF76EFC38B12C22D8
:109D200082710022C2712021BDE80840F6E508BD1D
:109D3000144B984224D003F58063984220D00288C7
:109D400022F040021204120C0280028822F0380332
:109D50001B041B0C59B141F48071002991FAA1F246
:109D6000B2FA82F108BF4FF0FF310139C9000B434D
:109D70009BB2038003889BB243F04003038070478B
:109D80004908DCE700380040F0B5044690F8590077
:109D900083B0002840F0AA806A4EF77A002F43D0A3
:109DA00004F114054FF48071A069FFF7C1FF94F826
:109DB00052201A212846FEF7E7FA012004F0AAFAF9
:109DC0000421A069FFF7B4FF28460623E56D6A4623
:109DD0004321A847D8B19DF802609DF803309DF853
:109DE00000509DF801109DF804009DF8052043EAFD
:109DF00006231BB2E3875BB241EA052142EA002257
:109E00000133A187A4F8402006D003B0F0BDB4F917
:109E10003E305BB20133F8D194F93C300133F4D1D8
:109E2000062003F01DFEF0E704F114054FF48071E5
:109E3000A069FFF77DFF80226B212846FEF7A4FA78
:109E4000962004F0C1FA032268212846FEF79CFA06
:109E5000962004F0B9FA03226B212846FEF794FA03
:109E60000F2004F057FA10226A212846FEF78CFAD8
:109E70000F2004F04FFA3A466C212846FEF784FA88
:109E80000F2004F047FA94F8542019212846FEF7D1
:109E90007BFA0F2004F03EFA18221B212846FEF719
:109EA00073FA0F2004F036FA10221C212846FEF720
:109EB0006BFA0F2004F02EFA102237212846FEF705
:109EC00063FA0F2004F026FA012238212846FEF713
:109ED0005BFA0F2004F01EFA0421A069FFF728FFA7
:109EE000012004F017FA0123F3725BE7FFF784FB0C
:109EF0000546D8B1202300218371C171FFF70EFD03
:109F00002146114B41F8103F284627F05BFCAB88F7
:109F1000B3FA83F3C3F11F03012212FA03F33FF4F0
:109F20003BAF0A490A6813430B6035E70146FFF768
:109F3000F5FC2146044B41F8103F284627F042FC2F
:109F40002AE700BFB41E00207D890008003C0140C4
:109F5000F8B50501684C694B625961199A4204EBE6
:109F6000050704BF01230B730646387A30F078FAF0
:109F70003B7A03F01F015B090122032B02FA01F275
:109F80006DD0042B66D0022B5CD063190136187992
:109F9000FFF732FBF6B2074610B11223C671837188
:109FA00063195879FFF728FB10B11323C671837129
:109FB00063199879FFF720FB10B11423C6718371E0
:109FC00066190A21F2793846FFF7DCFB7079FFF752
:109FD00013FBF2790A21FFF7D5FBB079FFF70CFBF1
:109FE000F2790A21FFF7CEFB6359454A934247D0E5
:109FF000424A934250D0434A934259D0424A9342F4
:10A0000062D0424A93426BD0414A93422CD02C44B6
:10A01000227BE2B901200222198801F4415141F466
:10A0200045710A4302431A809A8B22F4006212049B
:10A03000120C07219A8319821A8892B242F04002C8
:10A040001A80F8BD334B596A0A435A629DE70020D3
:10A050000246E1E72F4B19690A431A6195E72D4B38
:10A06000196A0A431A6290E702F564424FF400103D
:10A07000536A43F4001353622AF0A4FA6359C6E703
:10A0800002F584324FF48050536A43F48053536294
:10A090002AF098FA6359BAE702F500324FF480408B
:10A0A000136A43F4804313622AF094FA6359AEE7CB
:10A0B00002F5FE324FF40040136A43F4004313628A
:10A0C0002AF088FA6359A2E702F582324FF4005071
:10A0D000536A43F4005353622AF074FA635996E7C3
:10A0E00002F568424FF48010536A43F480135362C0
:10A0F0002AF068FA63598AE784A7002000380040F4
:10A1000000300140003C004000340140005001405C
:10A110000054014000380240427A02B9704710B53D
:10A1200004460368406804F10A01984700236372FB
:10A1300010BD00BF437A5A1C0344D2B242729972D6
:10A14000037A934200D802B9704710B504460368F9
:10A15000406804F10A0198470023637210BD00BFF4
:10A16000302828D0312828D0322828D0332828D0A9
:10A17000342828D0352828D0202828D0212828D0B5
:10A18000102828D0112828D0122828D0132828D009
:10A19000142828D0152828D0162805D0172808BF3D
:10A1A0000F2202D0002070470E22114B03EB420316
:10A1B00093F8290070470022F7E70122F5E7022211
:10A1C000F3E70322F1E70422EFE70522EDE7062299
:10A1D000EBE70722E9E70822E7E70922E5E70A2299
:10A1E000E3E70B22E1E70C22DFE70D22DDE700BF0A
:10A1F000F0E3030870B5448806460D46C4F30B042B
:10A2000022460021284634F03FF83369094A934238
:10A2100009D3094A934206D2224628461946BDE888
:10A22000704034F00CB823B121462846BDE8704098
:10A23000184770BDFC0500080207000838B5054C3A
:10A24000054DAC4200D338BD61682046FFF7D2FF10
:10A250001434F6E788010008FC050008064B07499E
:10A260008B4202D30023184670471A88C2F30B02B0
:10A270009042F8D01433F3E788010008FC05000889
:10A28000024A136823EA00001060704798600020BB
:10A29000F8B5174D2B78A32B28D16B78BE2B25D181
:10A2A000022229464FF6FF70FEF746FA114FAC1C0A
:10A2B00022884AB1A618BE4218D2052A16D92146CC
:10A2C000FEF73AFA3446F3E721460222FEF734FA63
:10A2D0000222A118FEF730FA0634074B641B1C80DB
:10A2E00041F60F53C31A58425841F8BD0020F8BD3B
:10A2F0000040000800800008284400202DE9F04FAD
:10A30000DFF84C914D4F8BB00326A7EB09071822BD
:10A31000002104A833F0B8FF494BCDF81090059701
:10A320001A69002A04DA474A5A6002F188325A60F0
:10A3300001228DF82420F322DA60434B434C1B8822
:10A34000ADF800300222694604A8FEF73DFE022265
:10A3500069464FF6FF70FEF7EFF9DFF8F8A0804688
:10A360004FF0000B544539D30AAC002524F8245D86
:10A370000222214604A8FEF727FE0222214640467B
:10A38000FEF7DAF940BAC043ADF80800022202A98C
:10A3900004A8FEF719FE079878B106ABC0F10402D5
:10A3A0002946184433F070FF089818B9069904A894
:10A3B000FEF76CFD0023089007939DF82430089A5F
:10A3C00023B11F490B6943F000430B61013E2DD0BF
:10A3D000002A9CD1FFF75CFF50B32CE065888DF814
:10A3E0000DB0C5F30B05AB1DADF808302388C3F3E2
:10A3F0000B02ADF80A201B0B062202A904A88DF857
:10A400000C30FEF7E1FD062202A94046FEF794F962
:10A41000616880462A4604A8FEF7D6FD616840467A
:10A420002A46FEF789F9143480469BE7002AD1D0EA
:10A43000052003F015FB0BB0BDE8F08F008000088D
:10A44000003C02402301674538E403088801000806
:10A4500000400008FC0500080378202B024600F1AC
:10A460000100F9D0092BF7D02D2B2CD02B2B03BFBB
:10A470005378B7EE000A0246B7EE000AA3F13001A6
:10A48000C8B209289FED467A10D8F2EE046A07EEAA
:10A49000901AF8EEE77A12F8013FE7EE267AA3F178
:10A4A0003001C8B20928B0EE677AF0D92E2B4CD013
:10A4B00003F0DF03452B0BD0F7EE007A67EE276A37
:10A4C00020EE260A70475378BFEE000A0246D5E711
:10A4D00010B451782D2959D02B290ABF9178501CDE
:10A4E000901C0024A1F13003092B53D8002303EB67
:10A4F000830301EB430310F8011FA1F13002092A85
:10A50000A3F13003F3D9B3F59A7F28BF4FF49A73C0
:10A51000072B42D9DFED236A1A46F7EE007A083A94
:10A52000072A67EEA67AFAD803F007032BB1F2EEFA
:10A53000046A013B67EEA67AFBD124B3C7EE276A13
:10A540005DF8044B20EE260A70475378A3F13001E2
:10A55000C8B2092802F10102AAD8F2EE046AF0EEAC
:10A56000665A07EE901AF8EEE77A12F8013F87EE86
:10A57000A66AA3F13001C8B2092866EEA56A37EED3
:10A58000067AEED994E767EE276AD9E7901C9178AE
:10A590000124A7E7F7EE007ACFE7F7EE007AC5E7E8
:10A5A0000000000020BCBE4CB5EEC00ADFED317AE1
:10A5B000F1EE10FACCBF30EE270A30EE670ADFED7D
:10A5C0002E7A20EE270A30B5FDEEC07A87B017EE5E
:10A5D000904A054684EAE470002303A9A0EBE470E6
:10A5E0000193009302932DF0B1FA002CACBF20230D
:10A5F0002D2303A88DF8003030F020FE012803A998
:10A6000024D002282DD0032805BF30236846684691
:10A610008DF8013033F05EFE684630F00FFE0338EF
:10A62000C4B222466946284633F0B2FE00232B55B9
:10A63000284630F003FE2E22431C2A540DEB040161
:10A64000E81833F064FE284607B030BD3023684672
:10A650008DF801308DF802308DF8033033F03AFE7A
:10A66000DAE7302368468DF801308DF8023033F098
:10A6700031FED1E76F12033A00007A442DE9F04130
:10A68000064615460846B6FBF2F43CB905FB1464D1
:10A69000124B1B5D00F8013BBDE8F081B4FBF2F703
:10A6A00067B90E4B05FB174705FB1464DA5D00F82C
:10A6B000012B1B5D00F8013BBDE8F081B7FBF2F810
:10A6C000B8F1000F02D04046FFF7D8FF05FB18781D
:10A6D000024B13F8082000F8012BE3E704140408E8
:10A6E00030B402681146531C036011F8024B01603C
:10A6F000D31C517803609378151D05601B0443EA51
:10A700000123D078234343EA006030BC704700BF88
:10A710000368591C1A46016012F8021B026058783F
:10A7200041EA0020704700BF03685A1C0260187895
:10A73000704700BF38B504460068154633F07FFD0A
:10A7400022682A44226038BD036810B40A0E5C1CDB
:10A7500004601A7003680A0C5C1C04601A700368B9
:10A760000A0A5C1C04601A7003685A1C02601970A3
:10A770005DF8044B704700BF036810B40A0A5C1C04
:10A7800004601A7003685A1C026019705DF8044B6B
:10A79000704700BF03685A1C026010B41970036848
:10A7A0000A0A5C1C04601A7003680A0C5C1C0460D2
:10A7B0001A700368090E5A1C026019705DF8044B88
:10A7C000704700BF03685A1C026019700368090AC9
:10A7D0005A1C0260197070472DE9F047002488B0B8
:10A7E00080460F461E46A14605AD531C03931178C3
:10A7F00039B3252933D1931CCDF8109003935078A9
:10A8000030284ED04FF0000AA0F13003DBB2092B04
:10A8100042D96C2819D0642800F0938024D82528C8
:10A820001CD063D9582876D063281BD13178404694
:10A83000B847039A531C0393117804360134002956
:10A84000D7D1204608B0BDE8F087039B5A1C03927D
:10A850001B78642B7CD02AD8252B54D12521404647
:10A860000134B847039AC0E7732833D044D9752818
:10A870004FD106F1040E30682B4600220A2176469D
:10A88000FDF750FE049A0095534639464046FDF7C1
:10A8900087FE039A0444A8E704AA03A91FF0B8FF9F
:10A8A000B7E7D31C039390784FF0010AACE7732B02
:10A8B00010D05BD9752B3AD0782B96D1A3F15802E2
:10A8C000B2FA82F2306852092B4610210436FDF7A5
:10A8D00029FED7E73368049A00933946002340469F
:10A8E000FDF75EFE04360444039A7EE70028B9D1E2
:10A8F000204608B0BDE8F0876E28B3D1039A3368CC
:10A9000004361C6071E72AD9582BD7D0632B8DD021
:10A910006BE77828A6D1A0F15802B2FA82F230682B
:10A9200052092B461021FDF7FDFD0436AAE706F17A
:10A93000040E30682B4600220A217646FDF7F2FD10
:10A94000A0E7331D306829461E46FDF7BDFD99E797
:10A95000331D306829461E46FDF7B6FD92E7002BF1
:10A960007FF443AF204608B0BDE8F0876E2BC6D019
:10A970003BE700BF0EB400B584B005AB019053F8BF
:10A98000042B0649039301A8FFF726FF019B002231
:10A990001A7004B05DF804EB03B0704795850008A9
:10A9A0000FB430B583B006AB0A490B4853F8042BFB
:10A9B000096800680193FFF70FFF084C05462068FF
:10A9C000FEF75AFC0028FAD0284603B0BDE8304014
:10A9D00004B07047CC3B0020D03B002004A70020EF
:10A9E000DFED2B7AB4EEE70AF1EE10FA4ADDDFED87
:10A9F000296A9FED297A01E0B0EE670AB4EEC70A32
:10AA0000F1EE10FA70EE667AF6DC9FED247AF4EE41
:10AA1000C77AF1EE10FA38D5DFED1E6A9FED207A85
:10AA200001E0F0EE407AF4EEC77AF1EE10FA37EE7C
:10AA3000A60AF6D4DFED1B7AB4EEE70AF1EE10FABF
:10AA400014DDDFED137A37EEC00A60EE006A9FED89
:10AA5000166A9FED167ADFED167AA6EE867A20EE5C
:10AA6000266AE6EE877AA6EE270A7047DFED117AAE
:10AA7000B4EEE70AF1EE10FA44BFDFED087A37EEE4
:10AA8000C00AE2E7F0EE407ABFE7B0EE670AD1E72E
:10AA9000DB0F4940DB0FC940E4CB1641DB0F49C057
:10AAA000E4CB16C1DB0FC93F92E741B99730083CB0
:10AAB00015A82ABEDB0FC9BF80EAE073A3EBE073E1
:10AAC0008B4205DB002801DD401A704702D1704738
:10AAD000002070470844704709B909E0194690FB07
:10AAE000F1F301FB13030846002BF7D1084670472A
:10AAF0000146FBE7F0EEC07AB0EEE07AB4EEE77A1A
:10AB0000F1EE10FAB4BFB0EE676AB0EE476AB5EE88
:10AB1000406AF1EE10FA46D0B4EEE77AF1EE10FAA0
:10AB20008CBFF0EE675AF0EE475AC5EE866A9FED8D
:10AB30001F3A9FED1F6A9FED1F4A9FED1F5ADFEDE1
:10AB40001F3ADFED1F4ADFED1F5AA6EEC36AE6EE9D
:10AB5000A34AA6EE864AB7EE006AA6EE845AA6EE8F
:10AB6000A46AE6EE855AC5EE866AB4EEE77AF1EE9F
:10AB700010FA48BFDFED147AF5EEC00A48BF77EE51
:10AB8000E66AF1EE10FA48BFDFED107AB5EEC00AC2
:10AB900048BF77EEE66AF1EE10FA48BFF1EE666A5A
:10ABA000B0EE660A7047DFED076ADEE739094E3D11
:10ABB000E3B59E3E88FA163E45FE7F3F99FB243F53
:10ABC00069A2163EA7DFA834DB0FC93FDB0F49405F
:10ABD000DFED317A30EE277AFDEEC76A16EE903A55
:10ABE0002033402B02D99FED2D0A7047B4EEE70ABF
:10ABF000F1EE10FA4DDD9FED2A6ADFED2A6A01E0E1
:10AC0000B0EE677AB4EEE67AF1EE10FA77EE467AB5
:10AC1000F6DC9FED257AF4EEC77AF1EE10FA35D521
:10AC2000DFED1F6A9FED217A01E0F0EE407AF4EE4D
:10AC3000C77AF1EE10FA37EEA60AF6D4DFED167AEF
:10AC4000B4EEE70AF1EE10FA1BDCDFED197AB4EE90
:10AC5000E70AF1EE10FA44BFDFED137A37EEC00ACF
:10AC600060EE006A9FED136A9FED137ADFED137AB1
:10AC7000A6EE867A20EE266AE6EE877AA6EE270A08
:10AC80007047DFED0F7A37EEC00AE9E7B0EE670AEA
:10AC9000D4E7F0EE477ABCE7DB0FC93F00000000C5
:10ACA000DB0FC940E4CB1641DB0F49C0E4CB16C132
:10ACB000DB0FC9BF92E741B99730083C15A82ABEFF
:10ACC000DB0F4940FDEEC07A17EE903A2033402B5F
:10ACD00051D8DFED2D7AB4EEE70AF1EE10FA50DD2F
:10ACE000DFED2A6A9FED2A7A01E0B0EE670AB4EE42
:10ACF000C70AF1EE10FA70EE667AF6DC9FED257A5F
:10AD0000F4EEC77AF1EE10FA38D5DFED206A9FED48
:10AD1000227A01E0F0EE407AF4EEC77AF1EE10FA12
:10AD200037EEA60AF6D4DFED1D7AB4EEE70AF1EEAF
:10AD300010FA1BDCDFED1A7AB4EEE70AF1EE10FA36
:10AD400044BFDFED147A37EEC00A60EE006A9FED73
:10AD5000156A9FED157ADFED157AA6EE867A20EE5C
:10AD6000266AE6EE877AA6EE270A7047DFED067AB6
:10AD700037EEC00AE9E79FED0E0A7047B0EE670AAA
:10AD8000D1E7F0EE407AB9E7DB0F4940DB0FC9406D
:10AD9000E4CB1641DB0F49C0E4CB16C1DB0FC93F42
:10ADA000DB0FC9BF92E741B99730083C15A82ABE0E
:10ADB0000000000010B507EE901A2DED028BB8EEE2
:10ADC000678ADFED217A28EE008A044628EE278A7A
:10ADD000B0EE480A31F08EF9F0EE408AB0EE480A43
:10ADE00031F0EAF8F7EE007A9FED187AF0EE675A44
:10ADF000E8EE875A0023A361B0EE676AC7EEA56A42
:10AE000063612362E361A8EEC76ABDEC028B77EE53
:10AE1000C07AB6EE007AF8EE005A27EE877A20EE76
:10AE2000250A27EE267A26EE266A67EEA67A20EE17
:10AE3000260A84ED046AC4ED017A84ED007A84ED7B
:10AE4000027A84ED030A10BD27D4D236F304353FCD
:10AE500010B44C09012250F8243001F01F0102FA0D
:10AE600001F10B4340F824305DF8044B704700BFFC
:10AE70004B0901F01F0150F82320012303FA01F1CF
:10AE8000114214BF18460020704700BF0C4B984277
:10AE900013D0A3F5806398420FD003F58043984206
:10AEA0000BD003F58063984207D003F58063984286
:10AEB00003D0044B186840087047024B186870476D
:10AEC00000040140C0870020F0B5774B774A87B077
:10AED0001968914200AF00F0DB800023744A3B60A8
:10AEE0007B60136843F48033136003E03B68B3F581
:10AEF000A04F09D0136803F400337B603B68013333
:10AF00003B607B68002BF1D0694B1B6813F4003366
:10AF100018BF01237B607B68012B7BD0654D644BA0
:10AF2000654AEA606549586F654A0860AA605E6BC9
:10AF3000644C654A654826F080065E635E6F46F0A5
:10AF400080765E67196B0C431C63596B5963996B70
:10AF50009963196C41F05B5141F47B1141F41F611D
:10AF600041F00F011964596C07F118040A4348F2C3
:10AF7000FF715A6444F8101D002621460123FB731B
:10AF80003E737E73BE7329F0FBF921464FF6FF73C3
:10AF90004F48BB6029F0F4F94FF6FF7321464D4846
:10AFA000BB6029F0EDF921464B4829F0E9F921462B
:10AFB0004A4829F0E5F92146494829F0E1F92146B6
:10AFC000484829F0DDF92146474829F0D9F92146BA
:10AFD000464829F0D5F9204629F0B2FB444B454CB0
:10AFE0001B68BA6844484549A4FB03439B09A0FB7E
:10AFF0000202013B920CB3F1807F0A6007D2404A03
:10B00000F0200721536085F82300966011601C37FB
:10B01000BD46F0BD264B3B4D1A6C3B4842F080527A
:10B020001A642C684268816844F440442C609C682F
:10B030009C609C6844F400449C609C6844F4A05468
:10B040009C600068120642EA801242F480024908BD
:10B0500042F00802013942EA01425A601A6842F09D
:10B0600080721A601A689201FCD52849104A40F291
:10B0700005700860996821F003019960996841F0B2
:10B0800002019960936803F00C03082BFAD145E79D
:10B0900000221A6062B61E4B1B6883F308881D4BA2
:10B0A0001B689847FEE700BFFCFF0120EFBEADDE46
:10B0B0000038024000ED00E00005FA05245D0020A4
:10B0C00000000008FF916700335F070000000240A6
:10B0D0000004024000080240000C02400010024040
:10B0E0000014024000180240001C024000200240F0
:10B0F000C0870020D34D621083DE1B4358B200206E
:10B1000010E000E00070004000000020003C024021
:10B110000000FF1F0400FF1F08B5054B1B6803B1AB
:10B120009847044B044A1A6072B6FDF731FC00BF21
:10B1300058530020FCFF0120EFBEADDE08B5034BE5
:10B140001B6803B1984772B6FDF722FC58530020E4
:10B15000084B10B507281B68C8BF143818440C46A4
:10B16000007EFEF749FA20B12146BDE81040FEF707
:10B1700099BC10BD2868002030B50446406D61714F
:10B180008389A26823F400531B041B0C838185B0C0
:10B19000A379009213F0040230D04FF4805213F0E0
:10B1A0000203ADF8042063D1ADF806304FF480639C
:10B1B0000022ADF8083011F00103ADF80C2028D1C1
:10B1C000ADF80A3008238D07694648BFADF80A304C
:10B1D00023F08CFFA279636DD10724D412F0080FFD
:10B1E0009A8A1BD122F008021204120C9A829A89C0
:10B1F00092B242F400529A8105B030BD13F00203BE
:10B20000ADF8042031D04FF400551346ADF8065088
:10B21000CEE70423ADF80A300C23D4E792B242F013
:10B2200008029A82E3E714498B421CD0A1F54C41F5
:10B230008B4216D001F580618B4210D001F5806100
:10B240008B420AD001F548418B42C7D1052001212C
:10B25000FFF77EFFA279636DC0E70320F7E70220C6
:10B26000F5E70120F3E70020F1E7ADF806309FE7AE
:10B270004FF4005398E700BF0010014010B504469A
:10B28000406DA160838923F400531B041B0C838150
:10B29000A37984B013F00402009135D04FF48052AA
:10B2A00013F00203ADF8042063D1ADF806304FF47B
:10B2B00080636279ADF80830D1074FF00003ADF834
:10B2C0000A30ADF80C3045BF0423ADF80A3008232E
:10B2D0000C236946920748BFADF80A3023F006FFF9
:10B2E000A279636DD1071FD412F0080F9A8A16D184
:10B2F00022F008021204120C9A829A8992B242F445
:10B3000000529A8104B010BD13F00203ADF804207E
:10B310002CD04FF400511346ADF80610C9E792B295
:10B3200042F008029A82E8E713498B421CD0A1F54B
:10B330004C418B4216D001F580618B4210D001F553
:10B3400080618B420AD001F548418B42CCD1052067
:10B350000121FFF7FDFEA279636DC5E70320F7E742
:10B360000220F5E70120F3E70020F1E7ADF8063011
:10B370009FE74FF4005398E70010014038B50C4B9D
:10B3800007281B68CCBFA0F11404044623440546DB
:10B39000187EFEF731F950B101342722C471827151
:10B3A0002FF07CF828460021BDE83840D0E638BDB3
:10B3B00028680020064A00235168814202F11C02DD
:10B3C00004D00133102BF7D100207047D8B270475A
:10B3D00064010020074BC0EBC00030B403EB8000D9
:10B3E000054C0569236B2B4323630176427630BC01
:10B3F000704700BF64010020003802402DE9F04F83
:10B40000614C54F8204083B0002C00F0B880E56D0A
:10B41000002D00F0B68017465C4A9846064604F1B7
:10B4200062032869226004F262226361A2614FF420
:10B4300000736A68A160E36023616265A14668B138
:10B44000FFF7B8FF721CD2B20C21FFF7C3FF636D88
:10B45000A9682A6922630433A1632365E86880B37D
:10B46000FFF7A8FF721CD2B20B218246FFF7B2FF92
:10B470004748DFF820E1EB7FDEF83010CAEBCA0A5C
:10B4800000EB8A009B0902690A43CEF83020DFF8FE
:10B4900008E1417B446100228DF80530C0F808E0E6
:10B4A000012301A88DF804108DF806208DF80730CF
:10B4B00023F0E4FD636DA968EA6862630433E16325
:10B4C000E36494F86100FEF797F8824694F8600010
:10B4D000FEF792F88346287F00284DD118F0080F18
:10B4E00036D1BA070DD5BAF1000F0AD00B22731C62
:10B4F0008AF806208AF8073050466A7F2221FEF734
:10B5000041F9FB0715D4A36B7BB9AA7F8DF8042002
:10B5100095F820208DF8063001A8930901228DF8B6
:10B5200005308DF8072023F0A9FD484603B0BDE89B
:10B53000F08FBBF1000FE6D001360C238BF80760CB
:10B540008BF8063058466A7F2221FEF71BF9DAE7AE
:10B550000136F6B2BAF1000F04D00B238AF8076067
:10B560008AF8063018F0100F504614BF022112213D
:10B570006A7FFEF707F9C6E72EF072FFAEE7A14635
:10B58000D3E7A946D1E700BFD83B00203CE403083D
:10B590006401002000380240B58900080348D0F853
:10B5A000AC3113B100F5D270184770476401002028
:10B5B0000348D0F8903113B100F5C47018477047B4
:10B5C000640100200348D0F8743113B100F5B6705F
:10B5D00018477047640100200348D0F8583113B170
:10B5E00000F5A87018477047640100200348D0F8A0
:10B5F0003C3113B100F59A70184770476401002080
:10B600000348D0F8203113B100F58C70184770470B
:10B61000640100200348D0F804310BB1FC30184716
:10B62000704700BF640100200348D0F8E8300BB138
:10B63000E0301847704700BF640100200348D0F88D
:10B64000CC300BB1C4301847704700BF64010020F4
:10B650000348D0F8B0300BB1A8301847704700BF8E
:10B66000640100200348D0F894300BB18C301847A7
:10B67000704700BF640100200248836F0BB1703037
:10B6800018477047640100200248C36D0BB1543065
:10B6900018477047640100200248036C0BB1383032
:10B6A00018477047640100200248436A0BB11C3000
:10B6B00018477047640100200248836803B11847A7
:10B6C000704700BF64010020431C00F014812DE985
:10B6D000F04F4FEAC00808EB00039B00DFF8F4A22C
:10B6E0005AF803B087B00AEB0304BBF1000F00F077
:10B6F000FF8014330AEB03010022DBF804704AF8E0
:10B7000003204A608A60CA600346A568019001333D
:10B71000D4F80C90DBB2002D00F0EE801522EB7116
:10B72000AA71B9F1000F00F00081162289F80620F5
:10B7300089F807309BF80E002EF092FEBB8823F4A8
:10B7400040731B041B0CBB802846FEF7A5F9484636
:10B75000FEF7A2F911212846FDF798FE112148466F
:10B76000FDF794FE0826642404E00A203CB102F0B0
:10B77000D1FD013C2846FEF7B7F90028F5D0284650
:10B78000FEF784F90A2002F0C5FD2846FEF784F989
:10B790000A2002F0BFFD013EECD14846FEF776F9E3
:10B7A0000A2002F0B7FD2846FEF770F90A2002F0E1
:10B7B000B1FD2846FEF770F90A2002F0ABFD4846BD
:10B7C000FEF76AF9019B08EB03040AEB84042846A0
:10B7D000637C002B0CBF122132210422FDF7D2FF23
:10B7E000637C002B0CBF1221322148460422FDF756
:10B7F000C9FF704B9F4200F0B7806F4B9F4200F033
:10B80000BD806E4B9F4200F0A580BB8801996C4AB9
:10B810006C4C23F440731B041B0CBB803B88884496
:10B820000AEB880A9BB243F001039AF810103B80A0
:10B83000BD8802A8002918BF144628F081FF049A89
:10B840006148B2FBF4F325F03F05A0FB02122D0482
:10B85000900C2D0C0543BD805C4C39884FF49672DA
:10B8600002FB00F284FB02409BB2D217002BC2EB1A
:10B87000A01221F0010108BF01230904013243F4A1
:10B880000043090C92B239803A84BB833B889BB257
:10B8900043F001033B803B8823F4816323F00203E0
:10B8A0001B041B0C43F480634FF480423B803A81BD
:10B8B0003B8823F080031B041B0C3B809BF810305B
:10B8C0008DF808300024012302A88DF80B308DF884
:10B8D00009408DF80A4023F0D1FB9BF80F308DF81A
:10B8E000083002A88DF809408DF80A4023F0ECFBDF
:10B8F00007B0BDE8F08F7047B9F1000F48D01622AD
:10B9000089F8073089F806209BF80E002EF0A8FD74
:10B91000BB8823F440731B041B0C2846BB80FEF736
:10B92000BBF84846FEF7B8F818E79BF80E002EF073
:10B9300097FDBB8823F440731B041B0CBB80284677
:10B94000FEF7AAF84846FEF7A7F811212846FDF7AA
:10B950009DFD07E71E4A136A43F4000313624FF488
:10B96000000028F037FE50E7194A136A43F4001329
:10B9700013624FF4001028F02DFE46E7144A136AB4
:10B9800043F4800313624FF4800028F023FE3CE769
:10B990009BF80E002EF064FDBB8823F440731B045B
:10B9A0001B0C4846BB80FEF777F84846FEF774F854
:10B9B000D8E600BF0054004000580040005C004042
:10B9C000009F2400804F120083DE1B43D34D621082
:10B9D00000380240003C0020F8B54FEAC00E274F67
:10B9E000069C0EEB000507EB85056E68002E42D025
:10B9F0004900C9B2A9754FF0000C0121EA7585F81C
:10BA000019C0A9762B76697585F814C0B3882C62A5
:10BA10009905EC6114D43388DA050CD44FF48054C2
:10BA200001E0013C1ED033889B05FAD433889BB2D9
:10BA300043F480733380B3889BB243F44073B38084
:10BA40000EEB000107EB81024FF4805401E0013C52
:10BA500008D0537D002BFAD107EB81073C7D84F0A1
:10BA60000100F8BD064A138801339BB21380FFF72B
:10BA70002BFE2046F8BD3046F8BD00BF003C00203C
:10BA80002644002070B590F904506C1C82B00AD096
:10BA9000032D08DC16460A46417900962846FFF732
:10BAA0009BFF02B070BD002002B070BD00B50378EE
:10BAB000012B83B004D1032301AA0021FFF7E2FF89
:10BAC0009DF805309DF804209DF806001B0243EA0E
:10BAD0000243184303B05DF804FB00BF08B5FFF74D
:10BAE000E5FF014B586008BDB41E002008B5FFF704
:10BAF000DDFF014B186008BDB41E0020F0B585B015
:10BB000002AB04460093032206231E210120FFF707
:10BB100063FF00283CD09DF808509DF809109DF85F
:10BB20000A709DF80B209DF80C609DF80D3041EADD
:10BB3000052142EA072243EA062309B212B21BB2E8
:10BB4000144D06EE901A07EE102A07EE903AF8EE22
:10BB5000E66A95ED035AD5ED055A95ED046AB8EEFF
:10BB6000C77AF8EEE77A66EE856A27EE257A67EE01
:10BB7000867AFDEEE66ABDEEC77AFDEEE77A16EE4E
:10BB8000901A17EE102A17EE903A2180A280638057
:10BB900005B0F0BD0000002000B583B00120009288
:10BBA0000A466821FFF718FF03B05DF804FB00BFE9
:10BBB000F0B5C60033189B00254DEA585468A28A98
:10BBC00083B092B20192019A2B4412F4706F1CBFA1
:10BBD00001221A75019B13F4E06F07460CD1A38A6A
:10BBE0003E4423F4706305EB86051B041B0C002206
:10BBF000A3826A7503B0F0BD238BA38823F480630E
:10BC00001B041B0CA380019B9B05E8D4238898058B
:10BC1000E5D42388D9050ED52388DA05FCD42388FA
:10BC20009BB243F40073238023889B05FCD43846E1
:10BC3000FFF74AFDD3E723889BB243F400732380C8
:10BC4000A38823F440731B041B0CA380C7E700BF29
:10BC5000003C0020F0B583B0441C8DF8073001D0C3
:10BC6000032802DD002003B0F0BDC700244E3B18BE
:10BC700006EB83035D68002DF4D04900C9B29975C5
:10BC800001240021DA755C7699761C765C7519754D
:10BC9000A9880DF107028905DA611A6214D42B888C
:10BCA000DA050CD44FF4805401E0013C1ED02B88FF
:10BCB0009B05FAD42B889BB243F480732B80AB880E
:10BCC0009BB243F44073AB80074406EB87024FF40A
:10BCD000805401E0013C09D0537D002BFAD106EBE2
:10BCE00087073C7D84F0010003B0F0BD054A13884E
:10BCF00001339BB21380FFF7E7FC2046B3E700BF98
:10BD0000003C0020264400202DE9F043322083B07F
:10BD100002F05AFB112300221E210120FFF79AFF97
:10BD20000122104660231E21FFF794FF642002F0D9
:10BD30004BFB6846FFF7E2FE0024DFF854812546FE
:10BD400026460A270123184602221E21FFF782FFFA
:10BD5000322002F039FB6846FFF7D0FEBDF902E061
:10BD6000BDF90410BDF900208E457346A8BF0B46EF
:10BD70009342A8BF134643454FF0010075440C445D
:10BD8000164479DBFDF7A6FA013FDBD14FF001093C
:10BD9000122300221E210120FFF75CFFDFF8F08054
:10BDA0000A270123184602221E21FFF753FF3220E3
:10BDB00002F00AFB6846FFF7A1FEBDF902E0BDF9FB
:10BDC0000410BDF900208E457346A8BF0B46934270
:10BDD000A8BF134643454FF00100A5EB0E05A4EBA9
:10BDE0000104A6EB02064ADBFDF774FA013FD8D145
:10BDF00007EE906AF8EEE76A07EE905AB8EEE77A37
:10BE000007EE904ADFED1F5A9FED1F5A1F4EF8EEC6
:10BE1000E77A85EEA66A702300221E210120C5EE76
:10BE2000876A85EE277AB0EEC66AF0EEE66AF0EE33
:10BE3000C77A86ED036AC6ED046AC6ED057AFFF798
:10BE400009FF0122104620231E21FFF703FF0023D4
:10BE500002221E210120FFF7FDFE642002F0B4FA49
:10BE6000B9F1000F04D14FF07E53F3603361736179
:10BE7000012003B0BDE8F0834FF0000988E74FF0E0
:10BE80000009B5E700406F4601C05E460000002093
:10BE900001F0FFFF0378012B00D07047417990F942
:10BEA00004005822D6E600BF0378012B00D070476B
:10BEB000417990F904004822CCE600BF13460120E6
:10BEC0000A466821C6E600BF0220FCF71FBE00BF7D
:10BED00002206DE60120FCF719BE00BF012067E6D5
:10BEE0000020FCF713BE00BF002061E61549164B89
:10BEF00016480A6810B48C681549B2FBF4F203FBCB
:10BF000002F30360D1F88820124B134C42F4700204
:10BF1000C1F888201A68002042F001021A60986077
:10BF20001A6822F0847222F480321A605C601A6807
:10BF30004FF0006422F480221A60D8608C605DF8B3
:10BF4000044B70470000002040420F00C0870020D3
:10BF500000ED00E00038024010300024044B4FF4A4
:10BF6000F0700A21022283E80700FFF7BFBF00BF7D
:10BF70000000002038B50B4C23688BB15A68821A38
:10BF8000002A054604DA0CE05A68AA1A002A07DBE0
:10BF90009A68226018461A6890472368002BF3D1EC
:10BFA00038BD38BD885600200B4B002210B40272F9
:10BFB00003F5C074022102E0072A09DC9979890798
:10BFC00002D51979815401329C4203F11803F3D14F
:10BFD0005DF8044B704700BF9406040810B40D4C84
:10BFE00002232146002200E08B7913F0010301F1C6
:10BFF000180106D10132112AF6D103705DF8044B05
:10C00000704702EB420204EBC2025DF8044B137965
:10C010000370704794060408012310B432213324BE
:10C02000312244704171C2700370037183705DF8F6
:10C03000044B704708B51AF053FCFFF77FF800BFB8
:10C04000024A034B1278197818F04EBF9C21002049
:10C050009D210020038A2DE9F0478589ADB21D405E
:10C0600029D00F4606464FF000484FF00009B5FAB8
:10C0700085F328FA03F2D24391B21B3B154031827B
:10C08000042B16D8DFE803F03129211903007B6A5D
:10C09000002B32D003F1FF3A1FFA8AFAC7F8249036
:10C0A0003C6A34B123682046514698476468002CA6
:10C0B000F8D1002DDBD1BDE8F0873868716B0368DB
:10C0C00089B29847002DD2D1F5E77868B16B036843
:10C0D00089B29847002DCAD1EDE7B868F16B0368C3
:10C0E00089B29847002DC2D1E5E7F868316C036842
:10C0F00089B29847002DBAD1DDE7F36A1FFA83FAB7
:10C10000CEE700BF2DE9F04F2DED028BA0F10A0321
:10C1100089B00C46E72B00F29E86DFE813F01C0185
:10C120009C069C069C069C069C069C069C069C06FF
:10C130009C069C069C069C069C069C069C069C06EF
:10C140009C069C069C069C069C069C069C068D01F3
:10C150009C069C069C067E019C069C069C06710122
:10C160009C062D019C069C069C069C069C063F0294
:10C170009C061A029C06EE019C069C069C06E801A1
:10C18000E1019C06DA019C069C06D3019C06AB01EA
:10C190009C069C069C0676049C069C069C069C06B7
:10C1A00057049C06FC009C06610649059C069C06FB
:10C1B0009C069C069C069C069C06EB049C06BD0403
:10C1C0009C0689049C066D059C0687069C069C06B9
:10C1D0009C069C06FF02FB05F305C205E80022034E
:10C1E00081026A02F3029C06BC02A0029C069C0625
:10C1F0009C069C0695029C069C06CF039C069C060A
:10C200009C06970380036C039C069C069C069C0678
:10C210005D034603480428049C069C069C069C0675
:10C220009C069C069C069C069C069C069C069C06FE
:10C230009C069C069C06FF029C069C069C069C068F
:10C240009C069C069C069C069C069C069C069C06DE
:10C250009C06F0039C069C069C069C069C069C067D
:10C260009C069C069C069C069C069C069C069C06BE
:10C270009C069C069C069C069C069C069C069C06AE
:10C280009C069C069C069C069C069C069C069C069E
:10C290009C069C069C069C069C069C069C069C068E
:10C2A0009C069C069C069C069C069C069C069C067E
:10C2B0009C069C069C069C069C069C069C069C066E
:10C2C0009C069C069C069C069C069C069C069C065E
:10C2D0009C069C069C069C069C069C069C069C064E
:10C2E0009C069C069C069C069C065F023606AF4E8A
:10C2F000337853B1AE4F002537F8021F2046FEF7C2
:10C3000061FA33780135AB42F6DC012009B0BDECAF
:10C31000028BBDE8F08FA54E3378002BF5D0A54FEA
:10C320000025B846236817F81520591C21601A709B
:10C3300098F8011001EB810101EB810101F2EE217E
:10C3400089B22046FEF73EFA33780135AB4208F158
:10C350000208E7DCD9E7984D28462EF06FFF002849
:10C36000D3DD2B460544226813F8011B501C9D4267
:10C3700020601170F7D1C8E7904D0B682A7A591CDC
:10C3800021601A70A98B2046FEF71CFA298B2046E3
:10C39000FEF718FA698B2046FEF714FA2368EA7C48
:10C3A000591C21601A70A98C2046FEF70BFAE98C03
:10C3B0002046FEF707FA2368AA7F591C21601A70ED
:10C3C000236895F82020591C21601A70698C20463A
:10C3D000FEF7F8F92368EA7A591C21601A70E968B7
:10C3E0002046FEF7D7F923682A7C591C21601A7071
:10C3F000236895F82120591C216001201A7085E7D7
:10C400000B686F4A581C11782060197023685278A5
:10C41000591C216001201A7078E76A4D0846298866
:10C42000FEF7D0F9A9882046FEF7CCF920462989E5
:10C43000FEF7C8F9012069E7634D05F15006287839
:10C440002DF0F4FF2368027A591C21601A702368CA
:10C450006A78591C21601A702368AA78591C2160D7
:10C460001A702368EA780435591CAE4221601A70AC
:10C47000E5D14AE70B68524A524D1178534A581C8D
:10C480002060197011682046FEF784F923684B4A32
:10C49000591C127A21601A7029882046FEF792F9F9
:10C4A000A9882046FEF78EF929892046FEF78AF9E9
:10C4B00000212046FEF786F920460021FEF782F98A
:10C4C000012023E7084608223C49FEF733F9012002
:10C4D0001CE70B683E4A581C91782060197095E75C
:10C4E0000B6801229918216010461A700EE7084661
:10C4F0000021FEF74FF9012008E7364D05F140070E
:10C5000003E00835BD423FF400AF95F902603046C4
:10C5100012F09EFC0028F4D023685A1C22601E7082
:10C5200029882046FEF74EF92368EA78591C2160D5
:10C530001A7023682A79591C21601A702368AA7915
:10C54000591C21601A7023686A79591C21601A707D
:10C55000D7E7214B03F15A0522685979501C206016
:10C56000117022681978501C206011702268597867
:10C57000501C2060117022689978501C2060117046
:10C580002268D978501C206011702268197906330E
:10C59000501C9D4220601170DED1B6E60B68074A40
:10C5A000591C527D216001201A70AFE66C470020B3
:10C5B00002A600207877002054600020F85C00205C
:10C5C000A4600020783C0020A86000209860002033
:10C5D00094600020486E002048440020A24D084688
:10C5E000E989FEF7EFF82046A989FEF7EBF801206C
:10C5F0008CE69E4D08462988FEF7E4F869882046B7
:10C60000FEF7E0F8B5F90430994AD91782FB032305
:10C61000C1EBA301204689B2FEF7D4F8012075E6EC
:10C62000944B08461988FEF7CDF8934B204619889D
:10C63000FEF7C8F8914B22681B78511C03F00103E8
:10C6400021600120137061E68D4952232268501C3D
:10C650002060137011F8013F002BF7D155E689488F
:10C6600000232268056803EB4301561C6D5C2660BD
:10C670001570026825680A446E1C527826602A707C
:10C68000026825680A4401339278691C0A2B2160EC
:10C690002A70E6D139E67C4D0B682A68591C12785D
:10C6A00021601A702B6822689978531C236000233C
:10C6B00011702A6821681A4401335279481C032BEF
:10C6C00020600A70F5D123682A68591C127A21600B
:10C6D0001A7023682A68591CD27821601A7023685E
:10C6E0002A68591C127921601A702B6820465989D2
:10C6F000FEF768F82A682368527A591C21601A707C
:10C700002A6883E6614B08461968FEF743F8604BD8
:10C7100020461988FEF756F80120F7E500258146E6
:10C72000DFF89081DFF890B105950495069507959F
:10C7300001214FF6FF7A05E001350B2D00F08E83C5
:10C7400018F9011F4F1C4AFA05F3F5D0DE07F3D59F
:10C75000BBF800302B41D807EED506A8FEF778FBD2
:10C76000EAE74C4B0A681B784B4D511C03F002035F
:10C770002160137023682A7D591C21601A70296872
:10C780002046FEF707F869682046FEF703F8298976
:10C790002046FEF717F8E9892046FEF713F82046F1
:10C7A000298AFEF70FF80120B0E50A683B4B501CC0
:10C7B00019782060117022685978501C206011701F
:10C7C00022689978501C206011702268DB78511C17
:10C7D00021600120137099E5314D0846298AFDF743
:10C7E000F1FF698A2046FDF7EDFF2046A98AFDF793
:10C7F000E9FF01208AE50B682A4A1B4910782A4A7A
:10C800005D1C2560187023688978581C2060197099
:10C8100023689278591C216001201A7076E50A6815
:10C82000224B23491878551C2560107022685878CF
:10C83000551C2560107022689B78501C2060137076
:10C840002046C988FDF7BEFF01205FE5184D084668
:10C850002988FDF7B7FF69882046FDF7B3FFA9884F
:10C860002046FDF7AFFF50E578600020B07400204F
:10C8700067666666B4640020B664002068640020C1
:10C8800064E40308F84600202C440020AC74002027
:10C89000A0740020D0740020D47400209C65002077
:10C8A00024580020545B0020886000207060002025
:10C8B000B04F002094E40308CC640020AF4D05F194
:10C8C0006006A9882046FDF77DFFE9882046FDF730
:10C8D00079FF29892046FDF775FF2368AA7A591C3C
:10C8E00021601A702368EA7A591C21601A7055F881
:10C8F0000C1B2046FDF74EFFAE42E2D105E50B686A
:10C90000DFF8A8C2591C9CF8002021601A709CF81E
:10C910000030002B3FF4F9AC994E9A4D9A489B4950
:10C920000023226816F8017F02F1010EC4F800E02E
:10C930001770226815F8017F02F1010EC4F800E0BB
:10C940001770226810F8017F02F1010EC4F800E0B0
:10C950001770226811F8017F02F1010EC4F800E09F
:10C9600017709CF8002001339A42DADCCDE40B68A2
:10C97000874F591C3A7821601A703B78002B3FF49E
:10C98000C4AC0025EEB2304623F0FCF823684278B0
:10C99000591C216030461A7023F0F4F801892046B2
:10C9A000FDF710FF3B780135AB42EBDCADE4794B92
:10C9B0007949B3F9003081FB0321DB17C3EBA101F7
:10C9C000204689B2FDF7FEFE01209FE40B68734DFF
:10C9D000591C2A7921601A7023686A79591C2160D0
:10C9E0001A7029882046FDF7EDFE2368AA79591CA4
:10C9F00021601A7069882046FDF7E4FE2368EA7911
:10CA0000591C216001201A7080E40B6800255A1C13
:10CA10000A6020461D702946FDF7BCFE29462046C7
:10CA2000FDF7B8FE20462946FDF7B4FE01206DE46F
:10CA30005B4E0B6872795B4D591C21601A702B6834
:10CA40002046198CFDF7BEFE2B682046D98BFDF7DA
:10CA5000B9FE71892046FDF7B5FEB1892046FDF784
:10CA6000B1FE2B682046598CFDF7ACFE2B682046A2
:10CA7000998CFDF7A7FEF1892046FDF7A3FE318AC8
:10CA80002046FDF79FFE2A68236892F82620591C4D
:10CA9000216001201A7039E4414EF378002B00F038
:10CAA000B7820B680822591C21601A702368012282
:10CAB000991821601A7023683B4D591C2A7921600E
:10CAC0001A702368AA78591C21601A702988204698
:10CAD000FDF778FEE9892046FDF774FE2368F279B8
:10CAE000591C21601A702368EA78591C21600120C2
:10CAF0001A700BE418F0DCF9FF28064600F0948267
:10CB000008A9002501F8125D0DF10D008DF80D50FA
:10CB10002BF086F908A800F8115D2BF075F908A82C
:10CB200000F8105D2BF064F908A820F8085D18F0F3
:10CB30009FF923685A1C22601E7023689DF80D20FF
:10CB4000591C21601A7023689DF80E20591C216021
:10CB50001A7023689DF80F20591C21601A702368F1
:10CB60009DF81020591C21601A702046BDF818103D
:10CB7000FDF728FE0120FFF7C9BB00BF30500020A1
:10CB8000B7650020C7650020E7650020D765002055
:10CB9000D1610020886000206766666668450020D5
:10CBA000545B0020F846002024580020B565002082
:10CBB0000B68BC4E01255A1C0A601D700B68B278C8
:10CBC000591921601A701FF06DFA2368B64AB749E7
:10CBD0005F1927601870B1F90010B2F90000FDF775
:10CBE0007BFF23685A192260187031882046FDF7B0
:10CBF000E9FD2846FFF78ABB00212046FDF7E2FD4C
:10CC000000212046FDF7DEFD00212046FDF7DAFD7C
:10CC10002368A74D00265A1C22601E7023682A68CC
:10CC2000591C92F82C2021601A7023682A68591C1C
:10CC300092F8362021601A7023682A68591C92F8ED
:10CC4000372021601A7023685A1C22601E702368E6
:10CC50005A1C22601E7023685A1C22601E702B68AA
:10CC60002046598FFDF7AEFD2B682046198FFDF742
:10CC7000A9FD23682A68591C92F82E2021601A7099
:10CC800023685A1C22601E702B682046598EFDF7BF
:10CC900099FD2B682046998EFDF794FD0120FFF742
:10CCA00035BB844D844E9FED858ADFF85082DFEDE1
:10CCB000848A05F120070EE0FCEEE77ACDED017ADB
:10CCC000BDF8041020460435FDF77CFDAF4206F1A7
:10CCD00018063FF41AAB717C0029F3D0794BD5EDDF
:10CCE000007A1B78012BE7D1774B1B68DB0440F1FE
:10CCF0008581F5EE407AF1EE10FA40F0AE8140F217
:10CD0000DC51DFE7084610227049FDF713FD0120D2
:10CD1000FFF7FCBA6E4B9B8AB3F5006F00F2768189
:10CD2000B3F5806F00F29781B3F5007F34BF012720
:10CD30000227684D05F10C0655F8041B91FBF7F12D
:10CD4000204689B2FDF73EFDB542F5D1624D634FF5
:10CD500005F10C06B5EC010AD7ED087A80EE270A3A
:10CD60002FF07CF981B22046FDF72CFDAE42F1D1C7
:10CD70005B4D05F10C0655F8041B204689B2FDF702
:10CD800021FDB542F7D1FFF7C0BA564B03F170054C
:10CD900022681978501C2060117022685978501C44
:10CDA0002060117022689978501C206011702268F0
:10CDB000D978501C2060117022681979501C2060AD
:10CDC000117022685979501C20601170226899797D
:10CDD0000733501C9D4220601170D9D1FFF795BADE
:10CDE0000A68414D511C01232160137095F82420DD
:10CDF0003E49002A40F04D812268501C206013708B
:10CE0000236841F2B4105A1C085C226041F2781287
:10CE1000187089582046890AFDF7BCFCA96A20468B
:10CE20004908FDF7B7FC0120FFF770BA0B68304ADC
:10CE30003049D078304A5D1C2560187023684979E4
:10CE4000581C206019702368D278591C2160012079
:10CE50001A70FFF75BBA0020FFF758BADFF8A0A0FE
:10CE600000254FF008080135C5F1200208FA02F24A
:10CE7000A5F120032AFA05F6164328FA03F31E4308
:10CE8000252D06F001024FF000033BD01343EAD0FA
:10CE9000E8B22CF0ADF90028E5D0294606A8FDF748
:10CEA000D7FFE0E720710020D25E0020D45E002092
:10CEB000F8460020785E00206457002000004042C1
:10CEC00000E0824448580020785B0020685E002023
:10CED00058740020907400206C5B0020B4A70020E0
:10CEE000204700203C490020D8A4002028900020A2
:10CEF00078600020A467002088600020DB9B9141BF
:10CF000090E33FF4794B1B78DA0700F19480002519
:10CF1000774E2F4602E00135252D0DD029463046AB
:10CF2000FDF7A6FF0028F6D0294606A8FDF7A0FFCA
:10CF300000285ED10137EEE76E4B6F4DB3F850100D
:10CF40002046FDF73FFC6D4B1988204689B2FDF75E
:10CF500039FC6B4B19684B0103F02002C1F340030D
:10CF60001343C1F3800243EA4203C1F3C00243EA20
:10CF70008203C1F3401243EAC20301F010011943D6
:10CF80002046FDF71FFC04A904222046FDF7D2FB32
:10CF9000236829785B4A581C20601970118864291D
:10CFA000A8BF64212046FDF70DFCB9F1960F47D0CC
:10CFB00000212046FDF706FC2168B7F1190348BFA0
:10CFC000A7F11203A3F3C4034A1C226020461A46A9
:10CFD0000B7005A9FDF7AEFB23684B4A581C1021C6
:10CFE0002060197020461188FDF7D4FB0120FFF75F
:10CFF0008DB9394604A8FDF72BFF9BE7F4EEC87AFC
:10D00000F1EE10FA4DDA4FF47A715BE6082790E6FC
:10D010000B68B1783D4A581C20601970236812785B
:10D02000591C21601A7046E523685A1C22600120B1
:10D030001E70FFF76BB9069B43F00103069366E78A
:10D0400023680322591C21601A7023686A78591CCE
:10D0500021601A70B0E704276BE6F4EEC87AF1EEAF
:10D0600010FA3FF54CAEF4EEE87AFDEEE77AF1EE19
:10D0700010FA17EE901A2BD86FF4F973303903FBBE
:10D0800001F140F2E73391FBF3F101F2DB5189B298
:10D0900018E64B78022B16D0032B0CBF0423012378
:10D0A000AAE6FDEEE77A40F2E73217EE903A303B1F
:10D0B00002FB03F388FB0312D917C1EB622101F2D3
:10D0C000E93189B2FEE5042A34BF0223032393E643
:10D0D00040F2F313A1F5836103FB01F140F2E73362
:10D0E00091FBF3F101F2DD5189B2EBE560620020C2
:10D0F0007CA70020F8030020EC46002026440020F6
:10D10000CC7400202A440020227500206C6000208E
:10D1100008B501210220FCF7CDFC094B1B7803F078
:10D120000503052B08D000210120FCF7C3FC0021DA
:10D130000846FCF7BFFCFEE719F064FCF3E700BF0C
:10D14000D43B0020022828BF022010B4084C094B11
:10D15000207000EB8002C0EBC20207495DF8044B6F
:10D16000013003EB4203C0B20B6013F0FDB900BF06
:10D17000EC46002004700020F846002010B5FDF7B2
:10D180005DF8094A094B0A490A4C0B481460002211
:10D190001A705A7008601BF043FFFDF7AFF8BDE846
:10D1A00010401BF025BF00BFF8460020EC460020D1
:10D1B0002C44002004700020FC46002008B51BF021
:10D1C0002FFFFDF79BF8BDE808401BF011BF00BF23
:10D1D00038B5484B5A899989914224BF00225A8117
:10D1E000198ADA89914224BF0022DA81DA78CAB139
:10D1F000072A41496AD091F85700404D0124002187
:10D200000A282C709C70D9715DD00C2807D0002A98
:10D210006CD0DFED3B7A072A0ED00A2862D0DFED12
:10D22000397A09E0344A92F857000A2856D00C2877
:10D230005BD1D979DFED347A344C9FED350AA27891
:10D24000002918BFF0EE407A062A04D8314901EBD4
:10D25000820191ED0F0A217979B1013A032A0BD8A5
:10D26000F7EE007A87EE800A2EF0F8FE23889842C7
:10D2700028BF1846208038BD38BD9B781F4A07EE6E
:10D28000103A1178B8EEC77A67EE277A07EE101ACF
:10D29000B8EEC77A27EE277AB4EEC70AF1EE10FA95
:10D2A000EADD80EE277AFDEEC77A17EE903A102B72
:10D2B000A8BF1023012BB8BF0123DBB28B4238BFBC
:10D2C0000B46137038BDDFED147AA4E791F85700D0
:10D2D0000A2803D00C28ACD0D9799AE7D979DFEDA8
:10D2E0000E7AA9E7DFED0D7AA6E7D979DFED047AAA
:10D2F000A2E700BF545B0020B4A700206C600020B0
:10D300006F1203396F12833A0AD7A33924580020C9
:10D310006F12033864E403085304E9380F506E3A7F
:10D320002DE9F84F4FF48C7200218B488B4C8C4DBB
:10D330008C4E8D4FDFF84C82DFF84C9230F0A4FF1A
:10D340008A488B49DFF844E2DFF844C200221358D0
:10D350008B4200F0C280B3F1804F00F0D180AB422D
:10D3600000F0D580B34200F0D580BB4200F0D580FC
:10D37000734500F0D580634500F0D580434500F04B
:10D38000D5804B4500F0D580DFF808A2534500F06A
:10D39000D3800AF5806A534500F0D180AAF5983A07
:10D3A000534500F0CF800AF5806A534500F0CD80E8
:10D3B0000AF5806A534500F0CB801832B2F5CC7F75
:10D3C000C5D16A4E6B4F06F5CC784FF0030A4FF08B
:10D3D000020902E0183646457DD0B379002BF9D01A
:10D3E00033791C09013C042C03F00F03F2D8624A84
:10D3F00032F8140040FA03F2D207EBD5012505FA02
:10D4000003F3013B18402EF0C3FB5C4B1B5D18443B
:10D4100017EBC002DED057F83030594C317A03F1A7
:10D420003F4000F57E00800A205C00F01F044009A8
:10D43000032805FA04F55DD0042855D0022804D14C
:10D440004648406C054345484564B2F804E0BEFADE
:10D450008EF2C2F11F0292B2D00803EB800002F0FC
:10D460000702046A92000F25954024EA050404622D
:10D47000046A01FA02F22243002502624FF0010C15
:10D480002A4603E0102A05F10205A3D00CFA02F0A7
:10D4900030EA0E0102F10102F4D11C680AFA05F12A
:10D4A000C9430C401C60D3F800B009FA05F444EA03
:10D4B0000B041C609C680C409C609C689C605C68D1
:10D4C00024EA0000586058685860D8680140D96064
:10D4D000D968D960D6E7BDE8F88F4FF0010A636CD0
:10D4E00043EA0A03636468E71C48006B05431B4872
:10D4F0000563AAE71948006C054318480564A4E7CA
:10D500004FF0010A236C43EA0A03236455E74FF006
:10D51000020AF7E74FF0040AF4E74FF0080AF1E7D0
:10D520004FF0100AEEE74FF0200AEBE74FF0020A47
:10D53000D5E74FF4803AD2E74FF4003ACFE74FF403
:10D54000802ACCE74FF0400ADCE74FF0800AD9E7A9
:10D550004FF4807AD6E700BF683D002000380240D3
:10D560000004004000080040000C0040940604083D
:10D57000000001409CAF0020F8130408F0130408D9
:10D58000E81304080004014000400140001000407E
:10D59000001400400044014001490248FEF75ABD12
:10D5A000583E00200040014001490248FEF752BDAC
:10D5B000303E00200004014001490248FEF74ABD08
:10D5C000303E00200004014001490248FEF742BD00
:10D5D000083E0020000C004001490248FEF73ABD19
:10D5E000E03D00200008004001490248FEF732BD3E
:10D5F000B83D00200004004002494FF08040FEF793
:10D6000029BD00BF903D002001490248FEF722BD20
:10D61000683D00200000014001490248FEF71ABDA4
:10D62000683D002000000140F0B504684D4DA30A9C
:10D63000AB427AD009D94C4DAB426ED00F35AB42DC
:10D640005AD0103DAB4274D0F0BD023DAB4268D021
:10D6500056D8B3F5801F70D14FF0480E0126477998
:10D66000B0004FEA970C002968D063460227A589CD
:10D670009F4083190CEB43032F4303F1040C3B4DF4
:10D68000BFB245F8231045F82C20A781EFF3118194
:10D69000502282F31288821905EBC2021369002B13
:10D6A00032D013620433821905EBC202576917B1F5
:10D6B0001F6053690433821905EBC202976917B1E1
:10D6C0001F6093690433821905EBC202D76917B151
:10D6D0001F60D36904330027CAB21F6082F3118828
:10D6E000304405EBC000036A8BB9A38923F0010322
:10D6F0001B041B0CA381F0BD4FF4887E0626AEE709
:10D700004FF0980E0326AAE705EB0E03CBE7A3899B
:10D710009BB243F00103A381F0BD4FF0E80E052654
:10D720009DE74FF0700E022699E74FF0C00E0426D9
:10D7300095E74FF0200E002691E7F0BD0223BF08C9
:10D7400003FA07F7A389094D9BB223EA0703871958
:10D750000CEB470CA3810CF1040345F82C1045F8A1
:10D76000232093E70300100041001000683D0020D3
:10D7700010B5036883480139834282B089B200F052
:10D78000CB80A0F58060834200F0C68000F5804029
:10D79000834200F0B88000F58060834200F0B380DF
:10D7A00000F58060834200F0AE80774C18882468D2
:10D7B0006408B4FBF2F4013CA4B282B2B3F1804F2E
:10D7C0000AD07248834207D000F58060834203D0BC
:10D7D00000F58060834202D122F0700292B26C4860
:10D7E000834200F0A28000F58060834200F0A780B1
:10D7F00022F4407200F56C4092B283421A80D962E2
:10D800001C854FD05F4A93424CD001229A821A88DD
:10D8100092B242F001021A80B3F1804F00F0998079
:10D820005A4A934200F0978002F58062934200F0DA
:10D83000948002F58062934200F0918002F580624C
:10D84000934200F08E8002F58062934200F08B805C
:10D8500002F57042934200F0888002F570529342C4
:10D8600000F0858002F58062934200F0828002F52C
:10D87000806293427FD0A2F5983293427DD002F528
:10D88000806293427BD002F58062934208BF0D22F2
:10D8900015D002A84FF0012340F8043D21F0EEFB23
:10D8A00002B010BD0122002119869A821A883948D7
:10D8B00092B242F0010283421A80ADD10A46364B41
:10D8C00003EBC20301A893F85D408DF804400123E7
:10D8D00000228DF805308DF807308DF8062021F0F4
:10D8E000CDFB1B2C08D02E2CDAD12C4B019301A898
:10D8F00021F0C4FB02B010BD294B019301A821F017
:10D90000BDFB02B010BD204C18882468B4FBF2F4B3
:10D91000013CA4B282B251E71B4C18882468B4FBC6
:10D92000F2F4013CA4B282B256E701201A80D96217
:10D930001C8598821A8892B202431A8070E70120EF
:10D940001A80D9621C8598821A8892B202431A8082
:10D9500062E70122B3E70222B1E70322AFE7042224
:10D96000ADE70522ABE70622A9E70722A7E70822D1
:10D97000A5E70922A3E70A22A1E70B229FE70C22D1
:10D980009DE700BF00040140C08700200004004064
:10D99000001000400000014064E403082C01000175
:10D9A000190100012C4B98423DD0B0F1804F3CD082
:10D9B000A3F57C4398423AD003F58063984238D06F
:10D9C00003F58063984236D003F58063984234D0E3
:10D9D00003F58063984232D003F57043984230D00B
:10D9E00003F5705398422ED003F5806398422CD0F3
:10D9F00003F5806398422AD0A3F59833984228D043
:10DA000003F58063984207D003F58063984208BF0E
:10DA10000D2202D0002070470C22104B03EBC203F2
:10DA200093F85C0070470022F7E70122F5E7022235
:10DA3000F3E70322F1E70422EFE70522EDE70622F0
:10DA4000EBE70722E9E70822E7E70922E5E70A22F0
:10DA5000E3E70B22E1E700BF0000014064E40308B4
:10DA60002DE98048013085B0C3B203938A4D8B4FB6
:10DA70008B4C8C4E0A230293DFF82C9223F00EFD80
:10DA80004FF4FA7A4FF0100C4FF47A70D9F8043052
:10DA9000C3F30803002B40F0C180EFF31183002B88
:10DAA00040F0BC802968A26800BF2B689942F9D178
:10DAB000D7F800E000FB0EF39B1AB3FBFEF300FB6C
:10DAC00001314FF0010E0191D9F80430C3F308037E
:10DAD000002B40F08780EFF31183002B40F0828011
:10DAE0002B68A16800BF2A689342F9D1D7F800B02B
:10DAF00000FB0BF2521AB2FBFBF200FB0323019A6C
:10DB00009B1AB3F57A7FDFD3BAF1010ABED1039B2A
:10DB1000002B40F0BD804FF47A7ADFF88C915046AC
:10DB20004FF0100CD9F80430C3F30803002B40F079
:10DB30009280EFF31183002B40F08D802968A2685A
:10DB400000BF2B689942F9D1D7F800E000FB0EF333
:10DB50009B1AB3FBFEF300FB01314FF0010E019164
:10DB6000D9F80430C3F3080303BBEFF31183EBB917
:10DB70002B68A16800BF2A689342F9D1D7F800B09A
:10DB800000FB0BF2521AB2FBFBF200FB0323019ADB
:10DB90009B1AB3F57A7FE3D3BAF1010AC2D1029B93
:10DBA000013B02937FF468AFFDF7B6FAEFF31188FB
:10DBB0008CF31288A1682368DB0344BFC6F800E039
:10DBC000A1682B6832685FFA88F888F31188D7F863
:10DBD00000801A4400FB08F35B1AB3FBF8F300FB68
:10DBE0000233D4E7EFF311888CF31288A16823681D
:10DBF000DB0344BFC6F800E0A1682B6832685FFA17
:10DC000088F888F31188D7F800801A4400FB08F3DD
:10DC10005B1AB3FBF8F300FB023370E7EFF31182FA
:10DC20008CF31288D4F808E02368D90303D50123C4
:10DC30003360D4F808E02B683168D2B282F31188DF
:10DC40003A68194400FB02F3A3EB0E03B3FBF2F3B3
:10DC500000FB013135E7EFF311828CF31288D4F821
:10DC600008E02368D90303D501233360D4F808E022
:10DC70002B683168D2B282F311883A68194400FBEC
:10DC800002F3A3EB0E03B3FBF2F300FB013164E7F5
:10DC900018462CF055FD3EE754B2002058B2002043
:10DCA00010E000E050B2002000ED00E02DE9F04768
:10DCB000B04FB14E1BF0B4F9BE421ED2DFF8448320
:10DCC000DFF844934446258862197DB14A450DD258
:10DCD000052D0BD933886188C3F30B03994200F0FB
:10DCE000F680144625886219002DEFD17168304600
:10DCF0001436FCF77FFABE42E4D3A04A1378A3F1AE
:10DD0000170102290FD99E4911F83300002840F06D
:10DD10002381D8000144497829B19A4911F8333058
:10DD20000BB918231370984C6378022B84BF00231F
:10DD300063702378022B84BF00232370934B9A785F
:10DD4000042A00F0008132B91A88B2F5F07F84BF4E
:10DD50004FF4F0721A808E4D8E4A2B681A40002ABA
:10DD600000F00381D80700F1E980590400F1E18057
:10DD70001A0700F1D9809B0400F1CF80864D2B68F3
:10DD80005A8C998C914224BF00225A84FFF720FAC2
:10DD90001CF0D4FA002800F0BC804FF40070FCF7AF
:10DDA0006FFA4FF48030FCF76BFA4FF48020FCF7E9
:10DDB00067FA4FF40010FCF763FA4FF00070FCF7BD
:10DDC0005FFA4FF08060FCF75BFA6378022B06D8AD
:10DDD000724A734903EB430302EB83030B6023781E
:10DDE000022B07D803EB83016E4AC3EBC10302EB9E
:10DDF00043032B602BF074FA002130226A4830F084
:10DE000043FA286818F01EFA684B2D6803F1500198
:10DE100002E0043399427AD01A78002AF9D19C782A
:10DE2000D8788442F5D26249624B0A7028461D6058
:10DE300016F0B6FF604B614A1E7961496148624B3A
:10DE40001160C825642212FB0652604C406B31F809
:10DE5000061C5A60002221809A60DA601A615A61B9
:10DE60009A61DA6183F8202083F8212008B11AF042
:10DE70009DFF574B9FED575A1B88574A9FED576A96
:10DE80005579574C57495848086006EE903AF8EED5
:10DE9000E66A1388C5EE265A07EE103A53881279BF
:10DEA000C4ED005A07EE903AB8EEC77A4F4BF8EE41
:10DEB000E77A1D725A7227EE067A67EE867ABDE817
:10DEC000F04783ED017AC3ED007A1BF091B86379D6
:10DED0009B077FF406AF716894F804A03046FCF706
:10DEE00089F93388BAEB133F04D01436BE42FFF4ED
:10DEF000E9AE02E773887068AA1FC3F30B039A4266
:10DF000004F10601A8BF1A4630F099F9EDE70122A5
:10DF100089E7374810F042FE3FE73648FCF7B0F992
:10DF20004020FCF7ADF929E73348FCF7A9F92B6845
:10DF300021E73248FCF7A4F92B6819E73048FCF7D1
:10DF40009FF92B6811E79A8AB2F57A7FBFF403AF85
:10DF50004FF47A729A82FEE6D8000C186468002C9E
:10DF60007FF4D8AE17241470D4E643F008032B6076
:10DF7000F8E600BFFC05000888010008A460002046
:10DF8000240C040898020408EC46002024580020C1
:10DF90009860002009600002F8460020FC4600203E
:10DFA0002C4400200470002050220020A860002093
:10DFB000D81C0020842200206845002054A700209F
:10DFC0007E6000205874002044470020E452002066
:10DFD0008C240020C0C9FB48C81E002017B7D138C8
:10DFE00090240020F84300203661023DD4430020F5
:10DFF000486E002009400002016000020920000272
:10E0000008600002024000080080000808B51BF00C
:10E0100007F8FCF773F91AF0EBFFFFF747FE012052
:10E02000BDE8084012F0A0BA2DE9F04F013085B0EC
:10E03000C3B203930B4602918B4C8C4E002B00F025
:10E0400099808B4D8B4FDFF8309223F027FA4FF4F5
:10E05000FA7A4FF0100C4FF47A70D9F80430C3F309
:10E060000803002B40F0DE80EFF31183002B40F01B
:10E07000D9802968A26800BF2B689942F9D1D7F8E6
:10E0800000E000FB0EF39B1AB3FBFEF300FB013133
:10E090004FF0010E0191D9F80430C3F30803002BAF
:10E0A00040F08780EFF31183002B40F082802B68D3
:10E0B000A16800BF2A689342F9D1D7F800B000FBED
:10E0C0000BF2521AB2FBFBF200FB0323019A9B1ADC
:10E0D000B3F57A7FDFD3BAF1010ABED1039B002BDF
:10E0E00040F0BD804FF47A7ADFF88C9150464FF0C3
:10E0F000100CD9F80430C3F30803002B75D1EFF3EB
:10E100001183002B71D12968A26800BF2B68994246
:10E11000F9D1D7F800E000FB0EF39B1AB3FBFEF336
:10E1200000FB01314FF0010E0191D9F80430C3F327
:10E13000080313BBEFF31183FBB92B68A16800BF81
:10E140002A689342F9D1D7F800B000FB0BF2521ABB
:10E15000B2FBFBF200FB0323019A9B1AB3F57A7F13
:10E16000E3D3BAF1010AC4D1029B013B0293002B15
:10E170007FF467AF05B0BDE8F08FEFF311888CF343
:10E180001288A1682368DB0344BFC6F800E0A168D9
:10E190002B6832685FFA88F888F31188D7F8008016
:10E1A0001A4400FB08F35B1AB3FBF8F300FB0233DD
:10E1B000D2E7EFF311888CF31288A1682368DB03A0
:10E1C00044BFC6F800E0A1682B6832685FFA88F89F
:10E1D00088F31188D7F800801A4400FB08F35B1A13
:10E1E000B3FBF8F300FB023370E7EFF311828CF31B
:10E1F0001288D4F808E02368D90303D501233360DB
:10E20000D4F808E02B683168D2B282F311883A68FA
:10E21000194400FB02F3A3EB0E03B3FBF2F300FB84
:10E2200001317FE7EFF311828CF31288D4F808E014
:10E230002368D90303D501233360D4F808E02B68A1
:10E240003168D2B282F311883A68194400FB02F3B4
:10E25000A3EB0E03B3FBF2F300FB013118E7184602
:10E260002CF06EFA3EE700BF10E000E050B2002054
:10E2700054B2002058B2002000ED00E0204B5B6853
:10E28000C3F3080330B4BBB9EFF31183A3B91D4B3B
:10E290001D4C1868A16800BF1A689042F9D11B4B49
:10E2A0001C684FF47A7202FB04F3591AB1FBF4F1C3
:10E2B00030BC02FB00107047EFF31182102383F390
:10E2C000128811498C680B6813F4803F104B02D000
:10E2D000012018608C680B49D2B20D68186882F36F
:10E2E00011880A4B19684FF47A72284402FB01F333
:10E2F0001B1B30BCB3FBF1F302FB0030704700BFC7
:10E3000000ED00E054B2002010E000E058B2002020
:10E3100050B200202DE9F84F8046FFF7AFFF254EA1
:10E320002549DFF8A0E0254A254D844610274FF403
:10E330007A740120DEF80430C3F30803D3B9EFF395
:10E340001183BBB90B68D2F808A000BFD1F80090C8
:10E350004B45F7D1D6F800B004FB0BF9A9EB0A093D
:10E36000B9FBFBF904FB0393A3EB0C034345E1D397
:10E37000BDE8F88FEFF3118A87F31288D2F808B05E
:10E380001368DB0344BF2860D2F808B00B68D5F8E7
:10E3900000905FFA8AFA8AF31188D6F800A09944AF
:10E3A00004FB0AF3A3EB0B03B3FBFAF304FB0933FF
:10E3B000DAE700BF58B2002054B2002010E000E0BD
:10E3C00050B2002000ED00E02DE9F04FDFF830C141
:10E3D000474A4849484E494D8046102718F1FF38B2
:10E3E000C0F08480DCF80430C3F30803002B5CD158
:10E3F000EFF31183002B58D10B68946800BF0868B5
:10E400008342F9D1D6F800904FF47A7000FB09FEF0
:10E41000AEEB040EBEFBF9FE00FB03EEDCF80430AD
:10E42000C3F308034FF47A740120FBB9EFF31183AF
:10E43000E3B90B68D2F808A000BFD1F800904B45B3
:10E44000F7D1D6F800B004FB0BF9A9EB0A09B9FB28
:10E45000FBF904FB0393A3EB0E03B3F57A7FBDD264
:10E46000DCF80430C3F30803002BDFD0EFF3118A8C
:10E4700087F31288D2F808B01368DB0344BF286022
:10E48000D2F808B00B68D5F800905FFA8AFA8AF3E0
:10E490001188D6F800A0994404FB0AF3A3EB0B0300
:10E4A000B3FBFAF304FB0933D5E7EFF3118487F3E9
:10E4B0001288D2F808901368D80303D501232B6083
:10E4C000D2F808900B682868E4B284F31188D6F873
:10E4D00000A04FF47A7400EB030E04FB0AF3A3EBE5
:10E4E0000903B3FBFAF304FB0E3E97E7BDE8F08F98
:10E4F00010E000E054B2002058B2002050B20020DA
:10E5000000ED00E030B4EFF31183102282F31288A3
:10E510000649074C0A680748013200250A60256051
:10E52000DBB2026883F3118830BC704754B200201C
:10E5300050B2002010E000E00F4B1B88014643B9A9
:10E540000E4B0F4A1B7810680BB981F00101FBF7E5
:10E55000A9BA0C4B5A691AB118B91A6810605874E4
:10E560007047094A18681188084A92FBF1F20121A4
:10E5700002605974704700BF2CB200202EB20020F8
:10E5800030B2002034B200204CB2002020A107009D
:10E5900038B5254B5C69236B73B1636D626BCAB18F
:10E5A000998A1A88C90592B201D5D20700D438BD1C
:10E5B0004FF6F7721A8038BD636D99891A888906FB
:10E5C00092B2EBD59206E9D5E26ACAB1988880B2D8
:10E5D0009047E2E799891A880D0692B2E0D51006B5
:10E5E000DED5A26A616A8A4219D0A1692569885C70
:10E5F00098800132B2FBF5F105FB1122A262CFE750
:10E600009B88E2696169DBB28B54E269E068636D03
:10E610000132B2FBF0F100FB1122E261BEE7DA68E1
:10E6200022F08002DA60BBE7D83B002038B5254BEA
:10E63000DC68236B73B1636D626BCAB1998A1A8807
:10E64000C90592B201D5D20700D438BD4FF6F77292
:10E650001A8038BD636D99891A88890692B2EBD504
:10E660009206E9D5E26ACAB1988880B29047E2E79B
:10E6700099891A880D0692B2E0D51006DED5A26AF5
:10E68000616A8A4219D0A1692569885C9880013243
:10E69000B2FBF5F105FB1122A262CFE79B88E2698C
:10E6A0006169DBB28B54E269E068636D0132B2FBF1
:10E6B000F0F100FB1122E261BEE7DA6822F080028D
:10E6C000DA60BBE7D83B00202DE9F04F2DED028B3F
:10E6D00095B0804621F010FC8E4B1D7825B115B009
:10E6E000BDEC028BBDE8F08F8B4B1B685905F6D54E
:10E6F0008A4BDFF880B21B686BB1894ADBF80010E7
:10E700001368CB1A7C2B06D9864811600378013335
:10E71000037026F0D7FC844B1B78002B6DD0834C04
:10E72000834AD4F81031A8EB0303934201F2278304
:10E7300094F81891B9F1000F32D17E4F3868FAF78A
:10E74000ABFDC0B201280FD902287B4E42F01380E6
:10E750003378002B42F00881D4F81C31A8EB030376
:10E76000B3F57A6F82F0CE82D4F82031002B44D0FA
:10E7700094F81831BBB9714B1B689B7801211E3B83
:10E7800000228B4284F8181184F82C2142F26C820A
:10E7900038680221043026F047FC94F8243110E058
:10E7A000D4F820314BB3D4F8283140F6B732A8EB77
:10E7B0000303934221D994F82431002B01F0D98628
:10E7C0005C4F013BDBB284F82431002B01F00A845A
:10E7D000D4F8206194F82C2116F8011B94F82D31FF
:10E7E0003868C4F820610A44013384F82C2184F885
:10E7F0002D31FAF755FDC4F82881514BDBF8006044
:10E800001B7843B14F4F386828B14F4B1B78013B01
:10E81000012B41F2F6834D4B1B786BB14C4F3B689B
:10E8200053B1DBF80030414C03931A46D4F844311D
:10E83000D31A632B01F29381464F3B78022B01F0F0
:10E8400078863D4E96F87430032B01F0B683424B28
:10E850001B7873B1414D2B685BB1344CFFF70EFD53
:10E86000D4F85031039044F61F62C31A934200F269
:10E8700031813B4B1B78002B7ED13A4B1B7843B147
:10E880002A4CD4F8A03203F5C333A033984581F065
:10E890003782354B1B78002B3FF421AF234E334C8E
:10E8A000334D06F2C1272068FAF7F6FC00283FF442
:10E8B00016AF2068FAF7E8FC2B7880465A1E33B171
:10E8C00020682A70FAF7E8FC0028F2D107E7032253
:10E8D0003946781E2FF0BEFC96F8C03296F8C12259
:10E8E00086F8C38283F47F4383F0FF039B1A1FFAE9
:10E8F00088F89BB2B8EB132FD5D196F8C222DBB2C1
:10E900009A42D0D1781E21F0B7F92B78184428709C
:10E91000C9E700BFE6460020785B00208472002033
:10E92000A8740020A4740020AA630020D81E002030
:10E930003F0D030050740020280000205474002074
:10E94000AC63002088720020B4630020BC63002008
:10E9500048740020A2760020C4630020C863002011
:10E960003464002045640020CE630020D46300207E
:10E97000D863002054B20020484C2278A2B1484B02
:10E980009B7A53B1FFF77AFC464B1B68C31AA3F579
:10E990007A73B3F5FA6F07D82278434B4349186866
:10E9A000FAF746FC00232370414CD4F8983203F563
:10E9B000C333A0339845FFF460AF3E4DC4F898824E
:10E9C0002B78002B41F010873B4D2B78002B41F02A
:10E9D0006B8694F89C2239498D5CEA0702F1078026
:10E9E000AF0701F1C787680701F188872A0748D573
:10E9F000334B344E0D9314AA1146A3F13D0241F856
:10EA0000202D0020A3F140020D4603F8400C059193
:10EA1000022311215170937028463168FBF794FE50
:10EA200028467168FBF790FEF389274903EBC3037F
:10EA30009B00053381FB0321DB17C3EBA1012846B3
:10EA400089B2FBF799FE338A03EB8303590089B23D
:10EA50002846FBF791FE1D4B059D1B789B0743BF86
:10EA6000318901F57A7189B24FF47A712846FBF742
:10EA700083FE0C9B327D591C0C9128461A7021F0A4
:10EA8000CFF9134A94F89C321178013393FBF1F2D9
:10EA900001FB123384F89C32EFE600BF9C63002038
:10EAA000F85C0020C0560020386400205C63002021
:10EAB000D81E00203C6400203D64002040640020FB
:10EAC0005C630020D474002067666666D074002002
:10EAD0004464002094F85631002B41F0CB85D34B91
:10EAE0001A6802F00803002B48F603414AF60B406F
:10EAF0004BF60F4349F6074604BF03460E4612F095
:10EB0000040F4FF0190118BF1E46970684F85611DE
:10EB100003D546F4804646F02006C54B5F79C6F320
:10EB20000909002F42F013819B79002B42F01E82CD
:10EB30001F4664204FF0FF3A4FF0000E0C960D96E2
:10EB4000ADF83E70ADF83CE0CDF842E0CDF846E0DF
:10EB5000CDF84AE0CDF83890ADF840A08DF84E00E1
:10EB60000CAE0FCEB34F84F805E00FC796E80F0048
:10EB700007C727F8023B39464FF0010E1B0CFE2653
:10EB80001F20C82201F81E39A670A27184F807E080
:10EB9000E07094F86601207180F0F10383EA0313BA
:10EBA000DAB2130983F0E70343EA022383EAC203DC
:10EBB0001BB283EA0312D2B2C3F3072383EA121310
:10EBC00043EA022383EAC2031BB283F0C80282EA4B
:10EBD0000212D2B2C3F3072383EA121343EA0223D9
:10EBE00083EAC2031BB283EA0E0686EA0616F6B271
:10EBF000C3F3072282EA161242EA062200EB0E0352
:10EC000082EAC60607EB0E0084F86631268011F80A
:10EC1000013B734083EA0313DBB21A0982EA16222E
:10EC200042EA032282EAC3031BB29EB281422680DB
:10EC3000EDD183F07C0383EA0313DBB24FEA131EAA
:10EC40008EEA162E8EEA032E8EEAC30E0FFA8EFE81
:10EC50001FFA8EFC784FA4F800C05FFA8EFE4FEAD0
:10EC60001C2C84F828C084F827E007F5C77904F144
:10EC7000220A38687968BA68FB684E460FC61037B2
:10EC80005745B146F5D1386830606C4E3B7989F80C
:10EC9000043006F1270784F8B5E184F8B6C116F808
:10ECA000011F2868FAF7FCFAB742F8D194F85731F7
:10ECB000002B41F0E4846249DBF8002009780A2047
:10ECC00084F85701002901F000865E4E0129308842
:10ECD000079042F2518170880690022902F04F801D
:10ECE000B0880590032902F05E81F0880490042921
:10ECF00002F054810529308902F04C810629B6F8CA
:10ED00000A9002F044810729B6F80CC000D0F389BC
:10ED100094F866110C920F4687F0300282EA0212D4
:10ED2000D2B216094849089786F07A0646EA0226C2
:10ED30000988277186EAC202444EC1EB012186FB95
:10ED4000017A079E4FF0000E66F30F0E069E12B278
:10ED500066F31F4E8A44059ECDF834E0C917C1EB17
:10ED60006A2A002782EA0211C9B266F30F07C2F3CA
:10ED70000722002682EA111260F30F060020079294
:10ED80006CF30F00049A8DF845A063F31F40079BB6
:10ED9000109062F31F4769F31F464FF000090E976A
:10EDA0000F968DF8449043EA01220DF1300E82EA6D
:10EDB000C106BEE80F0036B286F0C80C8CEA0C1C07
:10EDC0001C4F84F805905FFA8CFCC6F307260FC72A
:10EDD00086EA1C1646EA0C239EE8030083EACC036D
:10EDE0001BB283F0230247F8040B82EA0212D2B26C
:10EDF000C3F30723089E83EA1213384643EA02232B
:10EE000083EAC20206F1010E20F814194FF0230C18
:10EE10001621FE26C82384F866E102372280E170BD
:10EE200084F807C0A670A371114611E0CC740020CD
:10EE3000B8740020E01E0020DA1E002067200020A9
:10EE40006C47002004A60020645E00200308208098
:10EE500010F8013B4B4083EA0313DBB21A0982EA44
:10EE6000112242EA032282EAC3031BB299B2B842DA
:10EE70002180EDD183F0F40383EA0313DBB24FEA80
:10EE8000131E8EEA112E8EEA032E8EEAC30E0FFA9F
:10EE90008EFE1FFA8EF7C84E27804FEA172C5FFAB6
:10EEA0008EFE84F81EE084F81FC07168B268306876
:10EEB000F36806F5C7770FC730697169B26904F264
:10EEC0008F1607C704F2AD1784F8ADC184F8ACE122
:10EED00016F8011F2868FAF7E3F9B742F8D194F859
:10EEE0005A31002B41F0DB83B44B06931B68192287
:10EEF000980684F85A2140F1EA82B14BB14E1B7852
:10EF0000990741F12187337D042B8CBF032702270A
:10EF1000FFF7B4F9338A32890C9003EB83035B006B
:10EF2000ADF84A304FF47A7033688DF84C700E9318
:10EF3000F18996F814E073688DF84DE000FB02F259
:10EF40004FF0000C0CAF4FF0FF30CDF834C01092F2
:10EF50000F93ADF848101190BE46BEE80F0005971C
:10EF6000994F0FC79EE80F0007C73A46182122F8AD
:10EF70001C39E17194F8661184F805C081F07803BA
:10EF800083EA0313D8B2030983F0F60343EA0023AC
:10EF900083EAC0031BB283EA0310C0B2C3F30723A2
:10EFA00083EA101343EA002383EAC0031BB283F011
:10EFB000C80080EA001E5FFA8EFEC3F3072080EAD5
:10EFC0001E1040EA0E2080EACE0000B280F0180346
:10EFD00083EA0313DBB2C0F3072080EA131040EA90
:10EFE000032080EAC30301F1010EFE204FF01E0C46
:10EFF0004FF0C809A0700237217184F866E12380C0
:10F0000084F803C084F80690184612F8011B4140AA
:10F0100081EA0111C9B20B0983EA102343EA0123F3
:10F0200083EAC10109B288B2BA422080EDD181F0F1
:10F03000180181EA0111C9B20A0982EA102383EAA0
:10F04000012383EAC1031BB29AB25B490491DBB28C
:10F050004FEA122C2280079384F827C084F82630C8
:10F060000F4601F5C77A04F1220938687968BA6851
:10F07000FB68D646AEE80F0010374F45F246F4D194
:10F080003868CEF80000DFF84C919DF81C3084F809
:10F09000B43109F1260784F8B5C1CA461AF8011F30
:10F0A0002868FAF7FDF85745F8D1FFF7E7F8069B0F
:10F0B00071681B683289069113F0140F4FF47A714E
:10F0C000D6F800E001FB02F141F00B860E4694F801
:10F0D00066A10C908AF06A003C4B3D4FB3F90420C6
:10F0E000CDF834E080EA0010C0B2030983F0D50304
:10F0F00043EA002383EAC0031BB283EA0310C0B2D1
:10F10000C3F3072383EA101343EA002383EAC0030F
:10F110001BB287FB0207D2174FF0000CC2EBA7020D
:10F120000698DDF814E0109683F0C8070E900F9152
:10F13000ADF84A20ADF844C0ADF846C0ADF848C0BF
:10F1400087EA0717FFB2C3F30726BEE80F0086EA77
:10F15000171646EA072686EAC7071B4E84F804A05E
:10F160003FB20FC687F021039EE8070083EA03132E
:10F17000DBB2C7F3072787EA13170AF1010E47EA44
:10F18000032786E8070087EAC30384F866E14FF0A7
:10F19000210A4FF0FE0E1C27C8220C3684F805C049
:10F1A00084F807A084F802E0A6F11C01E770184675
:10F1B000A271238010E000BFDA1E0020CC74002072
:10F1C000D0740020D4740020E01E0020B074002011
:10F1D000676666666720002011F8012B424082EACC
:10F1E0000212D2B2130983EA102343EA022383EA0C
:10F1F000C20212B290B2B1422080EDD182F0680218
:10F2000082EA0212D2B24FEA121A8AEA102383EA81
:10F21000022A8AEAC20A0FFA8AFA1FFA8AF3D74E3A
:10F2200023804FEA132C5FFA8AFA04F1220384F850
:10F2300025C084F824A006F5C77E0693F3683068DD
:10F240007168B26877460FC7069B10369E42BE466D
:10F25000F4D13388CA4E3B804F4684F8B2A184F87B
:10F26000B3C117F8011F2868FAF71AF8BE42F8D19F
:10F2700094F866E1C34AC44E84F804E08EF0EB03D0
:10F2800083EA0313D9B20B0983F0C50343EA0123D0
:10F2900083EAC1031BB283EA0310C0B2C3F30721A0
:10F2A00081EA101141EA002181EAC0010CCA09B2C9
:10F2B00081F0C80787EA0717FFB24FF0000C0C92E5
:10F2C000C1F30721059A0D93CDF838C081EA1713D1
:10F2D00043EA072307CA83EAC7031BB283F0310757
:10F2E00086E8070087EA0717FFB2C3F3072383EA1C
:10F2F000171343EA072383EAC703277A607AA17AC0
:10F30000E27A267B84F805C01BB25F4087EA0717C4
:10F31000FFB2C3F3072383EA171343EA072383EA01
:10F32000C7031BB2584080EA0010C0B2C3F30723E2
:10F3300083EA101343EA002383EAC0031BB2594057
:10F3400081EA0110C0B2C3F3072181EA101141EA3A
:10F35000002181EAC00109B24A4082EA0212D2B217
:10F36000C1F3072383EA121343EA022383EAC203A9
:10F370001BB25E4086EA0616F6B2C3F3072383EAA1
:10F38000161343EA0623607BA17BE27B277C94F87B
:10F3900011C083EAC6031BB2584080EA0010C0B215
:10F3A000C3F3072383EA101343EA002383EAC0036D
:10F3B0001BB2594081EA0111C9B2C3F3072383EAA2
:10F3C000111343EA012383EAC1031BB25A4082EAC4
:10F3D0000212D2B2C3F3072383EA121343EA0223D1
:10F3E00083EAC2031BB25F4087EA0717FFB2C3F389
:10F3F000072383EA171343EA072383EAC7031BB2F1
:10F400008CEA030C8CEA0C1C5FFA8CFCC3F3072318
:10F4100083EA1C1343EA0C2383EACC03A17CE27C3D
:10F420005A4F1BB2594081EA0111C9B2C3F30723F5
:10F4300083EA111343EA012383EAC1031BB25A4052
:10F4400082EA0212D2B2C3F3072383EA121343EA19
:10F45000022383EAC2031BB283F0270686EA061260
:10F46000D2B2C3F3072686EA121646EA022686EAD5
:10F47000C20636B20EF10103B2B231204FF0FE0CDB
:10F480000C2184F86631C8234FEA122E5FFA86FAFF
:10F490002280E07184F802C0E170A371049E84F8B8
:10F4A00014A084F815E07168B268F3683068B6F8A3
:10F4B00010C00FC727F803CB84F8A3E184F8A2A1FA
:10F4C00019F8011F2868F9F7EBFE4F45F8D194F8B9
:10F4D0005E71002F41F0DE802D4B94F866E1B3F9A8
:10F4E0000010B3F90220B3F904309FED2A6A677166
:10F4F00007EE103ADBF800300C938EF06A0383EAD3
:10F50000031306EE901AD9B20B0983F0D50343EA30
:10F51000012383EAC1031BB283EA03115242C9B239
:10F5200007EE902AC3F3072383EA111343EA01236A
:10F53000F8EEE77AF8EEE66AB8EEC77A83EAC10336
:10F540001BB267EE867A66EE866A27EE067A0020A0
:10F5500083F0C80CCDED0E7ACDED0D6A8DED0F7AEE
:10F560001090119012908CEA0C160DF13009F6B241
:10F57000C3F3072CB9E80F000EE000BFDA1E00202D
:10F580008B200020AC640020E01E002068200020BA
:10F59000B074002088C3E43A8CEA161C4CEA062CAE
:10F5A0008CEAC60CD04E0FFA8CFC0FC68CF01E07EE
:10F5B00099E8070087EA0717FFB2CCF3072383EA2D
:10F5C000171343EA072386E8070083EAC707C82121
:10F5D0004FF005094FF01E0CFE231C200EF1010216
:10F5E000A17184F85E9184F807C0A370E070A6F161
:10F5F000100184F804E00C36278084F8662111F8A5
:10F60000013B7B4083EA0313DBB21A0982EA17222B
:10F6100042EA032282EAC3031BB29FB2B1422780AF
:10F62000EDD183F0270383EA0313DBB24FEA131E05
:10F630008EEA172E8EEA032E8EEAC30E0FFA8EFE86
:10F640001FFA8EFCA94FA4F800C05FFA8EFE4FEAA5
:10F650001C2C84F825C084F824E007F5C77904F150
:10F66000220A38687968BA68FB684E460FC61037B8
:10F670005745B146F5D19E4E3B88A9F8003006F1BA
:10F68000240784F8B2E184F8B3C116F8011F286892
:10F69000F9F706FEB742F8D194F85F91B9F1000F7F
:10F6A00040F0F287934B1B68052284F85F219A068D
:10F6B00041F11581904ADFED917AD18907EE101A58
:10F6C000B8EEC77A13F0140F27EE277A01F0718392
:10F6D0008B4BDFED8A6AD3ED007AF8EEE77A67EEBE
:10F6E000A67A94F866C1874B874AB3F90410B2F939
:10F6F0000620864E86488DED0D7A8CF0220383EA33
:10F700000313DFB23B0983F0590343EA072383EA7B
:10F71000C703B2F5FA6F1BB2A8BF4FF4FA6283EACF
:10F720000317FFB2B2F57A7FC3F3072383EA1713F7
:10F73000B8BF4FF47A724FF0640E43EA0723A2F584
:10F740007A720EFB02F283EAC70786FB02E680FBB1
:10F7500001E03FB2C917D217C2EBA612C1EBA0035A
:10F760004FF0000A0CA987F0C806CDED0E7AADF86F
:10F770004220ADF84030CDF830A0CDF83CA08E4608
:10F7800086EA0616F6B20591C7F30727BEE80F0012
:10F7900087EA161747EA062787EAC606524FDEF8B9
:10F7A00000E084F804C00FC736B286F04A0383EA4B
:10F7B0000313DBB2C6F3072181EA13113A4641EA8B
:10F7C00003210CF1010C81EAC303142042F810E973
:10F7D000FE264FF04A0E002184F866C14FF0C80C97
:10F7E000E0702380043784F807E0A670617184F824
:10F7F00006C0184612F8011B414081EA0111C9B246
:10F800000B0983EA102343EA012383EAC10109B209
:10F8100088B2BA422080EDD181F0140181EA011151
:10F82000C9B24FEA111E8EEA102E8EEA012E8EEA20
:10F83000C10E2E4B0FFA8EFE1FFA8EF61F464FEAB0
:10F84000162C5FFA8EFE84F81CE084F81DC0386820
:10F8500059689A68DB68B7F818A0049726803E4676
:10F8600007F5C7770FC73069716903C704F28F16B0
:10F87000A7F800A0374684F8ABC184F8AAE104F2E7
:10F88000AB1A17F8011F2868F9F70AFDBA45F8D135
:10F89000204B214A1B781278013B12F00100DBB2A9
:10F8A00014BFC0214021172B03D81C4A134493F8DE
:10F8B00030901B4B1A8897071ABF002341F01001A4
:10F8C000012312F4027F18BF022312F0100F18BF99
:10F8D000062312F0200F18BF1023002841F00882E1
:10F8E0004FF0030C1EE000BFE01E0020DA1E0020D7
:10F8F00067200020CC740020D47400200AD7233C59
:10F90000AC740020B074002004A60020D34D621017
:10F9100067666666A4600020606200202CE503082C
:10F92000CC64002094F866E10C938EF0460383EAE1
:10F930000313DAB2130983F0920343EA022383EA42
:10F94000C2031BB283EA0310C0B2C3F3072282EAE8
:10F95000101242EA002282EAC00212B282F0C80704
:10F9600087EA0717FFB2C2F3072282EA17120023C1
:10F970008DF837C0032042EA072C059A8DF83490A1
:10F980008DF835308DF836108DF8380007CA8CEABE
:10F99000C70C0FFA8CFCD04FE3718CEA0C1903C72B
:10F9A0005FFA89F9CCF3072C8CEA191C4CEA09217F
:10F9B00081EAC90994F808C03A700FFA89F98CEA0B
:10F9C000090C8CEA0C1C5FFA8CFCC9F3072282EA52
:10F9D0001C1242EA0C22607AA17A94F80B906371AF
:10F9E00082EACC0212B2504080EA001C5FFA8CFC22
:10F9F000C2F3072080EA1C1040EA0C2080EACC0009
:10FA000000B2414081EA0111C9B2C0F3072282EA83
:10FA1000111242EA012282EAC10212B289EA020903
:10FA200089EA09195FFA89F9C2F3072282EA1912F1
:10FA300042EA092294F80CC0607BA17B84F804E0C0
:10FA400082EAC90212B28CEA020C8CEA0C1C5FFA40
:10FA50008CFCC2F3072282EA1C1242EA0C2282EAE0
:10FA6000CC0212B2504080EA0010C0B2C2F30722AA
:10FA700082EA101242EA002282EAC00212B2514027
:10FA800081EA0111C9B2C2F3072282EA111242EAE5
:10FA9000012282EAC102E17B94F8109013B281EA5C
:10FAA000030282EA0212D2B2C3F3072383EA1213DB
:10FAB00043EA022383EAC2031BB289EA030282EA11
:10FAC0000212D2B2C3F3072383EA121343EA0223DA
:10FAD00083EAC2031BB283F0320282EA0212D2B27C
:10FAE000C3F3072383EA121343EA022383EAC20320
:10FAF0001BB29AB24FF0FE0C5FFA83FB0920C821BB
:10FB00000EF1010E84F802C04FEA122CE070A171D0
:10FB100084F866E1228084F812C084F811B0049B56
:10FB2000186859689A68B3F80CA007F5C07EAEE86B
:10FB3000070007F5C8778EF80290AEF800A084F8A9
:10FB4000A0C184F89FB116F8011F2868F9F7A8FB37
:10FB5000B742F8D1039BC4F85031FEF78ABEDFF8F4
:10FB600098A15E4EDFF89491412025F009FABAF988
:10FB7000023086FB0320DB17C3EBA00080B225F028
:10FB8000E3F9BAF9003086FB0320DB17C3EBA000D2
:10FB900080B225F0D9F9BAF9043086FB0320DB17CF
:10FBA000C3EBA00080B225F0CFF999F800103868B7
:10FBB000F9F776FB94F848A11AF0010600F0F784F3
:10FBC000474B06931B689A0673D5464B464E1B78E7
:10FBD0009B0741F15180337D042B8CBF4FF0030A0A
:10FBE0004FF0020A472025F0CBF9306825F078F96C
:10FBF000706825F075F93D4AF3893868A2FB032344
:10FC0000C3F3471319460493F9F74AFB069B99F887
:10FC100000101A68049B12F0140F83EA010389F89C
:10FC2000003040F067863389642000FB03F025F044
:10FC300057F9367D38684AEA8606F6B23146F9F752
:10FC40002FFB99F8003038685E40314689F8006033
:10FC5000F9F726FB94F848A1BAF1000F29D1244EF8
:10FC60004F2025F08DF9306825F03AF9706825F0BD
:10FC700037F9504625F034F901213868F9F710FBBF
:10FC8000184A99F800301678386806F001063146AF
:10FC900083F0010389F80030F9F702FB99F800308E
:10FCA00038685E40314689F80060F9F7F9FA94F84F
:10FCB00048A1039B0F4AC4F844310AF10103DBB2A7
:10FCC000A2FB0312D20802EB8202A3EB420384F8E8
:10FCD0004831FEF7B1BD00BFE01E002067666666D2
:10FCE000CC740020D0740020D47400201F85EB5108
:10FCF000AC640020CDCCCCCCB07400204C7400207F
:10FD000094F8A432C24AC4F8A08202EB8302926C37
:10FD100042B314AD04F2AB23BE4E45F8203D0021A2
:10FD200004F2BD2331800D9380211523A52784F88B
:10FD3000AA32284684F8A91284F8A8729047284667
:10FD40003188FAF73FFD0C9DB34804F52A716D1A0E
:10FD5000152DA8BF15252A462EF071FAAF4A94F842
:10FD6000A4321570AE4A013382FB0312A2EBE37298
:10FD700002EB42029B1A84F8A432FEF78ABDA94A1C
:10FD8000A94BD4F81411DBF800001B88D77AA74AD6
:10FD9000401A4FF47A71DEB201FB07F11B0A967725
:10FDA000167588424FF00006D3775375967016711A
:10FDB00080F0D1849E4E9F4BD6F800C01B689E4EAB
:10FDC0009E48DFF8989201688068DFF894E286FB2D
:10FDD0000376DB17C3EB661303F5FA739BB29376D6
:10FDE0001B0AD37689FB0173C917C1EBA30189FBF9
:10FDF00000791177C0170912C0EBA90051778E491D
:10FE000082F820000CF5EA43001281FB0C713033BC
:10FE100082F821004FEAEC701B12C0EB6110884E93
:10FE20009EF800E082F823307830864B82F8240078
:10FE30000CF13001307D03901EF0020F82F8221089
:10FE4000987600F08584D6F800E07F4AD6F804A0C2
:10FE50007E48DFF810C282FB0E194FEAEE7182FB7A
:10FE60000A72C1EBA9514FEAEA79C9EBA25200FB31
:10FE700001E900FB02A009EB490900EB40004FEA51
:10FE800049094000049207468CFB09208014059024
:10FE90008CFB072CF089049A3689079702EB8202C3
:10FEA00006F5FA7600EBC00002EB8202B6B20496C9
:10FEB0000892059E8200099201EB81014FEAE972E6
:10FEC000B01A01EB8101624E06910246039906FBCE
:10FED0001292069E40B2052900EB86004FEAE771B8
:10FEE0004FEAAC4C5A4E0590ACEB0100014606FBC4
:10FEF0001070089E504FDFF870C14FEADA7A49B2AD
:10FF000001EB86014FEADE7E87FB006983F80EA0D5
:10FF100087FB026A099F83F809E0DFF850E13E465B
:10FF20008EFB066EBCF8006003969DF810605E754F
:10FF3000049EBDF814C083F80AC04FEA162689B2A1
:10FF400004964FEAE2724FEAE777424ED973C2EB6A
:10FF50006A12C7EBAE174FEA1C2A4FEA112E4FEA7E
:10FF6000E0700399368883F80BA0C0EB691083F822
:10FF700010E04FEA22291A739DF810209A754FEA73
:10FF8000202CC7F3072A4FEA112134BF4FF0320E5D
:10FF90004FF0330E9DF80C2083F80D90587483F8C1
:10FFA00012C0DF7183F808A0DA74197583F81BE0BA
:10FFB0001E77C4F81081FEF7BBBBDFF8B490D9F808
:10FFC0000000F9F759F900283EF441ACD9F80000D7
:10FFD0000121F9F74DF90222002386F874203B70C5
:10FFE000FEF735BC94F82C1194F82D3138684A1C72
:10FFF000013384F82C2184F82D31F9F751F9FEF7FB
:020000040801F1
:10000000FABB154CDFF86C904FF0000A3FE000BFE0
:100010002CE5030818630020C8510020DD510020A2
:1000200056555555DC620020D4620020DC63002068
:10003000A0740020AC7400201F85EB51907200204A
:10004000D4740020086400206BCA5F6B806967FF6E
:1000500040420F00B6640020D81E00206766666626
:10006000D074002083DE1B43B4640020D34D6210A3
:1000700028770020280000201B2B00F06F820D2B1A
:1000800000F04B814FF0010389F801303868F9F72F
:1000900003F9002839D03868F9F7F6F883B27E2BD7
:1000A000DBF800202AD099F801100029EED194F84D
:1000B0002E21002AE0D07D2B00F0368294F83CE11E
:1000C000BEF1000F04D080F02003DBB284F83C11B5
:1000D000511CC9B22244092984F82E1182F830310A
:1000E00000F016820829D1D8B4F83A21134403EB62
:1000F000132303F0FF03A4F83A31C7E784F82EA1D5
:1001000084F82FA189F801A0C0E794F83D3133B1FC
:1001100094F8313184F83D01302B00F0C18594F81A
:100120002F21C54BC549DFF850A3DFF850E39146B6
:100130004A46002A3EF46FABDBF80020921B012AEE
:1001400024D894F83E21002A40F01E8294F83FC142
:1001500033F81C00F8B94FF0010284F83F210A6817
:100160009706E5D59AF800209007E1D5B44EB54939
:10017000F2894FF4F36303FB02F381FB0321DB17E6
:10018000C3EB61114FF4036024F034FF002384F8C3
:100190002F31FEF740BB0CF1010C5FFA8CFCB0F57F
:1001A000E06F84F83FC100F098801BD8B0F5047F61
:1001B00000F0238135D8B0F5887F00F0CD80B0F510
:1001C000007F00F0B380B0F5807FB1D10A6852079C
:1001D000AED59D4B196824F00DFF002384F82F3114
:1001E000FEF719BBB0F5026F00F05A816AD8B0F57E
:1001F000E46F00F08180B0F5006F00F0D680B0F5BC
:10020000E26F95D1914BDA6B998A642303FB02F379
:1002100093FBF1F124F0EEFE002384F82F31FEF77A
:10022000FABAB0F5826F00F05181B0F5C06F00F0FE
:100230002781B0F5806F7FF47BAF94F840310133B4
:10024000DBB2032B00F2AD8142F2107184F8403131
:1002500001FB03F17E4B1B88002B40F0A081013194
:100260007C4B1B78DB077C4B1B8848BF0431DF07C6
:1002700048BF0A31980748BF14311A0648BF2831D1
:10028000DF0548BF2831580748BF64311A0748BF07
:10029000C8319F0548BF01F5C871980648BF01F5F0
:1002A0007A71DA0648BF01F5FA615F0648BF01F5C9
:1002B0007A614FF4806024F09DFE002384F82F3192
:1002C000FEF7A9BAB0F5046F1AD0B0F5116F52D08D
:1002D000B0F5036F7FF42CAF41E75C4B91469A6B0E
:1002E000998A642303FB02F393FBF1F124F082FE6D
:1002F00084F82F91FEF78FBA544B91461A6CEFE7B2
:10030000564BB3F9041001EB81019146490024F0EA
:1003100071FE84F82F91FEF77EBA4FF0010184F848
:100320002E1184F83031A4F83A21AFE69EF8062069
:10033000002A3FF4FDAE4A4B4A491B6881FB03216A
:10034000DB17C3EBA1014FF4007024F053FE002330
:1003500084F82F31FEF75FBA0A6852077FF5E8AEDE
:10036000414B4FF48870196824F044FE002384F850
:100370002F31FEF750BA9EF80520002A3FF4D8AE80
:100380003A4A107800283FF4D3AE394B1B8803EB70
:100390008303590091FBF0F14FF4116024F02AFE21
:1003A000002384F82F31FEF736BA0A6897067FF5E6
:1003B000BFAE9AF8002090077FF5BAAE1CF0010F8F
:1003C0001F4E204900F05C84726882EAE273A3EB5E
:1003D000E27303EB5303A1FB0331C908002AACBF4E
:1003E00041F0004141F040414FF4006024F002FE32
:1003F000002384F82F31FEF70EBA9EF80520002A5C
:100400003FF496AE194A107800283FF491AE194B8C
:100410005B7B002B00F09484154B1B8893FBF0F062
:1004200000EB800041004FF4047024F0E3FD002352
:1004300084F82F31FEF7EFB92CE50308CC740020C7
:10044000D47400201F85EB51AC7400205874002038
:100450002275002060620020CC640020B07400206F
:100460009072002067666666A0740020EA62002031
:10047000D4620020DC620020D0740020B874002018
:100480009EF80620002A3FF453AEC34B4FF4C060E1
:10049000996824F0AFFD002384F82F31FEF7BBB933
:1004A0000F68BF067FF544AE9AF800C01CF0020F3B
:1004B0003FF43EAEB94E33896421914601FB03F10E
:1004C00024F098FD84F82F91FEF7A5B90A689006EC
:1004D00040F1F180B24BB14E1878317D00F002034B
:1004E000002B0CBF00234FF47A7340F6B83208BFDC
:1004F0004FF4FA6210F0010F18BF134619444FF47D
:10050000826024F077FD002384F82F31FEF783B951
:10051000B4F83A21C2F1FF0293427FF4B3AD4FF039
:10052000010384F83D31ADE54FF0010384F83C311F
:10053000ACE5FDF7A3FE9B4B1B68C01A40F6B83331
:10054000984200F21E81DFF89CA29AF804303A2B00
:1005500000F0BA8200233B70FEF779B93868F8F7EB
:100560009BFE00287FF48EAD4FF0010384F82F31FD
:100570008CE5C4F8203184F818318B4F24F088FDC5
:1005800094F82431FEF71DB98849062024F01CFB9D
:10059000002384F83E0184F82F31FEF73CB9023184
:1005A0005EE6012384F8403142F2107152E6804B3E
:1005B0001B88D80513D4D90600F17A839A0600F176
:1005C000F183580600F1F383190700F1F983DA0784
:1005D00000F1148413F0020F0CBF04260C26754B97
:1005E000754A1B78D27803F001030AB143F0020385
:1005F0005320049324F0C4FC704A128802EB820258
:1006000002EB8202900080B224F09EFC002024F0D5
:100610009BFC6B4A6B4912883868C2EBC2125200CD
:1006200081FB023111444FEAE27ACAEB612A5FFA98
:100630008AFA5146F8F734FE99F80020049B38688E
:100640001E438AEA020A002189F800A0F8F728FE72
:1006500031463868F8F724FE99F80030386873405E
:10066000DBB2194689F80030F8F71AFE94F848A171
:10067000FFF7F2BA013B84F85631FEF717BB013B96
:1006800084F85731FEF72BBC09F1FF3984F85F91EC
:10069000FFF760BA013F84F85E71FEF7FDBF013BD2
:1006A00084F85A31FEF713BF47493A2024F08CFAF8
:1006B0002870FEF7E2B8454A1268120600F1FA8285
:1006C000434A127B002A3FF433AD94F841110329C9
:1006D00000F28A83DFE801F0322819023D4B1B68E3
:1006E00059799A79DB7901F1407101EB022101EB33
:1006F0000341002384F841314FF4826024F07AFCF6
:10070000002384F82F31FEF786B8334B1A68137A2A
:10071000507992781B0403EB002313444A1C84F89D
:10072000412103EB0161E7E72B4B1A68D37910797C
:1007300052781B0403EB00231344EFE7264B1A689F
:100740009379D07812781B0403EB00231344E5E778
:100750002D22DA762DE4214BDBF800101B78C4F84B
:100760001411013B012B3FF625AB102102239170A0
:100770001371FFF71FBB24F07BFC01233370FDF7DF
:10078000F3BF174AB2F84A3100210133A2F84A31C7
:100790003970FEF75CB800BF90720020D47400205E
:1007A000D0740020A876002050740020ED4F03087C
:1007B000CC6400206062002044470020D462002006
:1007C000645E00200308208081FE0208785B002020
:1007D000DC6200202C440020F84600202444002045
:1007E000D81E002090760020A64EA74B0093002430
:1007F000A6F13F01A54BA64A0A9106F8404CA5492F
:100800000B960CA8FAF7B6F80A9E731C0A9334707C
:100810000A9B2922591C0A911A700A9BEA22591C28
:100820000A911A700A9BC822591C0A910CA81A70C6
:100830002AF004FD471C0CA93A460A982DF0FFFC4B
:100840000A9AD31901330A93D4550A9B5A1C0A9267
:100850001C700A9B5A1C0A921C700A9B5A1C0A9212
:100860001C700A9B5A1C0A921C700A9B5A1C0A9202
:100870001C700A9B5A1C0A921C700A9B5A1C0A92F2
:100880001C700A9B5A1C0A921C700A9B5A1C0A92E2
:100890001C700A9B5A1C0A921C700A9B5A1C0A92D2
:1008A0001C700A9BFF22591C0A911A700A9B012294
:1008B000991814A80A911A7050F8283D9B1B3370A0
:1008C0001FF0AEFA2C70FDF7D8BF8C46894608465B
:1008D00004910591069107910B46FEF719BA9FED19
:1008E0006E7A13F0140F08BFF0EE477A7EF4F0AE84
:1008F000FEF7F7BE694B1868FFF799B9684A614B74
:1009000012680D93A3F14007002103F8401C212336
:10091000D100BB7040F13A8262490326624B1B88CA
:100920005A0500F12982D80700F13E8203F0020344
:100930005E4A002B1CBF03261146DFF88891324621
:1009400048462DF07CFC06EB090314A80133A9F1FD
:10095000020140F8203D00225B1A06F809207B7056
:100960001FF05EFAFEF742B8C4F81C8186F80090CA
:10097000FDF7FABE434A4E4B0D9214AEA2F13D0074
:1009800046F8200D19884B4FA2F1400300204FF08C
:100990000A0E02F8400C082283F801E030469A70F3
:1009A000F9F7EAFE3B684449DA1781FB0313C2EB0F
:1009B000A30399B23046F9F7DFFE0CF035F8BF68B3
:1009C0000C9B3A0C591C0C911A700C9B3A0A591C3E
:1009D0000C911A700C9B5A1C0C921F700C9B5A1C89
:1009E0000C92187030461FF01BFAFDF7FCBF334F16
:1009F0009FED338AB7F9022022480D9007EE902A26
:100A0000F8EEE77A14AE67EE887AA0F13D01FDEECC
:100A1000E77A46F8201D00F8403C0823CDED037A24
:100A200000F83F3C1E23BDF80C1000F83E3C304659
:100A3000F9F7A2FEB7F9003007EE903AF8EEE77A40
:100A4000304667EE887AFDEEE77ACDED037ABDF8A1
:100A50000C10F9F791FEB7F9043007EE903AF8EE72
:100A6000E77A304667EE887AFDEEE77ACDED037AD5
:100A7000BDF80C10F9F780FE30461FF0D1F9FDF7F4
:100A8000AFBF00BF5C630020F2460020481404089A
:100A9000501404085C14040800000000AC7400202A
:100AA000C05E002034140408CC6400204414040800
:100AB000D46200209072002067666666B0740020E1
:100AC00058A08B411F6300209AF80240C4B1013C3A
:100AD000E4B2013454445146002211F8013B534022
:100AE00083EA0313DBB2120ADE0042EA03228C42DD
:100AF00086EA131382EA0302EFD1002A7FF42AADBB
:100B0000C04AC14EC14B1288C149C24CF261DFF8E4
:100B100038931A6809689B68F262B4F84A21F06653
:100B2000F364D9F80000F163F265F7F725FB039051
:100B300000287DF487AE0221D9F80000F8F798FB71
:100B400094F84C319AF803200492642B4FF004027D
:100B500086F8742040F07C8194F84D31072B04BF57
:100B60009DF80C3084F84D3194F84D31079306EB25
:100B7000031ADAF80410039108462AF05FFBDAF84A
:100B8000081006915FFA80FA08462AF057FBC0B2B7
:100B900005900AEB0002079B9F48039903900832D7
:100BA000C27123F00F0286468272059803F00F038C
:100BB00000EBCA008EF80D3052468EF80E000EF192
:100BC0000F002DF03CFB954B059A06990AF10900A0
:100BD00018442DF034FB0398C37903F1010ACBB11B
:100BE000013B5FFA83FC0CF1080CDFF860E28444FF
:100BF0000023073010F8011B59408B00CA0883EA14
:100C0000410302F018024B404EFA02F25340844571
:100C1000DBB2EFD1814A04980AF8023027F0B2FB28
:100C200094F84D310022013384F84D3184F84C2181
:100C3000039BDDF80CA09B785BB11AF80510D9F87E
:100C40000000F8F72DFB01359AF80230EDB2AB4207
:100C5000F3D894F84C310322013384F84C3186F8F0
:100C600074203A70FFF7ABB902213868F8F700FB3F
:100C700094F82431FDF7A5BD4FF0010AFEF7B2BF8D
:100C8000326882EAE273A3EBE27303EB5303A1FB46
:100C90000331C908002AB8BF41F08041FFF7A4BB67
:100CA0005F49881F24F034F884F83E01FFF737BA13
:100CB000342694E410230026042218460CA98DF84B
:100CC00030308DF831208DF832608DF833608DF83A
:100CD00034608DF8356024F06DF984F82F61FDF7EC
:100CE0009ABD4B4B1E6806EB86067600FEF7EFB901
:100CF0004C4AD278002A0CBF4FF0040C4FF0050C80
:100D0000FEF710BE012338683370F8F7BDFA0646C7
:100D10003868F8F7B9FA72067DF426AD8A2851D002
:100D20008E287DF421AD94F81831002B7DF438AD78
:100D30003D4BC4F820312D2384F82431FDF71BBD31
:100D4000304B1888FFF76CBB0127FEF7E1B82D493F
:100D50009A790B8803EB830303EB83039F00BFB2F5
:100D6000002A00F01181294B1B680FFA83FA0BF05F
:100D70005BFE40B2FDF7E0BE03262C49DDE59C4654
:100D80009946184604930593FDF7C2BF284B294A9C
:100D90001B68294903F48003002B16BF1146042663
:100DA0000326BBE524261AE424490426C5E51026BB
:100DB00015E4138907EE903AF8EE677AFEF791BCD6
:100DC00020260CE41E4B1B689B067DF5CDAC94F8E9
:100DD0001831002B7DF4E4AC1A4BC4F820312D23DC
:100DE00084F82431FDF7C7BC4B1CDBB2042B84F81C
:100DF00041314FEA01613FF47CAC7DE40826FFF706
:100E0000EEBB00BFD46200202800002090720020BA
:100E1000AC740020D81E00204CA2002052A200205A
:100E20001020002044470020DC6300203814040810
:100E3000785B0020341404082C1404083C140408C3
:100E4000CC74002008640020287700200007090ED9
:100E500096F875A0574905951AF00F0F04BF0AF1CF
:100E6000010A5FFA8AFABAF1070F28BF4FF0010AA8
:100E70004FEA0A1C06EB0C03187C4F4B03930A182D
:100E8000002392F824104C4A93725FFA8CF31A46AE
:100E90004A4B964606EB0C024EEA000001291870F8
:100EA000D26803F101000CD90239C9B28D1C1D446E
:100EB000034603F8012BAB424FEA1222F9D101316C
:100EC0000844B44422F060030AF1010A9CF811209E
:100ED0005FFA8AFA1343BAF1080F037000F10103B5
:100EE00040D04FEA0A1C06EB0C01344A087C314919
:100EF00001449A1A91F8241055180EF1100E132D72
:100F00005FFA8EFEC6DD059D0398DFF8BCE0D2B225
:100F1000931DDBB243F04001C17103F1010CCBB171
:100F20000532D3B20833C31805930EF10100002334
:100F300010F8011B59408B0083EA4103CA084B405B
:100F40001F4902F0180241FA02F25340059A824208
:100F5000DBB2EDD104980CF80E3086F875A027F0BE
:100F600011FA65E6154A059D9A1ACDE7154B6420DE
:100F7000B3F900A0FDF7E0BD9C46994618460493DE
:100F800005930693FDF7C4BE4FF0FF33EDE69C4694
:100F9000FDF7BEBE9C469946FDF7BABE9C469946F3
:100FA0001846FDF7B5BE9C46994618460493FDF7D2
:100FB000AFBE00BF2CE503084CA2002059A20020C0
:100FC0000007090E9072002052A200202DE9F04780
:100FD000B0F908400C81E4B2442C8AB00D461646A4
:100FE00000F03D84074642D9812C00F0798300F25D
:100FF0009580542C00F0CC8040F2D6806E2C00F00E
:10100000FC83802C40F0D380754B93F8009009F15D
:10101000020919F0FF0900F09480724B724F734E71
:10102000DFF8F0A1994403F101080A2416E0322CFC
:1010300001F07482A4F13C00C0B2132841F2758221
:1010400000232A68511C296014702A68C14502F1E6
:1010500001012960137074D018F8014B0A2CE6D1F5
:10106000BAF80030FF2BA8BFFF23DBB2E9E7052C5D
:1010700000F0E3831FD8022C00F0828040F210833E
:10108000032C00F0B083042C40F09180584928468E
:101090002246F9F74FFB00212846F9F793FB2A680F
:1010A0000021531C01242B602046234611706B81C4
:1010B0000AB0BDE8F087242C60D040F2A782282C2B
:1010C00000F05683382C72D10A684A4B0124511C17
:1010D000296014702A6805211019286011702A6887
:1010E0000A211019286011702A680021101928603F
:1010F00011702A6819781019286011702A685978B7
:101100001019286011702A68997813192B602346EA
:10111000117020466B810AB0BDE8F087A02C17D073
:1011200040F29382B82C00F05C83FE2C3FD1324C0D
:1011300004F1080634F8021B2846F9F743FBA642DF
:10114000F8D10124234620466B810AB0BDE8F08720
:101150002A4B08461968F9F71DFB294B28461968E0
:10116000F9F718FB274B19682846F9F713FB0124F8
:10117000234620466B810AB0BDE8F087224BF2E798
:101180000422224928460124F9F7D4FA2346C0E76D
:101190000B6800215A1C2A6019702A68012413194F
:1011A0002B6023461170B4E7522C3FF478AF2946E8
:1011B0002046FAF7A7FF0028C3D1742C00F08382E1
:1011C000772C29D13B687A689A421BBF5A1C3A6037
:1011D000014619780E4A284629F0D4F8B1E700BF35
:1011E000D161002080E50308676666665C25002003
:1011F000F2460020F16F0020F4610020107AFF1FFA
:10120000147AFF1F187AFF1F98600020C814040882
:10121000F198030884250020F52C01F01782762C24
:1012200000F02583292C3E6801F0E381392C01F080
:10123000CF81212C01F0AC817A680B3C931BEF2C01
:1012400000F2A28701A151F824F000BF4923010850
:1012500089210108892101088921010889210108C2
:1012600089210108892101088921010889210108B2
:1012700089210108892101088921010889210108A2
:101280008921010889210108892101088921010892
:101290008921010889210108892101088921010882
:1012A000892101088921010889210108F922010801
:1012B00089210108B522010889210108932201082A
:1012C0008921010889210108892101086B2201086F
:1012D00089210108F52101088921010889210108D6
:1012E000892101088921010889210108E3210108D8
:1012F0008921010893210108892101080F21010892
:101300008921010889210108892101088921010811
:101310004311010889210108F320010889210108EE
:1013200089210108D9200108892101087B200108B1
:1013300089210108892101088921010889210108E1
:1013400089210108892101088921010889210108D1
:10135000D72401088921010889240108892101086D
:10136000892101084B2401088921010889210108EC
:1013700089210108892101088921010889210108A1
:10138000892101087F23010889210108F91F01082B
:1013900089210108131F010889210108711E010814
:1013A00089210108491E0108151E0108892101082B
:1013B0008921010889210108892101088921010861
:1013C0008921010889210108892101088921010851
:1013D0008921010889210108892101088921010841
:1013E0008921010889210108892101088921010831
:1013F0008921010889210108892101088921010821
:101400008921010889210108892101088921010810
:101410008921010889210108892101088921010800
:1014200089210108892101088921010889210108F0
:1014300089210108892101088921010889210108E0
:1014400089210108892101088921010889210108D0
:1014500089210108892101088921010889210108C0
:1014600089210108892101088921010889210108B0
:1014700089210108892101088921010889210108A0
:101480008921010889210108892101088921010890
:101490008921010889210108892101088921010880
:1014A0008921010889210108892101088921010870
:1014B0008921010889210108892101088921010860
:1014C0008921010889210108892101088921010850
:1014D0008921010889210108892101088921010840
:1014E0008921010889210108892101088921010830
:1014F000892101088921010889210108EB1D0108C2
:1015000089210108331E0108892101088921010868
:1015100089210108892101088921010889210108FF
:1015200089210108892101088921010889210108EF
:1015300089210108892101088921010889210108DF
:101540008F1D01083D1D0108011D010889210108A9
:10155000651C0108F51B0108D91B01088921010838
:10156000BF1B0108591B0108311B01081F1B010883
:10157000C11A010889210108931A0108892101086B
:1015800089210108711A0108431A01082F1A01085C
:10159000071A010889210108E5190108B91901088C
:1015A000A11901088921010889210108892101085F
:1015B000892101088921010889210108892101085F
:1015C000892101088921010889210108892101084F
:1015D0008921010889210108892101088719010849
:1015E00089210108892101082D1901088921010893
:1015F000892101088921010889210108892101081F
:101600008921010889210108BF180108202C7FF4D5
:10161000CEAD0B68B04C591C627829601A702B68EB
:101620002278591C29601A702B68A278591C2960ED
:101630001A7021892846F9F7C5F82B686279591C78
:1016400029601A702A68A1792BE5822C7FF4AFAD4E
:101650000B68A24AA24C11789F4A581C2860197046
:1016600011892846F9F7AEF89E4B2A681B88FF2B94
:1016700002F10101A8BFFF2329601370A16881F363
:10168000100189B22846F9F79DF8216801F30F018E
:1016900089B22846F9F796F8934B2A68197800E53D
:1016A000012C7FF484AD0B680022591C29601A704C
:1016B0002B685A1C2A601C702A682421531C2B603A
:1016C0002346117025E53B687A689A421BBF5A1C75
:1016D0003A6001461978854A284628F053FE30E5DD
:1016E000834B1E78033616F0FF063FF42AAD814B7C
:1016F000814F1E4403F101094FF00A0820E0B8F1C0
:10170000500F00F00887B8F1320F00F02487A8F1DD
:101710003C00C0B2132840F22287002421462B68E7
:101720005A1C2A60284683F80080F9F74BF82146B6
:101730002846F9F747F8B1453FF403AD19F8018B96
:10174000B8F10A0FDBD16D4B9C68196804EB840477
:101750004FF6FF7364009C42A8BF1C469942A8BF85
:10176000194624EAE47421EAE171A4B289B2D6E709
:101770000B68DFF8B481624E591C022229601A708E
:101780002B6806275A1C2A601F702B680A22591CD6
:1017900029601A702B6801241A192A601C70B8F885
:1017A00000102846F9F70EF8B8F802102846F9F7A5
:1017B00009F82B681A192A601F702B685022191912
:1017C00029601A702B680022191929601A70318853
:1017D0002846F8F7F7FF71882846F8F7F3FF234605
:1017E00097E4484BBFE40B685A1C0A601C700B68F6
:1017F0000222591C29601A7051E43A4B0A681B886E
:10180000374CFF2BA8BFFF23511C29601370A16820
:1018100081F3100189B22846F8F7D4FF3A4B2846E5
:101820001988F8F7CFFF216801F30F0189B2284624
:101830000124F8F7C7FF23466BE40B2233492846FF
:10184000F8F778FF082232492846F8F773FF012499
:10185000072230492846F8F76DFF234659E4002A4D
:101860003FF46FAC2C4B13600124234651E43B68DA
:101870005A1C3A601B78002B00F04287102B07BFE0
:10188000264A92E81200044621462A68501C286025
:1018900013702846F8F77EFF21462846F8F77AFFAE
:1018A0001F4B28461968F8F775FF28460021F8F7FE
:1018B00089FF00212846F8F785FFFFF7F0BB194B99
:1018C0001B78DB0700F160840124FBF777FCFCF751
:1018D000EDF923461DE400BFB8740020EA62002041
:1018E00090720020D46200202444002029A2030822
:1018F000D161002090E50308542500201025002028
:10190000442500203C440020645E0020D0140408DC
:10191000DC140408E814040835C0000888220020FC
:10192000802400206062002068600020731C3B60FF
:1019300033780F2B00F22884B21C3A60C3EBC30348
:10194000B34A7178D154F11C39601344B2785A709B
:10195000321D3A60F2789A70721D3A603279DA700C
:10196000B21D3A6072791A71F21D3A60B2795A71F9
:1019700006F108023A60F2799A71012414F0EAF94A
:101980002346FFF7C6BB3846F8F7C2FEA14EF081EA
:101990003846F8F7BDFE0124B0812346FFF7B9BBF6
:1019A0003846F8F7B5FE9C4A00EB8000430001245E
:1019B00013802346FFF7ADBB3246731C3B60974B49
:1019C00012F8021B19703A6072785A70F21C3A6071
:1019D000B2789A70321D3A60F278DA7001242346A8
:1019E000FFF797BB3846F8F793FE8D4E30823846A6
:1019F000F8F78EFE70823846F8F78AFE0124B0822E
:101A00002346FFF786BB3346721C3A60854A13F8BB
:101A1000021B11703B607F4A73789370F31C3B602C
:101A20007D4BB2789A7001242346FFF772BB7E4B40
:101A30007E4918684E2201242CF001FC2346FFF752
:101A400068BB3246731C3B60794B12F8021B19705D
:101A50003A6072785A70F21C3A60B2789A703846DE
:101A6000F8F756FE734B0124D8802346FFF751BB8D
:101A70003846F8F74DFE6F4E30803846F8F748FE8E
:101A800070803846F8F744FE0124B0802346FFF703
:101A900040BBDFF8C88198F80030002B3FF451AB11
:101AA000654E00243846F8F733FE14F097FE98F898
:101AB0000030A6EC010A01349C42F3DBFFF741BB86
:101AC0000D2B40F06183731C3B603478072C00F2CF
:101AD0005B83DFF88C8138460C26F8F719FE06FB8D
:101AE00004F608EB0604A0803846F8F711FEE08003
:101AF0003846F8F70DFE3B6820811A46591C3960BC
:101B000012F8021BA1723A605B78E3723846F8F76C
:101B1000E7FD012448F806002346FFF7FABA3846E5
:101B2000F8F7F6FD454B012418802346FFF7F1BA7C
:101B3000731C3B603078060600F15C86404B1B78D6
:101B4000DC073FF5FEAA032828BF00200124FBF78D
:101B5000F9FA2346FFF7DDBA731C3B60384696F866
:101B60000090F8F7BDFD80463846F8F7B9FD044609
:101B70003846F8F7B5FD06463846F8F7C9FD384649
:101B8000F8F7C6FD3846F8F7CFFDB9F1000F00F0C1
:101B90003C86B9F1100F7FF4D4AA2A4BC3F8008019
:101BA0005C600EB1284B1E602849294B0222081F99
:101BB00001241A7013F092F82346FFF7AABA204BBB
:101BC0001B78D8073FF5BDAA0124FBF7D7FAFCF72D
:101BD0006DF82346FFF79DBA194B1B78DA073FF5DE
:101BE000B0AA1C4A1378012443F00403137023465F
:101BF000FFF78FBA124B1B78D9073FF5A2AA164BF5
:101C00004FF4C87201241A802346FFF782BA00BF3E
:101C10003C49002078600020886000209C650020FE
:101C200024580020545B0020F846002030020408AD
:101C300070600020B04F0020084F00208465002015
:101C40006062002088220020802400208C22002056
:101C50006A640020D0740020F8A60020D161002022
:101C600030500020092B40F38F82DFF88483334605
:101C7000721CD8F800403A6013F8022B22703B60C7
:101C80007378A370F31C3B60B378642BA8BF642304
:101C9000321D63713A60F378642BA8BF6423721D10
:101CA000A3713A603379E371B31D3B607379642BA0
:101CB000A8BF6423F21D23723A60B379E37006F182
:101CC00008033B60F37923713846F8F721FD7A6801
:101CD0003B686081D11A00290CDD591CD8F800003E
:101CE0003960521A002A1978417203DD9A1C3A6051
:101CF0005B784370012427F0F3FA2346FFF709BA13
:101D0000AE4B1868F31C02462136991E396013F851
:101D1000031C1170591E396013F8021C51703B608E
:101D200013F8011C917003339E4202F10302ECD1BF
:101D3000012414F0FDFB2346FFF7EBB9731C3B6055
:101D400033789F4A002B00F07585137843F0020327
:101D5000B11C13709B4C3960737823753846F8F7C3
:101D6000BFFC20603846F8F7BBFC60603846F8F7E7
:101D7000CFFC20813846F8F7CBFC934AE0811378FA
:101D8000012443F0020313702346FFF7C2B9C3F3E3
:101D90004704122C00F2F881BCB10AAB0DF1020825
:101DA00003EB44094646A9F126093846F8F7B0FC8A
:101DB00026F8020FB145F8D1844B38F8022F23F8EA
:101DC000022F4645F9D1112C09D8814A6300023B04
:101DD00013440021223223F8021F9A42FBD17D4A8C
:101DE00001231C461370FFF794B93346721C3A6006
:101DF00013F8024B3B60F31C70783B60B178002C09
:101E000000F03585012C7FF49CA90AF0CBF823461D
:101E1000FFF77FB9704B1B7813F0010140F0B481DC
:101E2000731C3B603078012409F0FEFF2346FFF766
:101E300070B96A4E002338463360F8F751FC01242C
:101E400030602346FFF765B93346721C3A60644A36
:101E500013F8021BD1703B60624A73785371F31C14
:101E60003B60614BB278DA7001242346FFF751B929
:101E70003846F8F74DFC3846F8F74AFC3846F8F78C
:101E800047FC3846F8F750FC3B684C4C1946581C48
:101E90002268386011F8020B82F82C0039605978FA
:101EA00082F83610D91C39609B7882F83730384672
:101EB000F8F73AFC3846F8F737FC3846F8F734FCC0
:101EC00038462668F8F724FC708738462668F8F705
:101ED0001FFC3B687A683087D11A01290ADD591C3A
:101EE000226839601B7882F82E303846F8F71CFCDF
:101EF0003B687A68D31A032B09DD38462668F8F761
:101F000007FC708638462668F8F702FCB086206821
:101F10000EE7731C3B60294CDFF8D880337888F8D3
:101F2000053038462668F8F7F3FB308438462668D3
:101F3000F8F7EEFB7A683B68F083D11A072915DDC4
:101F40003846F8F7E5FBA8F80A003846F8F7E0FB52
:101F5000A8F80C0038462668F8F7DAFB7084384693
:101F60002668F8F7D5FB3B687A68B084D11A032954
:101F70000BDD3846F8F7CCFBA8F80E003846F8F72A
:101F8000C7FB3B687A68A8F81000D21A002A05DD62
:101F9000591C226839601B7882F82630FBF718F943
:101FA00017F0A6FD114B1B68002B00F04884206839
:101FB000012413F063FF2346FFF7ABB8F846002077
:101FC000D0740020D474002068640020AE75002016
:101FD000B0750020D4750020606200203C440020D1
:101FE00078600020A467002088600020A0600020A6
:101FF0002C440020545B00203346721C3A60DFF80A
:10200000F48213F8022B88F802203B60B04A737800
:102010001370F31C3B60AF4CB3782371331D3B60EE
:10202000F378092BA8BF09233846A370F8F770FB93
:102030003B687A682080D11A012905DD3846F8F717
:1020400067FB3B687A68E0819A4207D05A1C3A6085
:102050001B78003318BF012388F80730FBF7B8F866
:102060003B687A689A423FF46CA85A1C3A601B7825
:10207000E37001242346FFF74CB8731C3B60964B7A
:102080003278DFF86C821A700023C8F800303846C6
:10209000F8F726FB3A68D8F800309049904C034393
:1020A000501CC8F80030386013780B723846F8F7C7
:1020B0002FFB20603846F8F72BFB60603846F8F7B6
:1020C00027FBA0603846F8F723FB01243846F8F7D1
:1020D0001FFB2346FFF71DB8824B06F108020136AD
:1020E0003E6016F8011C03F8011F9642F7D1FFF776
:1020F00028B83346721C3A607B4A13F8021B917071
:102100003B607378537001242346FFF702B807221F
:10211000B3FBF2F2C2EBC2041B1B35D1D2B202F107
:10212000FF395FFA89F9002A3FF40BA809F1010988
:102130001C461EE086703846F8F7EAFA3B68A8F8B5
:1021400000001A46591C396012F8021B88F8031067
:102150003A605A7888F80420DA1C3A609A7888F84D
:1021600006201E1D3E60DB7888F805304C453EF4A5
:10217000E8AF731C3B6096F9006030460DF034FF09
:10218000013480460028D5D14FF0FF342346FEF7B6
:10219000C0BF731C3B6033780E2BF5D8B21C3A607D
:1021A00070780328F0D85149062202FB03F28B18FD
:1021B000F41C58713C60B0788854321D3A60F27853
:1021C0005A70721D3A6032799A70B21D3A60727913
:1021D000DA70F21D3A60B2791A7101242346FEF7D3
:1021E00098BF731C3B603D4B32785A7501242346DF
:1021F000FEF78FBF731C394C3B603378237238462F
:10220000F8F786FAA0833846F8F782FA2083384632
:10221000F8F77EFA3A686083531C3B601278E274E8
:102220007A68D31A032B00F3C6823B68D11A0529BA
:102230000EDD5A1C3A601B78E3723846F8F750FA04
:102240003B68E0605A1C3A601B7823743B687A68EC
:10225000D21A002A7EF775AF5A1C3A601B7884F8B0
:10226000213001242346FEF754BF731C3B601A49FA
:1022700030780870D21A002A7EF763AFB31C3B6037
:102280007378003318BF012301244B702346FEF7F7
:1022900040BF3846F8F73CFA114E30603846F8F740
:1022A00037FA70603846F8F733FA0124B0602346F5
:1022B000FEF72FBF0E4E002333603846F8F710FAB2
:1022C00033680124034333602346FEF722BF00BF77
:1022D0006C60002024580020A4600020F85C0020DE
:1022E000783C0020F75C00209460002048440020E7
:1022F00098600020545B0020731C3B603478132CE2
:102300003FF642AFB31C3B60707828F075F80028A8
:102310003FF43AAFC24B027803F82420F21C3A6033
:1023200003EB8403B2785A70321D3A60F2789A70E7
:10233000721D3A60BB493279DA700868012426F0D0
:102340005DFF2346FEF7E5BEB749102B4FF00002B4
:1023500028BF10230A604A608A60CA600A74002B92
:102360003EF4EFAE3A680139134401323A6012F894
:10237000010C01F8010F9342F7D1FEF7E2BE384697
:10238000F8F7C6F9044612F093FDFF283EF4D9AEE3
:102390003F2C00F2F9810DF12808002308F8243DB4
:1023A000E60841460DF103008DF80330013625F0B3
:1023B00037FD9DF80330F6B204F00704B34204F190
:1023C000010403D19DF80430A34203D021463046D6
:1023D00012F05AFD3B687A68D21A012A7EF7B1AE34
:1023E0005A1C0AA83A6000221C7800F8252D25F016
:1023F0000BFD9DF80330A3420AD08C4B1B683BB108
:102400009A79A24204D31B681B690BB120469847F6
:102410003B685A1C3A60404600221C788DF8042024
:1024200025F0E6FC9DF80430A3423EF48AAE7F4BD3
:102430001B68002B3EF485AE1B685B69002B3EF4E5
:1024400080AE20469847FEF77CBE794B1B78012B67
:102450003EF677AE731C31463B60DFF8EC8111F835
:10246000023B88F80230F31CD21A3960012A7078D6
:102470003B6040F3EF813846F8F74AF90124A8F8A9
:1024800000002346FEF745BE731C3B6096F80080B3
:10249000B8F1110F3FF678AEB31C3B60654C737812
:1024A00004F818303846F8F733F940F6CA03984272
:1024B000A8BF184640F2EE23984204EB4801B8BF8B
:1024C00018460124A0F2EE222346192092FBF0F2D6
:1024D0004A70FEF71EBE3346721C574C3A6013F822
:1024E000022B22713B60737863713846F8F710F95C
:1024F0003B6820805A1C3A601B78A3713846F8F775
:1025000007F93B6860805A1C3A601B78E37101242C
:102510002346FEF7FEBD494BFFF716B93388FF2B64
:10252000A8BFFF23DBB2FEF78CBD1DF02BFB0028FC
:102530003EF486AD03780A2B28D8B0F9023087FB29
:102540000312DB17C3EBA2039BB2FF2BA8BFFF2331
:10255000DBB2FEF776BD97E81200FFF7F7B81DF083
:1025600011FB00283FF4D9A803780A2B3FF6D5A821
:10257000B0F90430B0F9061003EB830383F3500481
:1025800021EAE171A4B289B2FFF7C9B80023DFE7FD
:102590003346721C3A602A4C13F8022B62703B607F
:1025A00073782370F31C3B60B378A3703846F8F758
:1025B000AFF83B682081591C1A46396012F8021B9B
:1025C00061713A605B78A37101242346FEF7A1BDD7
:1025D000731C3B6033780A2B00F09C803846F8F778
:1025E000A3F83846F8F7A0F83846F8F79DF8FEF754
:1025F000A8BD731C3B6033780A2B00F08680502BFB
:102600007FF460AD3846F8F783F80E4E30803846D8
:10261000F8F77EF8012470802346FEF77ABD00BFEC
:10262000A8600020F846002054600020BC870020ED
:102630001D71002078770020684500204825002083
:10264000B874002044250020207100203B687A687F
:102650009A4270D1894BFF221A704FF00009884CC2
:102660000BF018FE49462022864884F800902BF093
:102670000BFE8DF804909DF80430072B00F2828049
:10268000DFF83C827F4F4A469DF8043003EB43035A
:1026900008EBC3035B7CE3B19DF8043003EB430319
:1026A00008EBC30320215B699BB19DF8043003EB69
:1026B000430308EBC303586947F82200F7F72EF9E4
:1026C000237857F82300F7F7E7F922780132D2B2DE
:1026D00022709DF804300133DBB28DF804309DF890
:1026E0000430072BD0D92B68591C29601A70002E92
:1026F0003EF427AD644B336001242346FEF709BD49
:10270000624A92E81200FFF7C0B83846F8F700F8BE
:102710005F4E7BE7B31C3B605E4B72781A70F21C15
:102720003A60B2785A70321D3A60F2789A70012499
:102730002346FEF7EEBC5A1C19463A604F4811F882
:10274000022B027039605B784370042A03D9FF2A98
:102750007EF4A5AC81E750490978994205D8022A50
:102760007EF49DACFF2B7EF49AAC2B6801241A19E1
:102770002A601C70002E3EF4E4AC484B33602346C4
:10278000FEF7C7BC4A46AEE70DF10408404612F01A
:102790006FFBBDF80430A3423FF41CAE404B1B68F6
:1027A000002B3FF417AE1B689B69002B3FF412AE61
:1027B000204698470EE63846F7F7AAFFA084384629
:1027C000F7F7A6FF3B687A68E084D11A03297FF700
:1027D0002DAD1A46591C396012F8021BA1773A60D8
:1027E0005B7884F820303846F7F792FF3B687A68C8
:1027F00060841BE500F07F00032828BF002001242F
:1028000009F0ECFB2346FEF784BC204B1020C3F8F4
:1028100000805C600DF0C0FE224A137843F0010393
:102820001370002E3EF48DAC1F4B01241E60234616
:10283000FEF76FBC137803F0FD03FFF789BA1B485E
:102840001B491C4A1C4B036001240B601360234688
:10285000FEF75FBC194BB1781A88012412FB00F215
:10286000234692FBF1F2A8F80020FEF752BC0124A7
:1028700013F0CCFC2346FEF74CBC00BF9C2100208B
:102880001B480020AC76002095560208AC6400205E
:1028900068600020F16F0020D161002041C0000875
:1028A000BC870020D0740020802400202C4A002007
:1028B000804A0020804E002035870008D25E00202C
:1028C000645700202DE9F04F724B734A1C7893B087
:1028D00000F59C412031814607911160002C00F0E9
:1028E00027856E4A1268904240F227826C4A6D49F1
:1028F0001768DFF8E8B10492013C1C706A4C039140
:1029000007F48057002F40F02582039B5B7D002B4E
:1029100040F09B84049B1B681D0400F17787634B88
:102920009945A37800F27383002B40F07383604BCA
:102930000693049B1F6817F4805940F0FA83039BA9
:10294000BBF906605B8B9E42B4BF00260126594B43
:102950001B6813F0805300F00782069A127812F079
:10296000010200F0088203985349408C91ED037AEC
:1029700007EE900AF8EEE77AB4EEE77AF1EE10FA95
:1029800081F20A80002E40F0FD814C4D95F8A01098
:10299000002940F0F7814A484A49056895F82D50CA
:1029A00000200860486088604749002D40F0EB81B6
:1029B0000D70002A40F0EC81444B1A78002A50D167
:1029C0000399BBF900E04F8B898BBBF90200BE4530
:1029D000CCBF8025002545F040038E45A8BF2B467F
:1029E0009B0843F08005B842C8BF2B4643F0400522
:1029F0008842A8BF1D46BBF904E0BBF90600AD083C
:102A000045F08003BE45C8BF1D4645F040038E45D6
:102A1000A8BF2B469B0843F0800E284DB842C8BF84
:102A2000734643F0400E95F8A2708842B8BF7346D3
:102A30009F4201F04081A5F8A42085F8A6202449F2
:102A400085F8A2300F78002F01F0B1805F2B01F0E4
:102A500018816F2B00F0F887069B1B78D90740F18F
:102A6000BA87049B1B4A1B68059203F00403002BE2
:102A700040F04A850DF14008174D0023C8F8043096
:102A800005F15009109340F6330A192740F28336B6
:102A900029E000BF60570020E05200205C57002072
:102AA000785B0020F85C002044470020404B4C003D
:102AB00060620020C05E0020EC620020A0210020A7
:102AC000F8460020205E00200C2400202075002005
:102AD000D81C0020CC740020A860002004A6002090
:102AE00004354D4520D0AA78EB789A4217FB026155
:102AF000F6D26A78043217FB03633BF91220524581
:102B0000A8BF5246B2F5617FB8BF4FF461729142DF
:102B1000E6DA9A42E4DC29782429E1D840460435F3
:102B2000F8F796F94D45DED1B04B98E803001F78D1
:102B3000AF4B83E80300002F00F03C840121AC4838
:102B4000F8F796F9002840F09A81E378002B40F0DE
:102B50009681A84C23881DB225F00105AEB2B34280
:102B6000268000F0B286A44D02270E204FF01409F3
:102B70004FF0FF082F7085F8019085F802800DF066
:102B8000D9FB39469A482688F8F772F9002841F0AF
:102B9000458026F002039BB2B34223800AD0964BB5
:102BA0001421FF2202250E201D7059709A700DF01D
:102BB000C1FB2688914BDFF884A21978DAF804006B
:102BC0000393B50708BF81F00201C1F34001F6F796
:102BD00069FF24218648F8F74BF930B9069A137833
:102BE000590744BF23F004031370059B1B6813F0BF
:102BF0000A0F1DD005217E48F8F73AF9002800F0A9
:102C0000988625886F0740F1B58779480621F8F73F
:102C10002FF9002800F07A866E0640F18887072198
:102C20007348F8F725F9002840F03083059B1B68AE
:102C30009D0600F13B8327886D480C21F8F718F9B1
:102C4000002800F0388147F48073BB42238009D00C
:102C5000694B02251421FF220E201D7059709A70B5
:102C60000DF068FB664B1B78082B00F030810E2BB3
:102C700000F02D81049B1B685E0544D5614B1B79D8
:102C8000002B00F0E18014215948F8F7F1F80028F2
:102C900040F0DF801DF030F901200DF0E7F990B32E
:102CA000DFF89C8100254FF0CC0902E0DDB2022D57
:102CB00029D809FB05F76B1C58F80760002EF5D1E1
:102CC000C378514A90F9020052F82330019603224A
:102CD0000092012132460CF019F9034605EB45003C
:102CE00000EB0010049353B1314608EB8000CC2276
:102CF0002BF0CAFA049B48F807300135EDB21FF0FB
:102D000095FB0028D3D1069B1B78DD0740F1F280AC
:102D10003E493F4A01230B701370039BDAF8000011
:102D2000197801F00101F6F7BDFE059B1B685A07F3
:102D300000F1508113B0BDE8F08F364B364A1F6862
:102D4000049307F480570392DFF8F8B0334C002F58
:102D50003FF4DBAD00212648F8F78AF800287FF41D
:102D6000D4AD0BF031FCD0E578023FF5F6AD069A14
:102D7000127802F001022A4D002185F8A010002EE1
:102D80003FF409AE274901200870002A3FF414AE31
:102D9000F9067FF511AE244A1278D2063FF50CAE43
:102DA000B9F1000F7FF408AE002B7FF405AE7B0273
:102DB0003FF502AE1D4B1B78002B01F021841C4B0C
:102DC0009B78002E41F059843BB11A4A1A4B126885
:102DD0001B689B1A002BC1F28B841020104D0DF044
:102DE000A9FA012385F8A130E6E500BFE6460020F8
:102DF000C05E0020CC640020704500201CB2002082
:102E0000A4600020DC620020340604086162002017
:102E100094240020785B0020F85C002044470020C8
:102E2000A02100200C240020D0740020D81C0020F9
:102E30009460002054B20020803E002020B2002088
:102E400074A2002004A60020069B1B78D8077FF5FB
:102E500021AF3C2025F0ACF800283FF454AF0AF035
:102E600059F83C2025F032F800283FF44CAF0AF026
:102E700051F83C2025F02AF80028F0D143E7059BC3
:102E80001B689A077FF565AEBF4C2688F3073FF5B0
:102E900080AE46F001039E4223803FF47AAEBB4BE6
:102EA0001421FF2202250E201D7059709A700DF01A
:102EB00041FA26886DE627F480739BB2BB422380DB
:102EC0007FF4C6AEB24B1B78082B7FF4D0AE2288BD
:102ED00022F040039BB29A4223803FF4CBAEAB4B2F
:102EE00002251421FF220E201D7059709A700DF0DA
:102EF00021FABFE6A74B93F80090B9F1000F5FD11C
:102F0000DFF8E482A44F18F8030C3E784146A8F19C
:102F1000030526F043F9002800F0F083002E40F06E
:102F2000428405F10801687926F038F9002841F05B
:102F3000E9819A49A87A26F031F9002800F0F18356
:102F4000022E41F0E3819649E87B26F027F900281C
:102F500041F0E0819349287D26F020F9002800F017
:102F6000F183042E41F0DA818F49687E26F016F94C
:102F7000002841F0D7818D49A87F26F00FF900285D
:102F800000F0F183062E41F0B981894995F82300BC
:102F900026F004F9002840F05887864995F8280063
:102FA00026F0FCF8002800F0F183082E40F0378767
:102FB000814995F82D0026F0F1F8002840F0F183C2
:102FC0007E4B01221A7026F06EFB059B1B685A0788
:102FD0007FF5B0AE032026F00BF9002800F06686DE
:102FE000238813F008047FF4A5AE08200DF0ECFA56
:102FF0007348744D7449754A754BBBF80660006898
:103000002E80086014601C6013B0BDE8F08F0BB90F
:103010000123A3706F4B06931B201F7894F8216047
:1030200026F0E6F8012E07F00109824600F0258619
:1030300007F00203059394F82030DFF8B081664D65
:10304000052B69D8DFE813F05B004F000600DC00B9
:10305000FF008D00012E04BF052384F82030B9F154
:10306000000F00F05281039B5C4FB3F91810B8F8C1
:103070000030002261F30F0263F31F42002361F36B
:103080000F0361F31F43CBF8042039686269CBF862
:1030900000308A42C0F06784012E41F0FE82032294
:1030A00094F820300592CBE726F0CEF8012807D11E
:1030B0004A4FB8F802303A68642101FB03232361C8
:1030C000BAF1000F04D098F80630002B40F0908041
:1030D000012E21D0414F22693B689A42C0F03186CF
:1030E000012384F82030012E3BD098F80730012BC3
:1030F00000F014810FF084F994F82030A0E7B9F1C2
:10310000000FD1D14FF48060BAF1000F00F0FB83C3
:103110000DF05AFA00232361059B002B3FF409AC04
:1031200005980DF007F9049B1F6817F480593FF4C8
:1031300006AC1D212A48F7F79BFE00287FF4FFAB61
:10314000284A039BD2881B8BBBF90660991A8E42D2
:1031500040F3018613449E42B4BF00260126FFF7C8
:10316000F6BB1E4F3A68B8F80230642101FB032316
:103170004FF480600022236184F82020E2700DF07B
:103180000BFA94F820305BE7CC64002070450020F7
:10319000A4600020616200209E0000203C450020C9
:1031A00041450020464500204B4500205045002069
:1031B000554500205A4500205F45002094240020FA
:1031C000AC74002074240020802400207824002087
:1031D00070240020606200202275002054B200207C
:1031E000C05E0020B04F002032450020684500201E
:1031F0000FF006F903224FF47A7384F82020E3617C
:10320000A74F2B8843F002032B800BF0DDF93A68BF
:10321000E36913440422A36184F82020012E40F0C6
:103220009D853B68A2699A42BFF476AF9D4B1878A2
:1032300020B925F0DDFF00287FF46EAF2B8823F046
:1032400002032B808EE7964FE8E7039A013BD27D7D
:103250003BF91330002A40F08183A3F57A73B3F56C
:103260007A7FA8BF4FF47A7323EAE37307EE903AAC
:103270009FED8D7AF8EEE77A67EE877A8B4AFCEE5F
:10328000E77A17EE903A1380FFF749BB884B894ADB
:10329000B3F90430884982FB0302DB17C3EBA202B7
:1032A000059B0A801B689D067FF5C5AC834B1B7888
:1032B000980704D5824E337D042B00F2558527886C
:1032C00017F0300F3FF4B8AC10200DF065F9202056
:1032D0000DF062F97B4B278800221A707A4A7B48EE
:1032E0007B4E7C4D002111607B4A316000232960B8
:1032F00041608161036083604361C3611360516019
:10330000936053619161D36196E4654F3B6847F2E6
:1033100030520323E26184F8203072E70FF070F836
:10332000032240F6B83384F82020E3615C4F68E75D
:103330006A4F3B78002B00F09887694BDFF8B48127
:10334000DFF8B4B1DFF8B4A1039345465E460490BC
:1033500099460EE019F804109847032C28DC88B928
:103360003B782AF8020F01349C4205F1040580F2F3
:10337000EF80072CE1B23046DBF80430EADD9847F5
:1033800000B2EDE738F824206B88801A4FF47A7188
:103390009B1A01FB00F040F6CA0290FBF3F00844D0
:1033A000904240F2EE23A8BF10469842B8BF18469C
:1033B00000B2D5E7DFF848A1DFF84881494D0AF1AE
:1033C0005A064FF0010951461AF8010C25F0E6FEA5
:1033D000F8B19AF804009AF802309AF803E000EB8A
:1033E000400105EB8101013BD1F8B42003EB43031D
:1033F000434493420DD095F8E02081F8B0E009FAFB
:1034000000F022EA0000C1F8B430C1F8B87085F8C5
:10341000E0000AF1060A5645D5D13349204A334B1C
:10342000334D09681B78D2F8009008910793A5F1F5
:10343000B00A00266B685BB31F784FB3AA68A9EB8C
:103440000202002A0ADB9AF8E0200121B14022EAB8
:10345000010209F5FA718AF8E020A960079ABAB169
:103460002A7859780432D2B2002940F09B8203991D
:103470003BF91220098B01F1C800824240F33384EA
:103480009AF8E0109A7841FA06F3D80740F1C2841E
:103490000136042E05F10C05CCD1FFF74FBB00BF60
:1034A00054B20020D81C0020AAF1823F645E0020A4
:1034B000B07400206766666668240020D07400201F
:1034C000D47400206A640020646500201465002024
:1034D000E0230020F02400203C6500202C77002011
:1034E000F85C0020A02100202C4400206847002028
:1034F00050220020447700206C4700209E210020AD
:1035000049440020A0E50308A84D95F8AA3053B11E
:10351000069B1B78DE0706D5039BBBF906205B8B59
:103520009A4200F34D841121A148F7F7A1FC00282D
:1035300000F0208295F8AE302BB995F8A83013B979
:103540003223A5F8AC30012385F8AE30FFF792BAEC
:10355000DDF81090974A04921146974A0968A2FB39
:10356000092A42F201020A404FEA9A1A059200F033
:10357000FD81924D9248934C934A95F800E0007873
:1035800084F800E01070BEF1000F04D08E4A92F86B
:1035900000E08EF0010E854D0F2085F82400002BF1
:1035A00000F01283894B039E0C931B78B6F826C05B
:1035B0000B931C463B78B78C039E854A368B0E9640
:1035C0002646A2FB0442520802EB4202B21AD2B2D1
:1035D000CDF824C001F48051089295F82580DFF8D9
:1035E00008B2DFF824C20A900AF5967276460F9167
:1035F00005F1280400200692CDF83490AE46002E46
:1036000000F037823EF910201FFA82F9B9454FEADF
:10361000400103D3099DA94540F26F825CF8202048
:10362000924580F02F823BF90120059D002D40F04E
:103630004382013098422BF8012004F10604DEDBBE
:103640000A98644ADDF834908EF825800F280CBF64
:10365000012100218EF82400117000F0BC825E4C24
:103660005E4E5F4F35883868A1686268E06045F05B
:103670000405401A9042524F3580534D4FF00101DE
:1036800088BF00223970297088BF84F82120002B60
:1036900000F0B382049A03991768524EB1F824C01F
:1036A000B1F818E0504817F48057354640F0C7820B
:1036B00039460EE06A7802EB820202EB820202F2E5
:1036C000EE2292B201318B4220F8022B05F1020565
:1036D0000ED016F81120002A00F01382022AE9D039
:1036E0000131028820F8022B8B4205F10205F0D14E
:1036F0000C9A137801331370FFF704B908F1050130
:10370000687925F04BFD00283FF413AC012E40F002
:10371000F98505F10D01A87A25F040FD002840F05B
:10372000F5853249E87B25F039FD00283FF412ACDD
:10373000032E40F0EF852E49287D25F02FFD00282F
:1037400040F0EC852B49687E25F028FD00283FF4E9
:1037500012AC052E40F0E6852749A87F25F01EFD16
:10376000002840F0CB85254995F8230025F016FD6B
:1037700000283FF412AC072E40F06783204995F8EB
:10378000280025F00BFD002840F049831D4995F8DD
:103790002D0025F003FD00283FF412AC092E3FF464
:1037A0000FAC4FF009094B463CE300BFA0210020BD
:1037B000C05E0020785B0020D34D6210BC52002018
:1037C0004C010020684700204D010020D9760020E0
:1037D000ABAAAAAA6947002044470020227500200E
:1037E00054B200207877002004A600204145002034
:1037F000464500204B4500205045002055450020FF
:103800005A4500205F450020DC760020CC4DD5F8DD
:103810008830A9EB0303002BFFF681A8C94A95F86D
:103820008C30517C079AC5F888200133C64A039E24
:1038300032F81120B17D03F00F0385F88C302B4452
:1038400092B292FBF1F283F8902095F8901095F8DF
:10385000912095F8923095F89C000A4495F89310C1
:10386000134495F89420194495F895300A4495F836
:103870009610134495F89720194495F898300A4407
:1038800095F89910134495F89A20194495F89B30AF
:103890000A44134495F89D1095F89F20184495F814
:1038A0009E3001440B441A4442F30B12642AF17D0A
:1038B000A8BF642213B209B1C2F1640307EE903AC3
:1038C0009FEDA27AF8EEE77AD6E40221A048F7F756
:1038D000CFFA00283FF45DA92580B7073FF56AA914
:1038E00046F00203B34223803FF464A9994B0220BF
:1038F0001421FF2218700E2059709A700CF01AFDD6
:103900002688FFF757B90CF047FE03E425F0400383
:103910009BB2AB4223803FF482A98E4B0225142137
:10392000FF220E201D7059709A700CF003FDFFF7F6
:1039300076B9238823F00405ADB2AB4225803FF46D
:1039400064A9844B02251421FF220E201D7059709A
:103950009A700CF0EFFC2588FFF757B9C3F53B636D
:1039600008331BB279E403230593D0E47A4A92F832
:1039700000E008E695F8A830002B3FF47BA8069BF2
:103980001B7813F001037FF475A8012285F8A83095
:1039900085F8A920FFF76EB8694D012185F8A010C0
:1039A000FFF7F0B9012900F002849AF8E020012322
:1039B000B34001361343042E8AF8E03005F10C05BC
:1039C0007FF438ADFFF7BAB8069B644A1B781060E5
:1039D000DF0700F1038295F8A61000297FF441A8C3
:1039E000B5F9A430322B7FF73CA895F8A22001202E
:1039F000572A85F8A60000F09984049B1B6813F0F1
:103A0000040302D05A2A00F0E8855D2A00F0E6841B
:103A10005B2A00F026855E2A00F06C85562A00F0AD
:103A2000CD85972A00F08785A72A40F09E844C49CF
:103A3000049B0A781B6842F004020A70494A059206
:103A400003F00403FFF713B8B2F5FA7FFFF609A8F5
:103A500095F8A620002A7FF404A8069B1B78012174
:103A6000D80785F8A61000F1C48409F00FFFFEF70F
:103A7000F8BF002F3FD05CF8202092454FEA40016C
:103A8000FFF4D1AD384A384D525C05EB0109002AEC
:103A900000F0B880022A47D199F8012002EB820297
:103AA00002EB820202F2EE2292B2032833DD059D80
:103AB00012B2002D3FF4BDAD089D24F81520B8F1D9
:103AC000000F03D10B9D022D7FF6B3AD2288B4F811
:103AD0000290B4F804804A449044244A0FFA88F8CB
:103AE00082FB0852224DA2EBE87225F8018012B247
:103AF0004FF001089DE53A464100069D4CF82050E4
:103B000093E5CAB2022A04D9032A7FF4E9AD6246DA
:103B1000D8E57246D6E5012505FA00F90A9D25EAA1
:103B2000090512B20A9580E53BF80120BDE745F092
:103B30004003AB4223807FF4F0AEFFF770B800BFC4
:103B4000A0210020046800202068002014AE23413A
:103B5000C05E00207045002068470020843E0020A1
:103B6000D0740020CC74002078770020565555552D
:103B70001022002045F004039D4223800AD0B54B5B
:103B800002251421FF220E201D7059709A700CF02E
:103B9000D1FB2588B04BB14AB3F90430B04982FB60
:103BA0000302DB17C3EBA2030B80FFF72EB83946E5
:103BB000AC48F7F75DF900283FF406AF85F8A77029
:103BC00009F064FEFEF748BFA749A84A0C91DFF848
:103BD000C0B2012111701B21A2480593F7F748F9E3
:103BE000059B00287FF43BADA14CA24FE2683B68E7
:103BF000A3609B1AC82B00F25A83049B1F6807F42A
:103C0000805775E5C2B2022A40F2CF82032A8BD1D7
:103C10000E9A0F9D002D08BF3A4646E726F0010395
:103C20009BB2B34223803FF458AE0E202F7085F82C
:103C3000019085F802800CF07DFB26884DE600217E
:103C40000FE06A7802EB820202EB820202F2EE22BD
:103C500092B20131994220F8022B05F102053FF49E
:103C600047AD16F811201AB1022AEAD00288F0E70F
:103C7000CAB2032AFAD87246EBE700230593FFF78E
:103C8000DAB9B2F5FA7FFEF6ECAE95F8A630002B65
:103C90007EF4E7AE069B1B7801210B4085F8A61049
:103CA00000F0E7820AF090FCFEF7DBBE08200CF083
:103CB00073FCFFF73FB8704A70491068B5F9A4204B
:103CC000C76981FB07018911FF17781A00F5FF40CA
:103CD0007F3082423EF7B3AEC91B0A4412B2A5F848
:103CE000A420FEF7ACBEC8398A425CDA9AF8E0102C
:103CF0009A7841FA06F3D9073FF5CAAB5242012040
:103D000009920CF031FC7B1E099A162B00F24281BD
:103D1000DFE813F0E301F901CA0122020F023602C3
:103D20009D01880171015A014301400122023001C5
:103D300036029D0188011A010401EE00B201D6008D
:103D4000C0000EF05DFB032240F6B83384F820205B
:103D5000E361FFF756BA0126FEF7F9BD3A68E36959
:103D60001344A361FFF7D8B90A2025F041FA278848
:103D70008046002800F05882F90640F14483404D07
:103D800095F8F080B8F1000F7EF456AF0D200CF0DE
:103D9000D1FA012385F8F0302788B8F1000F7FF4BD
:103DA0009DAAFEF749BF9AF8E0300122B24023EA0B
:103DB000020309F5FA728AF8E030AA60FFF768BBDF
:103DC00000212848F7F754F800287FF4ACAB3223E1
:103DD00085F8AA00A5F8AC30FFF7A5BB294B1B78E6
:103DE000002B3EF43EAEE378002B7EF43AAE95F81D
:103DF000A7300133DBB2032B85F8A7307EF631AE56
:103E0000214B5B7813B9002E7EF42BAE0AF0DCFB5D
:103E1000FEF722BE002A0CBF0120022070E74FF0FF
:103E200008094B4603EB83031D4487F80090A978EB
:103E3000687811F029F8069B144A1B78012111704B
:103E4000D9077FF5C0A8FEF768BF4FF007094B46BA
:103E5000E8E700BF70450020B07400206766666622
:103E600084650020C05E0020D976002069470020CC
:103E70004447002054B20020B8670020D34D6210A0
:103E8000A021002068470020946000209424002096
:103E900004A60020DAF8E400DFF81C8790F836105A
:103EA00098F8023011446429A8BF642121EAE17125
:103EB00080F83610002B40F04B8412F039FB74E58B
:103EC000DAF8E400DFF8F08690F8371098F802305E
:103ED0001144FE29A8BFFE2121EAE17180F83710C4
:103EE000002BEAD0162025F0E1F9DAF8E400E4E747
:103EF000DAF8E400DFF8C08681781144C829A8BF49
:103F0000C82121EAE171817098F80230002BD4D0E9
:103F1000142025F0CBF9DAF8E400CEE7DAF8E40073
:103F2000DFF8948641781144C829A8BFC82121EA46
:103F3000E171417098F80230002BBED0132025F0BB
:103F4000B5F9DAF8E400B8E7DAF8E400DFF86886F3
:103F500001781144C829A8BFC82121EAE171017084
:103F600098F80230002BA8D0122025F09FF9DAF83B
:103F7000E400A2E7DFF84086089898F8023041791B
:103F800011446429A8BF642121EAE1714171002B29
:103F900040F09383DAF8E4008FE7DAF8E400DFF822
:103FA0001886017A98F802301144C829A8BFC821A0
:103FB00021EAE1710172002B3FF47FAF0B2025F065
:103FC00075F9DAF8E40078E7DAF8E400DFF8E88574
:103FD000C17998F802301144C829A8BFC82121EA44
:103FE000E171C171002B3FF468AF0A2025F05EF942
:103FF000DAF8E40061E7DAF8E400DFF8BC858179FB
:1040000098F802301144C829A8BFC82121EAE171FB
:104010008171002B3FF451AF092025F047F9DAF800
:10402000E4004AE7DAF8E400DFF88C85417998F893
:1040300002301144C829A8BFC82121EAE1714171A9
:10404000002B40F04183112F7FF456AF35E7DAF8AB
:10405000E400DFF86485017998F802301144C8293A
:10406000A8BFC82121EAE1710171002B40F07483DF
:10407000102F7FF457AF20E70898DFF83C85417890
:104080001144B1F5967FA8BF4FF4967121EAE17112
:10409000417098F80230002B3FF47CAF152025F0DA
:1040A00005F9DAF8E40008E70899DFF80C850F79DC
:1040B0001744642FA8BF642727EAE7770F7125F01C
:1040C0000FF998F80230002B3FF464AF0320394613
:1040D00025F0ECF8DAF8E400EFE60898DFF8D88489
:1040E00001781144FA29A8BFFA2121EAE17101708F
:1040F00098F80230002B3FF44DAF012025F0D6F8A0
:10410000DAF8E400D9E60898DFF8AC848178114445
:104110006429A8BF642121EAE171817098F8023016
:10412000002B3FF437AF022025F0C0F8DAF8E400A6
:10413000C3E60898DFF88084C17998F8023011440A
:1041400081F30801C171002B3FF424AF052025F055
:10415000ADF8DAF8E400B0E6089BDFF85C84997902
:1041600098F8020011446429A8BF642121EAE17192
:104170009971002840F0B0820D2F7FF4FDAE09E761
:10418000DAF8E400DFF83084C17898F8023011449E
:10419000C829A8BFC82121EAE171C170002B40F0F5
:1041A00084820F2F7FF4D4AE87E60E9A7DE43BF92C
:1041B00012209978B2F5617F4FF4966393FBF1F387
:1041C0004ADB40F633019142A8BF11460C2FA1F5FE
:1041D000617191FBF3F100F08381182F7FF4E5AB5F
:1041E000C9B2C8290B46A8BFC823DAF8E400C27DCB
:1041F000DFB297423FF4D9AB9A1ADFF8BC83C77598
:1042000048BF0732D71098F802300137FFB23BB9E8
:10421000002F3FF4CAAB38460CF0A6F9FFF7C5BB38
:10422000182025F043F8F3E7FA0600F14F810B2040
:1042300024F0DEFF002840F01881BB0600F1528117
:10424000C34D95F8F030002B3FF4A0ADB8F1000F4E
:104250007FF444A8FEF7F0BC0C2F00F0EA80182F82
:104260007FF4A3AB00210B46BFE7BA4A0392FFF7E6
:1042700071B9B949096811F4003140F03F810B462A
:10428000B648C65C0F2E03F10C031ED00131152970
:10429000F7D1049BB2491B680591FA3AA5F8A4200E
:1042A000002203F0040385F8A620FEF7E0BBAD4A28
:1042B000049B1F68138823F004031380012307F471
:1042C000805784F82130FFF713BAA74ED6F800E0E4
:1042D0004B00BEF1000F07D05F1800EB87079EF878
:1042E00001E07F787745D4D20B44A04FA04900EB82
:1042F0008300002330603B800B60CAE74FF0060963
:104300004B468FE54FF001094B468BE54FF0020914
:104310004B4687E54FF003094B4683E54FF0040910
:104320004B467FE54FF005094B467BE5914B9249A3
:104330001A684FF47A73B3FBF2F3C3EB431203EB47
:104340008203049A1268DB001206A1F8B43000F16F
:10435000E580834B05931B685F0700F1D680049BC3
:104360001B6803F00403FEF782BB0021BB2A1091F7
:1043700000F08081B72A00F07981BE2A00F07481B4
:10438000BD2A00F04D81792A00F0DB817A2A00F005
:10439000D1819E2A00F0C8819D2A00F0BE81AE2AFC
:1043A00000F00182AD2A00F0F781EF2A00F0EE81E3
:1043B000FD2A00F0E581FB2A00F0DC81FE2A00F0F6
:1043C000D381F72A00F08E817B2A7EF44AAB4FF42A
:1043D000FA61022007F028FDFEF743BB674B00227D
:1043E0000120674D67492A700B600CF0BDF8FEF79D
:1043F00038BB049B64491B680A60594A059203F064
:104400000403FEF734BB10200CF0DEF820200CF083
:10441000C3F85E494E4D081F10F060FC5C4B022251
:104420001A7095F8F030002B00F03B812788FEF7DA
:1044300055BF00273946524B09915B78BB423FF488
:10444000B4AADFF87481384607F0C8FD98F8023046
:1044500009991BB1C9B20C2024F028FF0137FFB223
:10446000D6E64C4B01220220BBE74B4A4B4B52890C
:1044700093ED007A07EE902AF8EEE77AB0EEC77A6D
:10448000B4EEE77AF1EE10FA7FF5D7AE93ED017A4C
:10449000B0EEC77AF4EEC77AF1EE10FA7FF7CDAE40
:1044A000BB063FF5CDAE2A4D20200CF08DF82946F5
:1044B0007268336841F8EC2F05F1E800C5F8E83080
:1044C00010F00CFC324B01221A70AAE710200CF0FD
:1044D00063F82F4B278883F800804FF00108A6E689
:1044E000CFB2A8E720200CF057F8294B184D002236
:1044F0001A7096E72A4B0222032072E729490978AD
:10450000032900F0C5801946BAE6049B264A1B68B9
:104510000A21118003F00403FEF7A9BA234B1B788C
:104520009B077FF516AF224B1B7D042B7FF611AF47
:1045300010F05EFB0DE7049B1E4A1B684FF4C87128
:104540001180074A059203F00403FEF790BA00BFFA
:10455000A0210020F85C00203C440020B4FC0308AB
:10456000CC74002022750020B8230020562400209F
:1045700058240020685B0020B4A7002004700020AD
:10458000EC460020F8460020843E0020B064002065
:104590006A6400205270002008650020EC62002050
:1045A000A070002024440020F6A60020D074002033
:1045B000D4740020F8A600202071002014F030FDF3
:1045C000F5F79CFE14F014FDF9F770FB01200BF0D9
:1045D000CBFF95F8A220FFF724BA95F8A820002A6F
:1045E00040F0938095F8AA3083F0010385F8AA3053
:1045F000002B40F085800C200BF09CFEFEF731BABA
:10460000002E3EF4EAAB6B4D95F8A130002B3EF442
:10461000D3A90BF071FE002385F8A130FEF7CCB9C9
:104620004FF6FE73644A654896890590D0893344F5
:1046300001449381D18114F0F3FCF5F75FFE14F08F
:10464000D7FCF9F733FB01200BF08EFF049BB5F884
:10465000A4201B68FA3A0021A5F8A42003F0040363
:1046600085F8A610FEF703BA0223DBE70B464FF6E8
:10467000FE71D7E70B460221D4E7002BC3D0504987
:10468000504A09684FF47A7000FB03131360BAE7CD
:104690000BF032FEB5F9A420FBE503230593FEF7EA
:1046A0003FBD4FF00108FFF771BB0F20099224F0C6
:1046B000FDFDDAF8E400099A73E50E2024F0F6FD1A
:1046C000DAF8E400FFF7F9BB1120099224F0EEFDBF
:1046D000DAF8E400099AB6E40D20099224F0E6FD28
:1046E000099A49E50021042007F09EFBFEF7B9B9BD
:1046F000304D09F069FF002385F8A130FEF75CB961
:104700000B200BF017FEFEF7ACB92C4A85F8A81069
:1047100085F8A9000592FEF7AAB90021FF2027F02D
:10472000E7FA95F8A2203AE6012027F0E1FA95F899
:10473000A22031E6244A137A43F001031372FEF7F4
:1047400090B9214A137A23F001031372FEF789B955
:10475000172024F0ABFD1DE41020099224F0A6FDE3
:10476000DAF8E400099A83E40021032007F05CFBF7
:10477000FEF777B90021022007F056FBFEF771B96A
:104780000021012007F050FBFEF76BB9002108461D
:1047900007F04AFBFEF765B9FF21002027F0A8FAD1
:1047A00095F8A22001E60121002027F0A1FA95F852
:1047B000A220F7E5A021002078600020CC74002022
:1047C00054B20020803E00208C6500202DE9F04787
:1047D0008C4B1B78DB07074644D58B4B8B4D1C78E5
:1047E0008B4E012C59D01CD3022C07D189498A4AFF
:1047F00009881288914201D901241C70EB7AE3B137
:104800002B89D3B1854B1B78BBB108F00DF900287B
:1048100000F09B802B7B83422CBF01210021317053
:104820000CE07C497E4A098810886A7B801A88429D
:10483000E2DAEB7A0024002BE2D131782A79632A7C
:1048400006D8022C774E00F0BA803378002B5DD169
:10485000754AAB7A8C4238BF0C461470002B4CD191
:10486000BDE8F0876B4B694D19885B88E878CB1AF7
:1048700083EAE3728142A2EBE3721DD32B788B4271
:104880001AD3614B1C78E01E012861D96749097869
:1048900002294FD0012C5E4EA5D15F4A5D49128896
:1048A000687B0988121A914239DD5D4A12888A4272
:1048B000A4D200241C70A1E7B1EB400FE1DC524B05
:1048C0001C78E11E012940F29480022ADEDC57495F
:1048D0004F4E0878DFF84481DFF844C1DFF838E153
:1048E00000210324022834701C7088F80010ACF8F2
:1048F0000010AEF8001081D11FE0012C71D0022C05
:104900000BD10720BDE8F0470BF014BD7068381AD2
:10491000474B984258DD72709AE7BDE8F087022451
:104920001C706BE7022AD2DD4049097802294FF05A
:10493000040464D13949364E09783E48022ACCBF76
:1049400000220122C28081804BE70221317075E78D
:10495000022A9BDC95F800C091FBFCFC0CF1010CD9
:10496000BCF1080FDFF8B4A0304EA87895F801E04C
:1049700096F800802A4CDFF8A090254EA8BF4FF093
:10498000080C8AF800C01FFA8CFA10FB0AF01EFB14
:104990000AFE80B2DFF88CA02080A9F800E0002495
:1049A0004FF0640EB8F1020F34701C70CAF8044066
:1049B0008AF801E07FF439AF0FFA8CF1BDE7307867
:1049C000A0B9012377603370C2F164021A4B00FB77
:1049D00002F083FB0023C017A0EBA350643070707B
:1049E00036E70820BDE8F0470BF0A4BC7368F81A5E
:1049F0008EE7032C96D10D49097802299AD0044EEE
:104A0000FCE600BF60620020AC250020B8740020E6
:104A1000B2250020D4620020B0250020EA620020E8
:104A2000AE2500206024002024440020F0610020F6
:104A30007F969800F46100206BCA5F6B2DE9F04F00
:104A40002DED0A8B404B1B7893B0012B039001F0A6
:104A5000C4803E4C94F80021002A41F0CF80072BFF
:104A600001F0D6804FF0000ADFF8ECB0DBF804303C
:104A700058469847002800F06F81BBF8B4600022C8
:104A80008BF85520002E40F06887BBF93C50DBF8CE
:104A90002410BBF93E00DBF82820BBF94030691A2E
:104AA000CBF830102A490191821ADBF82C00CBF8A0
:104AB00034200D461B1A9BF85610CBF838300BF1FA
:104AC000300014F0F5F82B68990040F1E980DBED37
:104AD0000D5ADBED0C7A1F4A94ED416AD4ED426A1F
:104AE00094ED437AD4F810311268B8EEE58ADBED24
:104AF0000E5AF8EEE77AF8EEE58A013377EE867A19
:104B000038EE268A78EE878A9342C4ED417A84EDA6
:104B1000428AC4ED438AC4F8103101F0FD820A4B89
:104B20001E78142E02F0B1840023D4F81851029399
:104B3000062D00F2A880DFE815F00713F6121B120D
:104B40008B1211003114CA13F0610020942200204E
:104B5000785B00205C530020B4A70020D74B1A7864
:104B6000D4F81C71DFF8BCE39FEDD57AF8000EEBAA
:104B7000000383ED007A002A7AD0D249B0EE476A6A
:104B8000F0EE476A0023F1EC017A013367EEA77A71
:104B900005EE903AB4EEE77AF1EE10FAF8EEE55A47
:104BA000B8BFB0EE677A9A4276EEA76AA7EEA56A1A
:104BB000E9D1F5EEC06A0EEB0003F1EE10FA83EDD9
:104BC000007A55DDC6EE265ABF4BC04A1288F7EE72
:104BD000007A75EEE75AD3ED007A65EEA77AFDEE1E
:104BE000E77A17EE903A812B43F327839342A8BFCD
:104BF000134607EE903AF8EEE77AB54BC11903EB8E
:104C0000810393ED057AD3ED003A93ED066A93EDB7
:104C1000014AD3ED046AD3ED034A93ED025AA3EEA1
:104C2000A77AA4EE276A66EEC76AA7EE646ABDEEAD
:104C3000C77AE5EE276A17EE101A812983ED056A17
:104C4000C3ED066A43F3F6828A42A8BF0A4607EE1E
:104C5000902AF8EEE77AFCEEE77ACDED047ABDF81B
:104C600010300EEB0002938017B9132E03F0B687B5
:104C7000152E42F0CF817044DFF8AC82838828F88B
:104C80001730D4F81851934B013583FB05235A197B
:104C9000EB17C3EBA203C3EBC303ED1AC4F818511F
:104CA0008D4B1B78002B01F0EF808C4DCDF808A0C8
:104CB000DFF87882DFF87092DDF804A005F2DC6797
:104CC0000026874BDBED087A1B78172B01F04E840A
:104CD00095ED007AB8EEC78A082B28EE278A07D10F
:104CE000B0EE480A019327F0B9F9019B29F81600A4
:104CF000DAF8002092000BD5002E04F00081B0EE0F
:104D0000480ADBF8783707F170009847B0EE408A20
:104D1000B0EE480ADBF89836A7F170009847DBF848
:104D20000837384698476E4B1B78032BB0EE408A05
:104D300001F0FB83D5F85C06DBF8B830B0EE480A2A
:104D400098470136032E07F12407A8EC010A05F164
:104D50000405B6D1DDF808A0614B1F78072F00F0DD
:104D6000BC8694F828310493002B40F0C4865D4B38
:104D70005B79002B40F0EB850123594A84F82831F8
:104D80001278072A01F0848600230693564B94ED8F
:104D90004C9A93ED007A554BDFF89481D3F800A03C
:104DA000534B0293F7EE007A37EEC9BA08F11C03B1
:104DB0002BEE07BA0025B4EEE7BAF1EE10FA059330
:104DC000D4ED4BBA4B4BDFF86CB1DFED4B8A9FED66
:104DD0004BAADFED3BAADFED4A9ADFF85C91494F21
:104DE000019388BFB0EE67BA2E46474B98ED008A14
:104DF0002B44D3ED007AF5EE407AF1EE10FA17D09D
:104E0000424B2B44D3ED006A38EE667AB0EEC76AA7
:104E1000F4EEC67AF1EE10FA08D5B5EEC07AF1EEEE
:104E200010FACCBF37EEA68A36EEE78A83ED008A09
:104E3000374B1A88930700F08180022E7ED0354BC5
:104E40009AF82E1033F9163007EE103A059B07EE4C
:104E5000901A2B44F8EEE76AB8EEC77AD3ED007AE1
:104E60004B42A6EEA77A700007EE903AF8EEE77A8A
:104E7000B4EEE77AF1EE10FA0AD407EE901AF8EEE3
:104E8000677AF4EEC77AF1EE10FA88BFF0EE477A4F
:104E9000214B22490344085EB3F90C30C01A07EED7
:104EA000100AB8EEC77AD007E7EE687A40F12B8691
:104EB0001B4B93ED008A27EE888A3FE06253002067
:104EC0000000000094220020645300206053002062
:104ED000985500209324499254530020E4A70020C1
:104EE000F0610020545B0020D44E0020F8460020E2
:104EF000685B0020145E0020CDCCCC3DAE47813FE6
:104F00000000C842205E0020C84E0020D4230020AC
:104F1000CC640020E023002078600020B0740020E2
:104F2000B04E002080550020F46100206C5B002012
:104F3000C8230020284A00202C5E0020029B94F801
:104F400068212B44D3ED01CA38EE6CCA002A3DD04B
:104F5000D34BD4F86C2103991B688A1A9A4235DD29
:104F60009AF84830022B01F0CA85022E03F06787B9
:104F7000CC4B1B68990740F16E87CB4BCB49DFF8D0
:104F8000A0E331F916C09EED008ADFF898E3C7ED83
:104F900000AA03EB460028EE288AB0F90C00A0EB2B
:104FA0000C0007EE900AF8EEE77ADEF8000027EE34
:104FB000888A904238EE6CCAC1F28380F7EE007A9C
:104FC000B4EEE79AF1EE10FA01F15280B84B2B449F
:104FD00093ED000A019B2BEE800A022E20EE0C0AB4
:104FE000A3EC010A019303F04487B24B9BED007AD6
:104FF000D3ED007AB04BD7ED006A93ED006AAF4B6A
:1050000067EE277A2B4427EE8B7AD3ED007A67EE92
:10501000277AF0EE665AECEE275AB1EE467AF4EEB5
:10502000C75AF1EE10FA08D4F4EEC65AF1EE10FAAF
:105030008CBFB0EE467AB0EE657A94ED4C6AF7EE2E
:10504000007AB4EEE76AF1EE10FAACBF0123002358
:1050500043B1F0EEE66AF0EEC77AF4EEE67AF1EEEE
:1050600010FA01D587ED007A022E03F0E186944A0A
:10507000944B52F826001B68B0EE6C0A9847924A8F
:10508000924B52F826001B6898479AF8373023B1A4
:105090008F4B1B88002B00F0C085B0EE6A8A8D4BC9
:1050A0009BED007A38EE400A2B4493ED008A83EDA5
:1050B000000A9AF8483030EE480AC0EE077A2BB35F
:1050C000854B1B78DB0721D5B7EE007AB4EEC79A83
:1050D000F1EE10FA04DB94F86831002B00F06F87D2
:1050E000D4F86C31039AD31A6D4A12689A420DDDD6
:1050F0007A4B93ED007AB0EECCCAB4EEC7CAF1EEAB
:1051000010FA40F1FA87002384F86831744B94F860
:1051100078212B4493ED007A2BEE877A67EE277A7D
:10512000C9ED007A32B9019BC7ED00AA43ED01AA8F
:10513000C9ED00AA0136032E08F1040809F104099B
:1051400007F1040705F104057FF44FAE654B1B78AA
:10515000072B01F02182012B01F09F840023029391
:1051600094F88031002B40F0A1855F4B5F4A1B68AB
:10517000126813F4805C92F82C2040F0AE865C49F3
:105180005C4891ED006A408B5B4984ED646A91ED67
:10519000007A5A4984ED657A07EE900AF8EEE76ADC
:1051A000D1ED037A564984ED626A37EE467A77EE9E
:1051B000E67AD1ED006A84ED617A012184F89811D4
:1051C000C7EEA65A4F48504990ED005A4F489FED00
:1051D000506A90ED004A4F48DFED4F6AD0ED004A2B
:1051E00091ED007A35EE045AF7EE007AF4EEE75AC4
:1051F00035EE245AF1EE10FA88BFF0EE675A25EE2C
:10520000065AF4EEE65AB1EE476AF1EE10FAB4EE41
:10521000C65AB8BFF0EE665AF1EE10FAC4ED675AFE
:1052200001F10780B4EEC75AF1EE10FA88BFB0EE74
:10523000475A3449DFED366AD1ED017A334991EDB1
:10524000014A344977EE847AD1ED014A77EEA47AA7
:1052500067EEA67AB4EEE76AF1EE10FA08DCB4EE77
:10526000E77AF1EE10FA8CBFB0EE676AB0EE476AEB
:105270002449DFED276AD1ED027A2449D1ED024AB3
:10528000264977EEA47A91ED007A67EEA67AB1EE20
:10529000473AF4EEC37AF1EE10FA4ED444E000BF80
:1052A000DC4E0020CC74002078600020B074002018
:1052B000844E0020A0000020F84E0020904E0020D8
:1052C000304A00202C4A0020844A0020804A0020D6
:1052D000CC6400200424002060620020E84E0020FE
:1052E0009C4E0020F0610020785B0020F8460020F2
:1052F000D85E0020F85C002048600020EC620020AE
:10530000B84F0020145E0020FC4E0020205E0020DC
:105310006F12833A2C5E002000000000004F002036
:10532000B04E0020D84E0020F4EEC77AF1EE10FA0D
:105330008CBFB0EE473AB0EE673AED49497809B90B
:10534000B1EE433A002A41F04B82F7EE003ADFF823
:10535000C8B39BF80020002A02F04582E549DFED42
:10536000E66AD1ED024A91ED017AD1ED037A66EE5B
:10537000244AE5EE074AE3EE274A63EEA44AF4EE38
:10538000E64AF1EE10FAB4BFB0EE664AB0EE644AF7
:1053900098BFF0EE646A012ACDED0A4A02F0448219
:1053A00091ED067AD1ED052AD1ED077A26EE077A3E
:1053B000A5EE227AA3EE277A23EE877AB4EEE67A78
:1053C000F1EE10FAB4EEC47A8CBFF0EE667AF0EE2D
:1053D000477AF1EE10FA98BFF0EE676AB4BFF0EECC
:1053E000447AF0EE477A022A8DED0B7A00F0DE80E7
:1053F00091ED0A7AD1ED092A91ED0B4A26EE077A52
:10540000A5EE227AA3EE047A23EE877AB4EEE67A4A
:10541000F1EE10FAB4EEE77A8CBFB0EE664AB0EE69
:10542000474AF1EE10FA98BFF0EE446AA8BFF0EEDA
:10543000477A032A8DED0C7A00F0B88091ED0E7A50
:10544000D1ED0D2A91ED0F4A26EE077AA5EE227ACC
:10545000A3EE047A23EE877AB4EEE67AF1EE10FA40
:10546000B4EEE77A8CBFB0EE664AB0EE474AF1EE92
:1054700010FA98BFF0EE446AA8BFF0EE477A042A0B
:105480008DED0D7A00F0928091ED124AD1ED112A46
:1054900091ED137A26EE044AA5EE224AA3EE074ABE
:1054A00023EE844AB4EEE64AF1EE10FAB4EEE74A8F
:1054B0008CBFB0EE667AB0EE447AF1EE10FA98BF87
:1054C000F0EE476AA8BFF0EE447A052A8DED0E4A49
:1054D0006CD091ED164AD1ED152A91ED177A26EE92
:1054E000044AA5EE224AA3EE074A23EE844AB4EE0C
:1054F000E64AF1EE10FAB4EEE74A8CBFB0EE667AF7
:10550000B0EE447AF1EE10FA98BFF0EE476AA8BF09
:10551000F0EE447A062A8DED0F4A47D091ED1A4AF3
:10552000D1ED192A91ED1B7A26EE044AA5EE224A06
:10553000A3EE074A23EE844AB4EEE64AF1EE10FAEF
:10554000B4EEE74A8CBFB0EE667AB0EE447AF1EE84
:1055500010FA98BFF0EE476AA8BFF0EE447A072A27
:105560008DED104A22D091ED1E7AD1ED1D2A91EDDC
:105570001F4A26EE077AA5EE227AA4EE037A27EEDA
:10558000237AB4EEE67AF1EE10FAB4EEE77A8CBF45
:10559000B0EE666AB0EE476AF1EE10FA8DED117A60
:1055A00098BFF0EE466AA8BFF0EE477A77EEE67A4B
:1055B000F7EE006AF4EEE67AF1EE10FAC4ED4C7AFA
:1055C00043F3A88286EEA77A022ADDED0B7A67EE16
:1055D000244A67EE877ACDED0A4ACDED0B7A2DD0BD
:1055E000DDED0C7A67EE877A032ACDED0C7A25D0B3
:1055F000DDED0D7A67EE877A042ACDED0D7A1DD0A8
:10560000DDED0E7A67EE877A052ACDED0E7A15D09C
:10561000DDED0F7A67EE877A062ACDED0F7A0DD091
:10562000DDED107A67EE877A072ACDED107A05D086
:10563000DDED117A27EE877A8DED117A2F49096811
:1056400011F0805800F0A387F6EE005AC4ED675AB7
:10565000002A02F0BF8094F99801D4ED654A284DE4
:10566000284994ED646A284E284FDFF8B0E0B5F879
:105670001AA0C978B6F9069097ED005A9EF800E096
:10568000D4ED616AD4ED627A07EE100AFDEEE44AC9
:105690001F4814EE905A0078FDEEC64A03F010063B
:1056A00003F4800300F00107B8EEC77A14EE900A05
:1056B0000193002941F0D4800E49002E40F08987E3
:1056C00091ED006A9DED0A5A124B25EE866AA5EE11
:1056D000076AB0EE675AA6EE265ABDEEC56A16EE08
:1056E00010EA16EE106AAE45A8BF2E4618E000BFBD
:1056F000A4600020284F002000000000C05E0020B1
:10570000F85C00204447002004A60020044F00203D
:1057100060620020785E0020D1610020485800209F
:105720007045C8BF064606EE106AB8EEC66A012A82
:1057300083ED006A00F0DC8091ED046A9DED0B5A68
:1057400025EE866AA5EE076AB0EE675AA6EE265ADF
:10575000BDEEC56A16EE10EA16EE106AAE45A8BF99
:105760002E467045C8BF064606EE106AB8EEC66AF9
:10577000022A83ED016A00F0BB8091ED086A9DED7D
:105780000C5A25EE866AA5EE076AB0EE675AA6EEB9
:10579000265ABDEEC56A16EE10EA16EE106AAE4540
:1057A000A8BF2E467045C8BF064606EE106AB8EE82
:1057B000C66A032A83ED026A00F09A8091ED0C6AB2
:1057C0009DED0D5A25EE866AA5EE076AB0EE675A82
:1057D000A6EE265ABDEEC56A16EE10EA16EE106A5F
:1057E000AE45A8BF2E467045C8BF064606EE106AF5
:1057F000B8EEC66A042A83ED036A79D091ED106A87
:105800009DED0E5A25EE866AA5EE076AB0EE675A40
:10581000A6EE265ABDEEC56A16EE10EA16EE106A1E
:10582000AE45A8BF2E467045C8BF064606EE106AB4
:10583000B8EEC66A052A83ED046A59D091ED146A60
:105840009DED0F5A25EE866AA5EE076AB0EE675AFF
:10585000A6EE265ABDEEC56A16EE10EA16EE106ADE
:10586000AE45A8BF2E467045C8BF064606EE106A74
:10587000B8EEC66A062A83ED056A39D091ED186A3A
:105880009DED105A25EE866AA5EE076AB0EE675ABE
:10589000A6EE265ABDEEC56A16EE10EA16EE106A9E
:1058A000AE45A8BF2E467045C8BF064606EE106A34
:1058B000B8EEC66A072A83ED066A19D091ED1C6A14
:1058C0009DED115A65EE865AE7EE055AE6EEA57A89
:1058D000FDEEE77A17EE901A8D42A8BF0D4688427A
:1058E000C8BF054607EE905AF8EEE77AC3ED077A8F
:1058F0002FB922B19200D649D64828F0A0FCD64B49
:105900001B68002B40F0AE84D44B1B7893B19BF8FE
:10591000000060B1CF4ED24F0025E8B23B68B6EC34
:10592000010A98479BF8000001358542F5DBCD4B15
:105930001B689847CC4B1B78072B00F0428601234D
:1059400084F8003113B0BDEC0A8BBDE8F08FC74B73
:105950001B78013BDBB2FFF710BAC54B02934FF443
:105960007A751B68B5FBF3F3C3EB4315C149DFF848
:10597000388391F80190BC49B8F906000F7803EB21
:105980008503DD00ADB2AE4201F09386DBF88810EE
:10599000BBF93CE0DBF86C304A1C07EE90EA73443C
:1059A000012ACBF88820CBF86C30F8EEE77A01F0CA
:1059B0008D86DBED1E5ADBED206A07EE102A37EEEE
:1059C000E56AB8EEC75A012E86EE057A37EE257ADB
:1059D00077EEC77A8BED1F7AE7EE866A8BED1E7A3B
:1059E000F0EE667ACBED216ACBED206A02F05E80A4
:1059F000DBF89C10BBF93EE0DBF870304A1C07EE88
:105A000090EA7344012ACBF89C20CBF87030F8EE72
:105A1000E77A01F07686DBED235ADBED256A07EEA7
:105A2000102A37EEE56AB8EEC75A012E86EE057ADF
:105A300037EE257A77EEC77A8BED247AE7EE866A21
:105A40008BED237AF0EE667ACBED266ACBED256AF4
:105A500002F05580DBF8B010BBF940E0DBF87430A1
:105A60004A1C07EE90EA7344012ACBF8B020CBF829
:105A70007430F8EEE77A01F05F86DBED285ADBED53
:105A80002A6A07EE102A37EEE56AB8EEC75A012EE9
:105A900086EE057A37EE257A77EEC77A8BED297A8E
:105AA000E6EE276A8BED287AF0EE667ACBED2B6A6C
:105AB000CBED2A6A02F04C80A8F80600BBF8B4309F
:105AC000694A013B1778ABF8B43002990023072FDD
:105AD0004B608B60CB607FF444A9F8F7CFFBDFF815
:105AE000C88194F828310493A0EB0A00A8F80000BC
:105AF000002B3FF43CA9013B84F8283113B0BDECE6
:105B00000A8BBDE8F08F94ED577AB1F90000D4ED1F
:105B1000586AB1F902E0584AF4EEC76A80EAE073C5
:105B20008EEAEE71A3EBE073F1EE10FAA1EBEE71E9
:105B3000B4BFB0EE476AB0EE666A8B42B8BF0B46A0
:105B400007EE103A1378B8EEC77A27EE287A002BC2
:105B500040F00682494BD3ED005AF4EECA5AF1EEFA
:105B600010FA40F19087B7EE005A75EE654ADFED06
:105B7000446A9FED445A444B36EEC77A24EE855A68
:105B8000D3ED006AE7EE055A65EEA65AF5EEC05A67
:105B9000F1EE10FA40F2F784C9EEA56AB7EE007A8A
:105BA000F0EE475AE6EE665AF0EE656AF4EEC76A22
:105BB000F1EE10FA88BFF0EE476AF5EEC06AF1EE3A
:105BC00010FAB8BFF0EE6A6A304B93ED007A67EED8
:105BD000877AA7EEA68AFFF7B1B92D4B2D4C19682D
:105BE0002D4ADFF8C48094F80031C9691288A8F8FA
:105BF0000010A8F80220002B3EF434AF03F0FCF9AB
:105C0000002384F80031184B1B78072B7EF42AAF51
:105C1000F8F734FB8246FEF727BF204B204A2B447F
:105C200093ED007AD2ED007A1E4B67EE277AF7EEFD
:105C3000006AF4EEE67AF1EE10FA93ED007A88BF8E
:105C4000F0EE667A67EE877A27EE888AFFF727BA42
:105C5000084F0020785E0020204A0020505B002082
:105C60003C58002044580020F06100206C60002067
:105C7000685B0020545B0020BC4E0020C44E002016
:105C800000003443610BB63BB84E0020B44E0020F8
:105C9000B8670020942200202A440020F02300202E
:105CA000AC4E0020A84E0020F4610020D94BDFF854
:105CB000B8B31B789BF80020DD077FF51AAE002AE9
:105CC0003FF41DAED4ED583A94ED574AD24BD4ED83
:105CD000627A93ED005A94ED617AD4ED555A94EDC1
:105CE000546ACE49CE4BF4EEC43AF3EE046AF1EEB8
:105CF00010FA77EEA64A00F15B8791ED026A26EE74
:105D0000656AB0EE674AA6EE074AB4EEE44A34EE9E
:105D1000666AF1EE10FA48BFB0EE456A012A83EDDB
:105D2000006A3FF4ECAD91ED066A26EE656AB0EECE
:105D3000674AA6EE074AB4EEE44A34EE666AF1EE2C
:105D400010FA48BFB0EE456A022A83ED016A3FF4BB
:105D5000D6AD91ED0A6A26EE656AB0EE674AA6EE08
:105D6000074AB4EEE44A34EE666AF1EE10FA48BF30
:105D7000B0EE456A032A83ED026A3FF4C0AD91EDAF
:105D80000E6A26EE656AB0EE674AA6EE074AB4EEE2
:105D9000E44A34EE666AF1EE10FA48BFB0EE456AA6
:105DA000042A83ED036A3FF4AAAD91ED126A26EE50
:105DB000656AB0EE674AA6EE074AB4EEE44A34EEEE
:105DC000666AF1EE10FA48BFB0EE456A052A83ED27
:105DD000046A3FF494AD91ED166A26EE656AB0EE62
:105DE000674AA6EE074AB4EEE44A74EE666AF1EE3C
:105DF00010FA48BFF0EE456A062AC3ED056A3FF483
:105E00007EADD1ED1A6A66EEE56AB0EE674AA6EE9F
:105E1000874AB3EE046AB4EEE44A74EE466AF1EEE1
:105E200010FA48BFF0EE456A072AC3ED066A3FF450
:105E300066ADD1ED1E6A66EEE55AE5EE877AF4EEC0
:105E4000E74A77EEC67AF1EE10FAC8BFF0EE457A6F
:105E5000C3ED077A53E5734BC7ED00AA1B68934265
:105E6000BFF6ACA8704B1A88002384F86831002A6A
:105E700041F015846D4A6E4B1178186881F001016C
:105E8000F3F710FEFFF7A2B86A4EDFF8E08106F2E2
:105E90004C7506F5F767F6EC017A9BED080ADBF81E
:105EA0007837F8EEE77A284627EE800A9847A5F17A
:105EB000E000DBF898369847A5F17000DBF808376A
:105EC0009847D6F85806DBF8B83098472435AF42E3
:105ED000A8EC010ADFD1FEF73FBF4E490978C80799
:105EE00003D45549098BA4F88C11544954480988A6
:105EF00090ED037A07EE901AF8EEE77AB4EEE77ABF
:105F0000F1EE10FA40F20C864E48008807EE900A37
:105F1000F8EEE77AB4EEE77AF1EE10FAC0F2D08547
:105F200049484A49D0ED006A91ED006A4848C4EDFD
:105F3000646ABCEEC75A76EE665A15EE101AC4EDC6
:105F4000626AC4ED615A84ED656AA4F88C1101217E
:105F5000D0ED006A84F8981177EE677AFFF730B9D0
:105F60003C4B93ED005AB5EEC05AF1EE10FA40F3F7
:105F70000A83394BD3ED006AF5EEC06AF1EE10FAF0
:105F800040F3018336EEC77A66EE695A87EE266AD9
:105F9000C5EE856AB7EE007AB4EEC76AF1EE10FA84
:105FA00088BFB0EE476AB5EEC06AF1EE10FA76EE41
:105FB000876AB8BFB0EE6A6A66EE266AF6E5274AD7
:105FC00092ED007AF0EEE76AF4EEC76AF1EE10FAAD
:105FD0007FF786A8224A92ED007AF0EECC6AF4EEC2
:105FE000C76AF1EE10FA7FF77BA81E4A98ED007A97
:105FF000D2ED006AB0EEC77AB4EEE67AF1EE10FAAE
:106000007FF56EA801220399C4F86C1184F8682109
:10601000FFF76AB860620020044F0020284F00207C
:10602000785E0020D84E00202CB200202EB2002036
:1060300030B20020E4A70020F85C0020BC4F002014
:10604000EC620020BE4F0020A84F002048600020D6
:10605000C44F0020B84E0020C04E0020EC4E00205F
:10606000E84E0020F04E0020D16100206C5B002043
:106070000299724BD1ED017A93ED007AF0EEE77A56
:10608000F4EEC77AF1EE10FA7EF5A0AFD1ED027A08
:10609000F0EEE77AB4EEE77AF1EE10FA7EF796AF1B
:1060A000D1ED037AF0EEE77AB4EEE77AF1EE10FA8A
:1060B0007EF78CAF624B1B689A077FF5D3AE6149C0
:1060C000614BB3F90C20B1F900E06048AEEB020E71
:1060D00000688EEAEE72A2EBEE728242BEF676AFF6
:1060E000B3F90E30B1F90220D21A82EAE273A3EBBF
:1060F000E27398427EF76AAFB4E6554B98ED007AAA
:10610000D3ED006AB0EEC77AB4EEE67AF1EE10FA9B
:106110007EF7FCAFFEF7F7BF07EE103A4D4BDFF806
:1061200040811B78C4F81061B8EEC77AF7EE006AB8
:10613000132B86EE879AB8F90400B4F814519BED3E
:10614000080A01F03882444B444A93ED001A93ED5B
:10615000053A93ED122A93ED176AD3ED091A93EDE0
:106160000E4AD3ED015AD3ED063A93ED0A7A93ED38
:106170000F5AD3ED132AD3ED186AD3ED044AD3EDA9
:10618000030A67EE897A69EE288A29EE088AA1EE69
:10619000273A02EB85060021A2EE286AC4F8041112
:1061A000C4F80811A1EE884AE5EEA73AA7EE085A0E
:1061B00093ED167AD3ED0D5A93ED021AD3ED0C1A26
:1061C00086ED003AE2EEA86A64EEC34A27EE467A0C
:1061D00093ED0B2AD3ED152A86ED204AE0EEC33A63
:1061E00065EEC45A93ED143AC3ED053AE1EE274A41
:1061F000F0EE477AA1EEC45AE2EE085AE2EEC66A21
:10620000E3EE287AC3ED064A83ED0E5AC3ED0F5A2A
:1062100086ED406AC3ED176AC3ED187AC4F80C1115
:10622000013505F01F05A4F81451A8F80400FEF785
:1062300076BCB0EE465AFEF7FCBF00BFE44E00202D
:10624000CC740020B074002078600020E04E002064
:10625000F04E0020F0610020045600208053002002
:10626000F4610020B44B1B78192B07D80121B34AE5
:1062700001FA03F31A40002A41F07884B04BB14E82
:10628000B14F01931B689D061CD5FB7AFF2B04D0F0
:10629000AE4A12789A4201F2F380B7F90880FB7D8A
:1062A000A6F80080FF2B04D0A84A12789A4201F287
:1062B000E280B7F914507580082022F099FF002879
:1062C00040F03586B7F90600B6F900C0B6F902E02D
:1062D000B7F91210B7F91E20B6F90450B7F9043017
:1062E000B6F906806045A8BF60467145A8BF7146F3
:1062F000AA42A8BF2A469C45A8BF03463380B7F9E7
:106300001030B6F908009E45B8BF1946B7F92A30D3
:106310007180B7F91C10B7F934E04345A8BF434674
:106320008D42B4BF0D461546B7F93620B580B7F992
:106330002850B6F90A108242A8BF0246A845ACBF51
:106340009846A846B7F94230B6F90C50A6F8068030
:106350008B42A8BF0B467045ACBF10467046B7F9DC
:106360004E203081B7F94000B6F90EE0AA42A8BF2E
:106370002A468842C8BF0346B7F95A00B7F94C10FD
:1063800073817045B7F95830714FA8BF70469E456C
:10639000A8BF0346A942D8BF1146B181F381BB898A
:1063A0002BB3DFF8BC81DFF8BCA1DFF89C9108F1CA
:1063B0001005B8F9023000EE103A5046B8EEC00AA7
:1063C000F2F75EF925F04AFEB9F90430B9F9062072
:1063D00000B298420AF1240A09F10C0903DB824257
:1063E0001346A8BF034628F8023FA845E1D1524B07
:1063F0001B78013B182B74D8DFE813F061007300A1
:10640000730019007300730073007C08730073003D
:106410007300730073009C087300730073007300B3
:10642000730019008A08730073009C086100494BCF
:10643000B6F908101A6802B111609B69B6F90A2012
:1064400003B11A60019B1B689A0601F1ED860222D6
:106450000492D9027FF558AAFE7B112E3FF654AA6A
:106460003D4BDDF810901D4633F9163000EE103A22
:106470004846B8EEC00A06F1010806F10E0708F01A
:1064800047FB4B465FFA88F89E1BFFB2A94600E027
:10649000A84608F1010508EB0600B8F1120FEDB2AD
:1064A000C0B23FF431AA39F9183000EE103AB8EE14
:1064B000C00A08F02DFBBD42EAD1FFF725BABB7B2D
:1064C000002B42F07B80254B1B7813F0010342F038
:1064D0007580204A1268002A02F04F84136001235D
:1064E0000493019B1B68980603D4134A1278052A6B
:1064F000AFD1049A13460233551CDBB21046EDB2FD
:106500000493B6F9003000EE103AB8EEC00A08F075
:10651000FFFAB6F9023000EE103A2846B8EEC00A8B
:1065200008F0F6FA019B1B6893E725F097FD29F820
:106530001600FEF7FFBB00BF244A002032413003A3
:10654000785B0020685E0020305000206C470020FF
:106550008C6E00209C6E002004A60020606200204B
:10656000665E00201C4800200000000095ED007AC7
:106570000BEB4602B8EEC78A928F29F8162028EE58
:10658000278AFEF7B5BB5FED086AFFF71DBB59020E
:106590003FF55AA8FFF75CB8F7F770FEA94B069ACB
:1065A0001B78DFF8A482801A012BA8F8020000F003
:1065B0007682072B7EF4D2ADF7F760FE0290FEF7ED
:1065C000CFBDF7F75BFE029A9F4B801AD880FFF78A
:1065D000B6B9002F41F0628191ED006A9DED0A5A33
:1065E0009A4B25EE866AA5EE076AB0EE675AA6EECC
:1065F000265ABDEEC56A16EE107A16EE106AAF4244
:10660000A8BF2E46B842C8BF064606EE106AB8EECE
:10661000C66A012A83ED006A3FF46CA991ED046A11
:106620009DED0B5A25EE866AA5EE076AB0EE675A15
:10663000A6EE265ABDEEC56A16EE107A16EE106A60
:10664000AF42A8BF2E46B842C8BF064606EE106A43
:10665000B8EEC66A022A83ED016A3FF44BA991EDB8
:10666000086A9DED0C5A25EE866AA5EE076AB0EE23
:10667000675AA6EE265ABDEEC56A16EE107A16EED9
:10668000106AAF42A8BF2E46B842C8BF064606EE03
:10669000106AB8EEC66A032A83ED026A3FF42AA99B
:1066A00091ED0C6A9DED0D5A25EE866AA5EE076AFE
:1066B000B0EE675AA6EE265ABDEEC56A16EE107AFF
:1066C00016EE106AAF42A8BF2E46B842C8BF0646B3
:1066D00006EE106AB8EEC66A042A83ED036A3FF438
:1066E00009A991ED106A9DED0E5A25EE866AA5EE78
:1066F000076AB0EE675AA6EE265ABDEEC56A16EED8
:10670000107A16EE106AAF42A8BF2E46B842C8BF34
:10671000064606EE106AB8EEC66A052A83ED046ADC
:106720003FF4E8A891ED146A9DED0F5A25EE866AB4
:10673000A5EE076AB0EE675AA6EE265ABDEEC56A08
:1067400016EE107A16EE106AAF42A8BF2E46B84277
:10675000C8BF064606EE106AB8EEC66A062A83ED82
:10676000056A3FF4C7A891ED186A9DED105A25EE11
:10677000866AA5EE076AB0EE675AA6EE265ABDEE07
:10678000C56A16EE107A16EE106AAF42A8BF2E4602
:10679000B842C8BF064606EE106AB8EEC66A072AB7
:1067A00083ED066A3FF4A6A891ED1C6A9DED115A8F
:1067B00065EE865AE7EE055AE6EEA57AFDEEE77A33
:1067C00017EE901A8D42A8BF0D468842C8BF0546F5
:1067D00007EE905AF8EEE77AC3ED077AFFF789B82B
:1067E0001B4A517900293EF4B0AD1A4909780029B5
:1067F0003EF4ABAD1278DFED184A07EE902A174A47
:10680000B8EE677A128807EE901A06EE902AF8EE34
:10681000E77AF8EE666A67EE277AB7EE007AC7EE97
:10682000A63AF4EEE43AF1EE10FA88BFF0EE643ADC
:10683000F4EEC73AF1EE10FAB8BFF0EE473AFEF7C1
:1068400086BD00BFF0610020F4610020785E00206A
:10685000B8740020EA620020713DAA3FD462002093
:10686000002E00F05482002F41F0D286C049BEF1C4
:10687000000F41F00F8591ED006ADDED0A4ABD4B36
:1068800025EE866ABDEEC55AA4EE876A15EE100A9B
:10689000B0EE675AA6EE265ABDEEC56A16EE107A1D
:1068A00016EE106AAF42A8BF2E46B842C8BF0646D1
:1068B00006EE106AB8EEC66A012A83ED006A3FF45C
:1068C00019A891ED046A9DED0B5A25EE866AA5EE96
:1068D000076AB0EE675AA6EE265ABDEEC56A16EEF6
:1068E000107A16EE106AAF42A8BF2E468742B8BF94
:1068F000064606EE106AB8EEC66A022A83ED016A01
:106900003EF4F8AF91ED086A9DED0C5A25EE866ACB
:10691000A5EE076AB0EE675AA6EE265ABDEEC56A26
:1069200016EE107A16EE106AAF42A8BF2E468742C6
:10693000B8BF064606EE106AB8EEC66A032A83EDB3
:10694000026A3EF4D7AF91ED0C6A9DED0D5A25EE2B
:10695000866AA5EE076AB0EE675AA6EE265ABDEE25
:10696000C56A16EE107A16EE106AAF42A8BF2E4620
:106970008742B8BF064606EE106AB8EEC66A042A19
:1069800083ED036A3EF4B6AF91ED106A9DED0E5AA9
:1069900025EE866AA5EE076AB0EE675AA6EE265A7D
:1069A000BDEEC56A16EE107A16EE106AAF42A8BFA9
:1069B0002E468742B8BF064606EE106AB8EEC66A93
:1069C000052A83ED046A3EF495AF91ED146A9DEDBE
:1069D0000F5A25EE866AA5EE076AB0EE675AA6EE54
:1069E000265ABDEEC56A16EE107A16EE106AAF4250
:1069F000A8BF2E468742B8BF064606EE106AB8EE1C
:106A0000C66A062A83ED056A3EF474AF91ED186AF2
:106A10009DED105A25EE866AA5EE076AB0EE675A1C
:106A2000A6EE265ABDEEC56A16EE107A16EE106A6C
:106A3000AF42A8BF2E468742B8BF064606EE106A90
:106A4000B8EEC66A072A83ED066A3EF453AF91EDAD
:106A50001C6A9DED115A65EE865AE7EE055AE6EE80
:106A6000A57AFDEEE77A17EE901A8D42A8BF0D4683
:106A70008842D8BF284607EE900AF8EEE77AC3EDC1
:106A8000077AFEF736BF3C4BD3ED005AFFF77EB8CE
:106A9000F7F7F4FB0690FEF779B9DFF81081F7F706
:106AA000EDFB364AD4F87C3112680290C31A9A1A68
:106AB000C4F87C01A8F80430A8F80620FEF750BB03
:106AC000B4F88C01884240F245852D482D49D0ED1F
:106AD000007A91ED007A2C48C4ED647A77EE676A0B
:106AE000C4ED627A0121C4ED616A84ED657AD0ED6E
:106AF000006ADFED267A84F89811FEF761BB244B1B
:106B00001B88002B40F04585224A234B11781868DA
:106B1000F2F7C8FFD4F86C21039B9A1AFEF725BA46
:106B20001E491F48D1ED006A1E4990ED006A0978A0
:106B3000C4ED646A84ED656A002940F0B78476EE9E
:106B4000C65AF0EE466ABCEEC76A1748C4ED615AF1
:106B500016EE101AC4ED626AA4F88C11FF21D0ED74
:106B6000006A84F8981177EEC77AFEF729BB00BF58
:106B7000284F0020785E0020B84E0020A060002042
:106B8000A84F002048600020C44F002000000000F3
:106B90002CB200202EB2002030B20020D85E00209F
:106BA000AC4F002048580020C04F0020F461002066
:106BB000D1ED015A65EEC65AB0EE674AA5EE874A96
:106BC000B4EEE44A74EE665AF1EE10FA48BFF0EE05
:106BD000455A012AC3ED005A3EF491AED1ED055A53
:106BE00065EEC65AB0EE674AA5EE874AB4EEE44AAF
:106BF00074EE665AF1EE10FA48BFF0EE455A022ADA
:106C0000C3ED015A3EF47BAED1ED095A65EEC65A8A
:106C1000B0EE674AA5EE874AB4EEE44A74EE665ACF
:106C2000F1EE10FA48BFF0EE455A032AC3ED025ABE
:106C30003EF465AED1ED0D5A65EEC65AB0EE674A28
:106C4000A5EE874AB4EEE44A74EE665AF1EE10FA05
:106C500048BFF0EE455A042AC3ED035A3EF44FAE46
:106C6000D1ED115A65EEC65AB0EE674AA5EE874AD5
:106C7000B4EEE44A74EE665AF1EE10FA48BFF0EE54
:106C8000455A052AC3ED045A3EF439AED1ED155AE2
:106C900065EEC65AB0EE674AA5EE874AB4EEE44AFE
:106CA00074EE666AF1EE10FA48BFF0EE456A062A05
:106CB000C3ED056A3EF423AED1ED196A66EEC66AED
:106CC000B0EE674AA6EE874AF3EE045AB4EEE44A01
:106CD00074EE656AF1EE10FA48BFF0EE456A072AD5
:106CE000C3ED066A3EF40BAED1ED1D6A26EEC66A10
:106CF000E6EE077AF4EEE47A77EEE57AF1EE10FA52
:106D0000B8BFF0EE457AC3ED077AFEF7F8BDC94982
:106D1000BEF1000F41F04A8191ED006ADDED0A4AB3
:106D2000C54B25EE866ABDEEC55AA4EE876A15EE00
:106D3000100AB0EE675AA6EE265ABDEEC56A16EEE8
:106D400010EA16EE106AAE45A8BF2E467045C8BFC1
:106D5000064606EE106AB8EEC66A012A83ED006A9E
:106D60003EF4C6AD91ED046A9DED0B5A25EE866AA0
:106D7000A5EE076AB0EE675AA6EE265ABDEEC56AC2
:106D800016EE10EA16EE106AAE45A8BF2E468645EE
:106D9000B8BF064606EE106AB8EEC66A022A83ED50
:106DA000016A3EF4A5AD91ED086A9DED0C5A25EE01
:106DB000866AA5EE076AB0EE675AA6EE265ABDEEC1
:106DC000C56A16EE10EA16EE106AAE45A8BF2E464A
:106DD0008645B8BF064606EE106AB8EEC66A032AB4
:106DE00083ED026A3EF484AD91ED0C6A9DED0D5A7F
:106DF00025EE866AA5EE076AB0EE675AA6EE265A19
:106E0000BDEEC56A16EE10EA16EE106AAE45A8BFD2
:106E10002E468645B8BF064606EE106AB8EEC66A2C
:106E2000042A83ED036A3EF463AD91ED106A9DED93
:106E30000E5A25EE866AA5EE076AB0EE675AA6EEF0
:106E4000265ABDEEC56A16EE10EA16EE106AAE4579
:106E5000A8BF2E468645B8BF064606EE106AB8EEB5
:106E6000C66A052A83ED046A3EF442AD91ED146AC8
:106E70009DED0F5A25EE866AA5EE076AB0EE675AB9
:106E8000A6EE265ABDEEC56A16EE10EA16EE106A98
:106E9000AE45A8BF2E468645B8BF064606EE106A28
:106EA000B8EEC66A062A83ED056A3EF421AD91ED7F
:106EB000186A9DED105A25EE866AA5EE076AB0EEB7
:106EC000675AA6EE265ABDEEC56A16EE10EA16EE11
:106ED000106AAE45A8BF2E468645B8BF064606EEE8
:106EE000106AB8EEC66A072A83ED066A3EF400AD62
:106EF00091ED1C6A9DED115A65EE865AE7EE055A32
:106F0000E6EEA57AFDEEE77A17EE901A8D42A8BF5D
:106F10000D468842D8BF284607EE900AF8EEE77A79
:106F2000C3ED077A002F7EF4EAACFEF7E2BC94F8DA
:106F3000C031012B01F0A184404B97F916005A880B
:106F400097F90AE01B883E4910FB03F31EFB02F28F
:106F500081FB020C81FB0301D217DB17C2EB2C1261
:106F6000C3EB211342441D4432807580FFF7AAB958
:106F7000344FD4ED017A94ED006A38887B6977EE5E
:106F8000A77AF0EE006AB0EE677AA6EE267A0138AC
:106F900004EBC002D6EE267A083A1033F6EE003A39
:106FA00027EE237A67EEA37A84ED207AC4ED217A66
:106FB000254C274604F1800192ED027A92ED036A96
:106FC000D7ED036AD7ED027A53ED014A13ED025A69
:106FD00037EE674A76EEC65A77EE277AE4EE845AA1
:106FE0000138A2F10802E5EE047A07F1080703F17F
:106FF000080336EE267A01F10801E4EE877AE5EE21
:10700000475A67EEA37A25EEA37AC1ED007A81EDA7
:10701000017AD1D1142E7DF436AEF7F72FF9029B09
:10702000DFF82880C01AA8F80200D4F81851FDF73C
:107030002ABE00BF284F0020785E0020B0740020D8
:107040001F85EB516853002094220020F46100203A
:10705000DFF8949499F80020900801F08986DFF811
:107060008CE400F1010C4FEA4C1C0EEB0C070EF106
:107070002003AEF1700113ED076A53ED056A13EDBD
:10708000037A53ED017A53ED025A13ED084A53ED9A
:10709000064A13ED045A26EE066A66EEA66A27EE45
:1070A000077A67EEA77AA4EE046A20339F42E4EEE3
:1070B000A46A01F11001A5EE057AE5EEA57AF1EEDC
:1070C000C65AB1EEE66AF1EEC76AB1EEE77A41ED73
:1070D000085A01ED076A41ED066A01ED057ACAD149
:1070E000ACF1200CE64404EB001012F0030318BFCF
:1070F0000EF1080E0FD05EED017A1EED027A67EEFA
:10710000A77A013BE7EE077A0EF1080EB1EEE77AB7
:10711000A0EC017AEFD1142E01F0FE850135C4F800
:107120001851FDF71DBDE34FE348BA68B98924F053
:107130001BF8E24B1E78142E01F07885D4F8185114
:107140000135C4F8185114E7DA4FB7F800E0D7F862
:1071500004C04FEA5E084FEA880204EB8E055FEA3E
:10716000DE0E04EB020300F0A08010320EF1010EDF
:10717000D34803EB0E1E2A4410330CF1100605F120
:10718000100111ED031A11ED042A50ED041A50ED0F
:10719000030A11ED015A11ED026A50ED025A50ED49
:1071A000014A52ED042A52ED033A52ED026A13ED00
:1071B000043A13ED034A13ED027A53ED017A12ED0E
:1071C000010A71EE828A30EE818A40ED048A00ED78
:1071D000038A75EE868A34EE858A40ED028A00EDD8
:1071E000018A73EE228A34EE238A43ED048A03ED8A
:1071F000038A77EE268A37EE808A43ED028A03ED12
:10720000018A33EEC44A31EEC22A56ED033A70EEDB
:10721000C11A32EEC33A23EEC28A56ED042A61EE59
:10722000A30A22EEC41AA1EEA28A10339E4563EE91
:10723000221AA3EE231A00F1100006F11006E4EE64
:10724000231A01F1100102F11002E2EE220A01ED0F
:10725000078A41ED080A02ED081A42ED071A35EED9
:10726000C66A36EEC77A74EEC55A56ED056A16ED53
:10727000065A70EE677A25EEA63A66EEC63A25EE15
:10728000674A67EE054AE5EE853AA6EE053AA7EEAF
:10729000264AE7EEA64A01ED063A41ED053A02ED2F
:1072A000064A42ED054A7FF46CAF1FFA88F8624641
:1072B000414681481AF084FC41467A6828461AF013
:1072C0007FFC7E4B1B78142B7FF4AFAEA5E6D4F881
:1072D0001CC1B4F814917B4BC9F120085FFA88F8FF
:1072E00009EB4C1703EB87075FEA980301F08484EE
:1072F000013318017449724A07EB000E07F11003BD
:1073000013ED024A13ED035A13ED016A13ED047AEB
:1073100051ED024A51ED035A51ED016A51ED047AE3
:1073200064EE244A65EE255A66EE266A67EE277AF1
:1073300010339E4542ED024A42ED035A42ED016A86
:1073400042ED047A01F1100102F11002D8D15F4937
:10735000A0F11002174401EB020E224418F00303BF
:1073600009D0B7EC017AFEEC017A67EE277A013B8F
:10737000E2EC017AF5D1B9F1000F41F0C980142E89
:107380007DF481ACF6F77AFF029BDFF86481D4F8D4
:107390001851C01AA8F80200FDF775BCD4F81C718A
:1073A0004B4B4C4ADFED4C7AD2ED008A4B4AF90048
:1073B0000B44F8EE688A9B8809EE103A643BC82BB0
:1073C000A8BFC82368EEA78AF8EE497A782BB8BF21
:1073D000782368EEA78A07EE903A3944B0EE680A3F
:1073E00002EB8108B8EEE78A24F084FEB8EEC99A71
:1073F000F0EE409AB0EE680A24F0DEFD38EE097A2D
:1074000079EE487A28EE098A67EE877AB7EE006A45
:1074100088EE277A142EF8EE007A77EE076A60EE8F
:10742000277A89EEA67A77EE065A36EE477AC6EEC6
:10743000256A67EEA67A27EE267AC8ED006A88EDFF
:10744000047AC8ED026AC8ED017AC8ED037A01F04A
:107450007384234B194A013783FB073CACEBE77C71
:107460000CEB4C0C0135A7EB0C0C1678C4F818513A
:10747000C4F81CC12DE71B4A32F91350FEF71BBF9D
:10748000184A32F91380FEF70ABFF6F7F7FE0B4BE6
:1074900002901E78142E05BFDFF85480D4F81851DE
:1074A000D4F81851A8F80050FDF742BB76EE665AA2
:1074B000FFF749BB6853002094220020F0610020B0
:1074C000A4220020805300201055002000550020E9
:1074D00080550020685B002027D4D23630AF0020D2
:1074E0005655555504A60020625300201423002051
:1074F000F4610020D54BB6F906101A6802B111608C
:107500009B69B6F90820002B7EF49BAFFEF79ABF6B
:10751000DFF88083002538F9023B00EE103AE8B22C
:10752000B8EEC00A013507F0F3FA042DF3D1049543
:10753000FEF7D7BFDFF86083002538F9023F00EE81
:10754000103AE8B2B8EEC00A013507F0E1FA062DAC
:10755000F3D1ECE7BE49BF48D1ED007ABE4990EDCA
:10756000007A0978C4ED647A84ED657A002901F027
:10757000CB8277EE676AB948C4ED627AC4ED616A7E
:10758000FF21D0ED006ADFEDB67A84F89811FDF79F
:1075900017BEB4494B69002B3DF4E7ACB248B34B7E
:1075A000008893FBF0F00B684FF0010E186081F833
:1075B00011E0FDF7DABCAE4EAE4F96ED004A96ED07
:1075C000057AD6ED014A96ED066AD6ED046A96ED87
:1075D000035AD6ED025A67EE897A07EB8503A4EECB
:1075E000277AA4EEA76A66EEC76AA5EE476AE5EEBB
:1075F000A76A20EE070A86ED056AC6ED066A83EDE6
:10760000007A29EE088A24F029FD69EE288AD6ED51
:107610000E5AD6ED176A96ED091AD6ED121A96EDA6
:107620000F5A96ED187A96ED0A2AD6ED132A96EDA2
:107630000D6AD6ED167A96ED0C3AD6ED0B3A96ED2C
